:100000000C94D5150C9404160C9404160C94041638
:100010000C9404160C9404160C9404160C940416F8
:100020000C9404160C9404160C9404160C940416E8
:100030000C9404160C9404160C9404160C94643A54
:100040000C9404160C9404160C9404160C940416C8
:100050000C9404160C94523B0C9404160C94041645
:100060000C9404160C94FA8D0C9404160C94268EA1
:100070000C9404160C94815B0C9404160C940416D6
:100080000C940F370C9404160C9404160C9404165C
:100090000C9404160C9404160C9404160C94041678
:1000A0000C9404160C9404160C9404160C94041668
:1000B0000C9404160C9404160C9404160C94041658
:1000C0000C9404160C9404160C9404160C94041648
:1000D0000C9404160C9404160C9404160C94041638
:1000E0000C940416792E9A2E9E2EB52E09300930C6
:1000F000093009300930093009300930E32EFF2E6C
:100100000930093009300930093009300930093027
:100110000D2FDE2E0930D22ED82E093009300930AD
:10012000242F09302E2F452F832E4F2F5A2F9D2FEE
:1001300045307A307F3064308930FC30FC306430B8
:10014000AC30FC30B030B530CA30CF30933098305E
:10015000A2306430A730FC304A308E30D430FC30CE
:10016000FC30D930546865205265706C69636174E5
:1001700030720083048800000014008C000000002E
:100180000000000030F8FFFF000000000000000049
:100190008E000000000000000000000000000000D1
:1001A000000000000057290400188304DC0500004B
:1001B00014008403690100001400901F891F95003A
:1001C00000000046696E64207468652034206B6E00
:1001D0006F6273206F6E20009501000000746865E7
:1001E00020626F74746F6D206F66207468652020C4
:1001F00020009501000000706C6174666F726D20C4
:10020000616E64207475726E20746F009507000033
:10021000007469676874656E20636F6D706C6574D7
:10022000656C792E00950000000049276D20676FEE
:10023000696E6720746F206D6F76652020200095B1
:1002400001000000746865206578747275646572D9
:1002500020746F202020202000950100000076618E
:1002600072696F757320706F736974696F6E732034
:100270002020009507000000666F722061646A7597
:1002800073746D656E742E2E2E009500000000496B
:100290006E206561636820706F736974696F6E2C7E
:1002A00020202000950100000077652077696C6CA4
:1002B000206E65656420746F202020202000950149
:1002C00000000061646A7573742074776F206B6E30
:1002D0006F627320617420009507000000746865E8
:1002E0002073616D652074696D652E2E2E0095005A
:1002F0000000004E6F7A7A6C657320617265206130
:100300007420746865202000950100000072696700
:10031000687420686569676874207768656E202056
:1003200020009501000000796F752063616E206ADE
:1003300075737420736C6964652061009507000013
:10034000007368656574206F662070617065722E39
:100350002E2E0095000000006265747765656E20A2
:10036000746865206E6F7A7A6C65202000950100B4
:100370000000616E642074686520706C6174666F43
:10038000726D2E20202000950100000047726162EE
:100390002061207368656574206F6620202020200E
:1003A000009507000000706170657220746F206115
:1003B00073736973742075732E00950200000050EA
:1003C0006C6561736520776169740083048800003F
:1003D0000014008C0000000000000000000000007D
:1003E00000000000000000008E000000000000007F
:1003F00000D007000000000000000000000D4503D1
:10040000001884036901000014008CA531000094D9
:100410001B0000D007000000000000000000009555
:1004200002000000506C656173652077616974009B
:100430008E0000000000000000D007000000000057
:1004400000000000001D471C00188E00000000CABC
:10045000E4FFFFD00700000000000000000000C023
:100460008C0D00188E00000000C9E4FFFF000000A2
:100470000000000000000000000D4503001895007A
:1004800000000041646A75737420746865206672A8
:100490006F6E742074776F0095010000006B6E6FB3
:1004A000627320756E74696C2070617065722020B3
:1004B000200095010000006A75737420736C6964F4
:1004C0006573206265747765656E2000950700008E
:1004D000006E6F7A7A6C6520616E6420706C617456
:1004E000666F726D009502000000506C6561736567
:1004F0002077616974008E00000000CAE4FFFFD01D
:1005000007000000000000000000000D4503001877
:100510008EEF220000CAE4FFFFD0070000000000B9
:10052000000000000020651100188EF0220000C9B4
:10053000E4FFFF0000000000000000000000000DCC
:1005400045030018950000000041646A757374202B
:100550007468652072696768742074776F0095010C
:100560000000006B6E6F627320756E74696C207092
:10057000617065722020200095010000006A75738B
:100580007420736C69646573206265747765656E49
:10059000200095070000006E6F7A7A6C6520616E0E
:1005A0006420706C6174666F726D009502000000CB
:1005B000506C656173652077616974008EEF22006D
:1005C00000CAE4FFFFD007000000000000000000A8
:1005D000000D450300188EF6DBFFFFCAE4FFFFD0D5
:1005E0000700000000000000000000E05623001893
:1005F0008EF6DBFFFFC9E4FFFF00000000000000F3
:1006000000000000000D45030018950000000041A7
:10061000646A75737420746865206C6566742074F0
:10062000776F200095010000006B6E6F627320757C
:100630006E74696C207061706572202020009501D5
:100640000000006A75737420736C696465732062BE
:1006500065747765656E200095070000006E6F7AFF
:100660007A6C6520616E6420706C6174666F726D67
:10067000009502000000506C656173652077616928
:1006800074008EF7DBFFFFCAE4FFFFD00700000015
:10069000000000000000000D450300188E0000005F
:1006A000007A1A0000D007000000000000000000DF
:1006B000008A322000188E000000007A1A00000024
:1006C00000000000000000000000000D45030018BD
:1006D000950000000041646A757374207468652099
:1006E0006261636B2074776F200095010000006BDE
:1006F0006E6F627320756E74696C207061706572C4
:100700002020200095010000006A75737420736C2E
:1007100069646573206265747765656E200095076E
:100720000000006E6F7A7A6C6520616E6420706CD8
:100730006174666F726D009502000000506C656117
:1007400073652077616974008E000000007A1A00DA
:1007500000D007000000000000000000000D45036D
:1007600000188EEF2200007A1A0000D00700000067
:100770000000000000000020651100188EEF22002C
:10078000007A1A00000000000000000000000000D5
:10079000000D45030018950000000041646A757360
:1007A00074207468652072696768742074776F00BC
:1007B00095010000006B6E6F627320756E74696C3A
:1007C0002070617065722020200095010000006A91
:1007D00075737420736C69646573206265747765E2
:1007E000656E200095070000006E6F7A7A6C6520B8
:1007F000616E6420706C6174666F726D00950200AA
:100800000000506C656173652077616974008EF03B
:100810002200007A1A0000D007000000000000004B
:100820000000000D450300188E54DCFFFF7A1A000B
:1008300000D0070000000000000000000000282396
:1008400000188E54DCFFFF7A1A0000000000000040
:10085000000000000000000D450300189500000096
:100860000041646A75737420746865206C656674F1
:100870002074776F200095010000006B6E6F62732B
:1008800020756E74696C2070617065722020200084
:1008900095010000006A75737420736C6964657358
:1008A000206265747765656E200095070000006E14
:1008B0006F7A7A6C6520616E6420706C6174666F0B
:1008C000726D008E55DCFFFF7A1A0000D007000021
:1008D00000000000000000000D450300188E00001D
:1008E000000000000000D007000000000000000031
:1008F0000000911E1600188E00000000000000008D
:100900000000000000000000000000000D45030092
:10091000189500000000436865636B20746861747B
:100920002070617065722020202000950100000079
:100930006A75737420736C6964657320626577747B
:1009400065656E200095070000006E6F7A7A6C6511
:1009500020616E6420706C6174666F726D2E008908
:100960001F860088000302DC00860188010302DC88
:1009700000860088001F02640088011F0264008452
:100980000369010000140083048800000014008C37
:100990000000000000000000B8F7FFFF00000000AA
:1009A000000000008E000000000000000088FFFF33
:1009B000FF00000000000000005729040018830415
:1009C000DC0500001400901F8E1F23000028E5FFA7
:1009D000FF1801000000000000000000006F592116
:1009E0000018910000910100910300910400910012
:1009F0007F91017F91037F91047F860086008700AD
:100A00006400FFFF8D006400FFFF860186018701FF
:100A10006400FFFF8D006400FFFF8E1E230000288E
:100A2000E5FFFF500000000000000000000000B4DF
:100A30005300001888010A010388010401FF8E1E7B
:100A400023000027E5FFFF5000000000000000A089
:100A5000FFFFFF804F1200188C1E23000028E5FFC7
:100A6000FF50000000000000006000000086008EC3
:100A700031E0FFFFB8E9FFFFF000000000000000D8
:100A800000000000229C3200188E31E0FFFFB7E921
:100A9000FFFFF0000000E3FFFFFF000000001C5814
:100AA00000001889888E31E0FFFFB7E9FFFF78006A
:100AB0000000EDFFFFFF0000000060180000188E2E
:100AC00031E0FFFFB7E9FFFF78000000E3FFFFFF21
:100AD00000000000F22B0000188E7BD1FFFFB7E969
:100AE000FFFF780000009BFEFFFF00000000862F44
:100AF0003000188E31E0FFFF6EEDFFFF7800000040
:100B0000310000000000000012720B00188E31E06E
:100B1000FFFF6EEDFFFF78000000E3FFFFFF000026
:100B20000000F12B0000188E29D5FFFF6EEDFFFFAE
:100B3000780000009CFEFFFF00000000A5232400B9
:100B4000188E31E0FFFF25F1FFFF78000000300034
:100B500000000000000031C80800188E31E0FFFFDF
:100B600024F1FFFF78000000E3FFFFFF000000001A
:100B7000F12B0000188E29D5FFFF25F1FFFF78002B
:100B800000009CFEFFFF00000000A5232400188E3B
:100B900030E0FFFFDCF4FFFF7800000030000000D1
:100BA0000000000031C80800188E31E0FFFFDBF4C0
:100BB000FFFF78000000E3FFFFFF00000000F22BC2
:100BC0000000188E29D5FFFFDCF4FFFF780000003D
:100BD0009CFEFFFF00000000A5232400188E31E0DA
:100BE000FFFF92F8FFFF78000000300000000000D7
:100BF000000031C80800188E31E0FFFF93F8FFFFB6
:100C000078000000E3FFFFFF00000000F22B00006F
:100C1000188E29D5FFFF92F8FFFF780000009CFE98
:100C2000FFFF00000000A5232400188E31E0FFFF25
:100C300049FCFFFF780000003000000000000000C9
:100C400031C80800188E30E0FFFF49FCFFFF780034
:100C50000000E3FFFFFF00000000F22B0000188EF1
:100C600029D5FFFF4AFCFFFF780000009CFEFFFF34
:100C700000000000A5232400188E31E0FFFF0000D3
:100C8000000078000000300000000000000031C8C3
:100C90000800188E31E0FFFF00000000780000001F
:100CA000E3FFFFFF00000000F22B0000188E29D5A3
:100CB000FFFF00000000780000009CFEFFFF000026
:100CC0000000A5232400188E31E0FFFFB6030000CA
:100CD00078000000300000000000000031C808006B
:100CE000188E31E0FFFFB703000078000000E3FF3B
:100CF000FFFF00000000F22B0000188E28D5FFFF38
:100D0000B7030000780000009CFEFFFF0000000019
:100D1000A5232400188E31E0FFFF6E070000780045
:100D20000000300000000000000031C80800188EEC
:100D300031E0FFFF6D07000078000000E3FFFFFFD8
:100D400000000000F22B0000188E29D5FFFF6E076F
:100D50000000780000009CFEFFFF00000000A523BB
:100D60002400188E31E0FFFF240B00007800000003
:100D7000300000000000000031C80800188E31E08B
:100D8000FFFF250B000078000000E3FFFFFF0000DD
:100D90000000F12B0000188E28D5FFFF240B000067
:100DA000780000009CFEFFFF00000000A523240047
:100DB000188E31E0FFFFDB0E0000780000003000ED
:100DC00000000000000031C80800188E31E0FFFF6D
:100DD000DC0E000078000000E3FFFFFF00000000D1
:100DE000F12B0000188E29D5FFFFDB0E00007800E4
:100DF00000009CFEFFFF00000000A5232400188EC9
:100E000031E0FFFF92120000780000003000000087
:100E10000000000031C80800188E31E0FFFF921278
:100E2000000078000000E3FFFFFF00000000F12B4E
:100E30000000188E29D5FFFF9212000078000000F4
:100E40009CFEFFFF00000000A5232400188E30E068
:100E5000FFFF49160000780000003000000000008D
:100E6000000031C80800188E31E0FFFF491600006D
:100E700078000000E3FFFFFF00000000F12B0000FE
:100E8000188E29D5FFFF49160000780000009CFE4F
:100E9000FFFF00000000A5232400188EAEEEFFFF28
:100EA000A5F8FFFFF0000000300000000000000087
:100EB00018821D00188EAEEEFFFFA5F8FFFF780028
:100EC0000000D0FFFFFF00000000AE250000188EDC
:100ED000AEEEFFFFA5F8FFFF78000000E3FFFFFF85
:100EE00000000000F12B0000188EAEEEFFFF5B0744
:100EF0000000780000009CFEFFFF00000000862F2D
:100F00003000188E65F2FFFFA5F8FFFF78000000A3
:100F1000300000000000000012720B00188E65F215
:100F2000FFFFA6F8FFFF78000000E3FFFFFF0000CF
:100F30000000F12B0000188E65F2FFFFAD030000EA
:100F4000780000009CFEFFFF00000000A5232400A5
:100F5000188E1BF6FFFFA5F8FFFF78000000300099
:100F600000000000000031C80800188E1CF6FFFFCA
:100F7000A5F8FFFF78000000E3FFFFFF000000007E
:100F8000F12B0000188E1CF6FFFFAE030000780066
:100F900000009CFEFFFF00000000A5232400188E27
:100FA000D2F9FFFFA5F8FFFF780000003000000035
:100FB0000000000031C80800188ED2F9FFFFA5F824
:100FC000FFFF78000000E3FFFFFF00000000F12BAF
:100FD0000000188ED3F9FFFFAE0300007800000078
:100FE0009CFEFFFF00000000A5232400188E89FD51
:100FF000FFFFA5F8FFFF78000000300000000000B0
:10100000000031C80800188E89FDFFFFA5F8FFFF1A
:1010100078000000E3FFFFFF00000000F12B00005C
:10102000188E8AFDFFFFAD030000780000009CFED3
:10103000FFFF00000000A5232400188E40010000DF
:10104000A6F8FFFF7800000030000000000000005C
:1010500031C80800188E40010000A5F8FFFF780095
:101060000000E3FFFFFF00000000F12B0000188EDE
:1010700040010000AD030000780000009CFEFFFF6F
:1010800000000000A5232400188EF7040000A5F836
:10109000FFFF78000000300000000000000031C8B1
:1010A0000800188EF7040000A6F8FFFF7800000083
:1010B000E3FFFFFF00000000F12B0000188EF70493
:1010C0000000AD030000780000009CFEFFFF000060
:1010D0000000A5232400188EAD080000A5F8FFFF2E
:1010E00078000000300000000000000031C8080057
:1010F000188EAE080000A5F8FFFF78000000E3FF9F
:10110000FFFF00000000F12B0000188EAE08000069
:10111000AE030000780000009CFEFFFF000000000E
:10112000A5232400188E640C0000A5F8FFFF7800AA
:101130000000300000000000000031C80800188ED8
:10114000650C0000A5F8FFFF78000000E3FFFFFF3B
:1011500000000000F12B0000188E640C0000AE03AC
:101160000000780000009CFEFFFF00000000A523A7
:101170002400188E1C100000A5F8FFFF7800000066
:10118000300000000000000031C80800188E1B105D
:101190000000A5F8FFFF78000000E3FFFFFF00005C
:1011A0000000F12B0000188E1B100000AD030000A2
:1011B000780000009CFEFFFF00000000A523240033
:1011C000188ED2130000A6F8FFFF78000000300050
:1011D00000000000000031C80800188ED213000083
:1011E000A5F8FFFF78000000E3FFFFFF000000000C
:1011F000F12B0000188ED3130000AD03000078001F
:1012000000009CFEFFFF00000000A5232400188EB4
:1012100089170000A5F8FFFF7800000030000000EB
:101220000000000031C80800188E88170000A6F8DA
:10123000FFFF78000000E3FFFFFF00000000F12B3C
:101240000000188E89170000AD0300007800000030
:101250009CFEFFFF00000000A5232400188E401B09
:101260000000A5F8FFFF780000003000000000003B
:10127000000031C80800188E401B0000A5F8FFFFD1
:1012800078000000E3FFFFFF00000000F12B0000EA
:10129000188E401B0000AE030000780000009CFE8A
:1012A000FFFF00000000A5232400188E3F1B000054
:1012B000AD030000780000003000000000000000D6
:1012C000D9920000188908860189188C401B0000FB
:1012D000AD03000078000000000000006000000086
:1012E0008E54ECFFFFF0E9FFFFF00000000000006B
:1012F0000000000000A3602800188E53ECFFFFEFF1
:10130000E9FFFFF00000000000000043000000972C
:10131000CD00001889908E54ECFFFFF0E9FFFF78B4
:1013200000000000000000EDFFFFFF601800001843
:101330008E54ECFFFFF0E9FFFF7800000000000092
:1013400000E3FFFFFFF22B0000188E5BF7FFFFEFBB
:10135000E9FFFF78000000000000009CFEFFFFA5F1
:10136000232400188E54ECFFFF9DEDFFFF78000052
:10137000000000000030000000EFC50800188E5388
:10138000ECFFFF9DEDFFFF7800000000000000E390
:10139000FFFFFFF12B0000188E5CF7FFFF9DEDFFB4
:1013A000FF78000000000000009CFEFFFFA5232442
:1013B00000188E54ECFFFF4BF1FFFF780000000097
:1013C00000000030000000EFC50800188E53ECFF4D
:1013D000FF4AF1FFFF7800000000000000E3FFFF7C
:1013E000FFF12B0000188E5CF7FFFF4BF1FFFF7839
:1013F000000000000000009CFEFFFFA52324001851
:101400008E53ECFFFFF7F4FFFF78000000000000B0
:101410000030000000EFC50800188E54ECFFFFF804
:10142000F4FFFF7800000000000000E3FFFFFFF280
:101430002B0000188E5CF7FFFFF8F4FFFF78000028
:1014400000000000009CFEFFFFA5232400188E531F
:10145000ECFFFFA5F8FFFF7800000000000000305F
:10146000000000EFC50800188E54ECFFFFA5F8FF40
:10147000FF7800000000000000E3FFFFFFF22B00F8
:1014800000188E5BF7FFFFA6F8FFFF780000000052
:101490000000009CFEFFFFA5232400188E54ECFFE3
:1014A000FF52FCFFFF780000000000000030000049
:1014B00000EFC50800188E53ECFFFF53FCFFFF78C8
:1014C00000000000000000E3FFFFFFF22B00001807
:1014D0008E5CF7FFFF52FCFFFF7800000000000069
:1014E000009CFEFFFFA5232400188E54ECFFFF0094
:1014F000000000780000000000000030000000EF55
:10150000C50800188E53ECFFFF00000000780000B3
:101510000000000000E3FFFFFFF22B0000188E5CCC
:10152000F7FFFF0000000078000000000000009CB2
:10153000FEFFFFA5232400188E53ECFFFFAE03002F
:1015400000780000000000000030000000EFC50837
:1015500000188E54ECFFFFAD03000078000000007F
:10156000000000E3FFFFFFF22B0000188E5CF7FF86
:10157000FFAE03000078000000000000009CFEFFAA
:10158000FFA5232400188E53ECFFFF5A07000078B4
:101590000000000000000030000000EFC508001847
:1015A0008E54ECFFFF5B0700007800000000000095
:1015B00000E3FFFFFFF22B0000188E5BF7FFFF5BDD
:1015C00007000078000000000000009CFEFFFFA55F
:1015D000232400188E54ECFFFF080B000078000055
:1015E000000000000030000000EFC50800188E5316
:1015F000ECFFFF080B00007800000000000000E393
:10160000FFFFFFF12B0000188E5CF7FFFF090B00B6
:101610000078000000000000009CFEFFFFA52324CE
:1016200000188E54ECFFFFB50E000078000000009B
:1016300000000030000000EFC50800188E53ECFFDA
:10164000FFB60E00007800000000000000E4FFFF7D
:10165000FFF12B0000188E5CF7FFFFB50E0000783D
:10166000000000000000009BFEFFFFA523240018DF
:101670008E53ECFFFF6312000078000000000000B2
:101680000030000000EFC50800188E54ECFFFF6327
:101690001200007800000000000000E4FFFFFFF1EE
:1016A0002B0000188E5CF7FFFF631200007800002B
:1016B00000000000009BFEFFFFA5232400188E53AE
:1016C000ECFFFF1116000078000000000000003061
:1016D000000000EFC50800188E54ECFFFF10160044
:1016E000007800000000000000E4FFFFFFF12B0085
:1016F00000188E5BF7FFFF10160000780000000056
:101700000000009BFEFFFFA5232400188E0AFBFFAC
:10171000FF9EEDFFFFF00000000000000031000020
:1017200000BEA41E00188E09FBFFFF9DEDFFFF7891
:1017300000000000000000CFFFFFFFAE25000018F2
:101740008E09FBFFFF9DEDFFFF7800000000000009
:1017500000E3FFFFFFF12B0000188E09FBFFFFA540
:10176000F8FFFF78000000000000009CFEFFFFA5CE
:10177000232400188EB6FEFFFF9DEDFFFF780000CA
:10178000000000000030000000EFC50800188EB710
:10179000FEFFFF9DEDFFFF7800000000000000E469
:1017A000FFFFFFF12B0000188EB6FEFFFFA5F8FF2C
:1017B000FF78000000000000009BFEFFFFA523242F
:1017C00000188E640200009DEDFFFF78000000000D
:1017D00000000030000000EFC50800188E64020011
:1017E000009DEDFFFF7800000000000000E4FFFF17
:1017F000FFF12B0000188E64020000A5F8FFFF78AF
:10180000000000000000009BFEFFFFA5232400183D
:101810008E110600009DEDFFFF7800000000000023
:101820000030000000EFC50800188E120600009D71
:10183000EDFFFF7800000000000000E4FFFFFFF173
:101840002B0000188E11060000A5F8FFFF7800009D
:1018500000000000009BFEFFFFA5232400188EBFA0
:101860000900009DEDFFFF7800000000000000313E
:10187000000000EFC50800188EBE0900009DEDFFB6
:10188000FF7800000000000000E3FFFFFFF12B00E5
:1018900000188EBF090000A6F8FFFF7800000000C6
:1018A0000000009BFEFFFFA5232400188E6C0D0096
:1018B000009DEDFFFF7800000000000000310000F7
:1018C00000EFC50800188E6C0D00009DEDFFFF783D
:1018D00000000000000000E3FFFFFFF12B000018F4
:1018E0008E6C0D0000A5F8FFFF78000000000000DE
:1018F000009BFEFFFFA5232400188E1A1100009DF7
:10190000EDFFFF780000000000000031000000EF54
:10191000C50800188E191100009DEDFFFF7800002A
:101920000000000000E3FFFFFFF12B0000188E1AFB
:10193000110000A5F8FFFF78000000000000009BE8
:10194000FEFFFFA5232400188EC71400009DEDFFA5
:10195000FF780000000000000031000000EFC50823
:1019600000188EC71400009DEDFFFF7800000000F6
:10197000000000E3FFFFFFF12B0000188EC71400EA
:1019800000A5F8FFFF78000000000000009CFEFFAB
:10199000FFA5232400188E741800009DEDFFFF782A
:1019A0000000000000000030000000EFC508001833
:1019B0008E741800009DEDFFFF780000000000000D
:1019C00000E3FFFFFFF12B0000188E75180000A642
:1019D000F8FFFF78000000000000009CFEFFFFA55C
:1019E000232400188E211C00009DEDFFFF780000CD
:1019F000000000000030000000EFC50800188E2233
:101A00001C00009DEDFFFF7800000000000000E3D7
:101A1000FFFFFFF12B0000188E221C0000A5F8FF2D
:101A2000FF78000000000000009CFEFFFFA52324BB
:101A300000188ECF1F00009DEDFFFF780000000012
:101A400000000030000000EFC50800188ECF1F0016
:101A5000009DEDFFFF7800000000000000E3FFFFA5
:101A6000FFF12B0000188ECF1F0000A5F8FFFF78B4
:101A7000000000000000009CFEFFFFA523240018CA
:101A80008E7C2300009DEDFFFF7800000000000029
:101A90000030000000EFC50800188E7D2300009D77
:101AA000EDFFFF7800000000000000E3FFFFFFF102
:101AB0002B0000188E7C230000A5F8FFFF780000A3
:101AC00000000000009CFEFFFFA5232400188E2AC2
:101AD0002700009DEDFFFF780000000000000030AF
:101AE000000000EFC50800188E2A2700009DEDFFBA
:101AF000FF7800000000000000E3FFFFFFF12B0073
:101B000000188E2A270000A6F8FFFF7800000000CA
:101B10000000009CFEFFFFA52324001889108E2AD8
:101B2000270000A5F8FFFFB8F1000000000000004A
:101B300000000036F864001888010A0102880104D8
:101B400001FF891F860088000302000086018801CA
:101B500003020000860088001F02000088011F02A7
:101B60000000891F4B00A30703124E6F205344202F
:101B70006361726420666F756E64006578697420B5
:101B80006D656E750048656C702054657874202012
:101B90000048656174204C454473004C4544204323
:101BA0006F6C6F72202020202000536F756E6400D0
:101BB000546F6F6C20436F756E74200043616C69C5
:101BC0006272617465204E6F7A7A6C65730052653B
:101BD00073746F72652044656661756C7473004739
:101BE000656E6572616C2053657474696E6773000D
:101BF000507265686561742053657474696E6773AB
:101C00000053746F7020426C696E6B696E672100BF
:101C1000426C696E6B204C454473202020202020AC
:101C200020004C6576656C204275696C6420506CB0
:101C300061746500456E61626C65205374657070F7
:101C400065727320200044697361626C652053746F
:101C50006570706572730052756E20537461727492
:101C60007570205363726970740046696C616D65AC
:101C70006E74204F7074696F6E7300486F6D6520CD
:101C800041786573004A6F67204D6F6465004D6F42
:101C90006E69746F72204D6F6465005574696C696C
:101CA000746965730050726568656174005072698B
:101CB0006E742066726F6D20534400556E506175CE
:101CC000736500506175736500596573004E6F0050
:101CD0005175697420746869732070726F636573DD
:101CE000733F0043616E63656C2074686973207094
:101CF00072696E743F00596573004E6F00446566EB
:101D000061756C742076616C7565733F0052657304
:101D100065742053657474696E677320746F200056
:101D2000506C6174666F726D20202020202020206E
:101D3000004C65667420546F6F6C2020202020209A
:101D4000202020202000526967687420546F6F6C37
:101D5000202020202020202020200050726568654F
:101D600061742053657474696E67732020202000AD
:101D70002020202020202020202020202020202063
:101D8000202020200045787472756465723A202006
:101D9000202D2D2D2F2D2D2D4300506C6174666F3D
:101DA000726D3A2020202D2D2D2F2D2D2D43004CEE
:101DB0002045787472756465723A202D2D2D2F2D73
:101DC0002D2D4300522045787472756465723A2057
:101DD0002D2D2D2F2D2D2D4300202D2D250047415C
:101DE0004D45204F56455221002020202020202004
:101DF000205A2B20202020202020202020002020BE
:101E00003C2D5920284261636B292020202020206E
:101E100020200020202020202020205A2D2020209B
:101E200020202020202020002020202020202020D2
:101E3000592D202020202020202020200020203C60
:101E40002D5820284261636B2920205A2D3E2020E6
:101E500020002020202020202020592B202020205E
:101E6000202020202020002020202020202020585A
:101E70002D20202020202020202020002020202075
:101E80002020284261636B29202020592D3E2020EC
:101E9000002020202020202020582B20202020201F
:101EA00020202020200020202020204A6F67206D45
:101EB0006F64652020202020202000556E4C6F612B
:101EC00064004C6F61640059657321004E6F0066B9
:101ED000726F6D20746865206E6F7A7A6C653F0052
:101EE00044696420706C61737469632065787472EE
:101EF00075646520004C65742773207472792061C5
:101F00006761696E2E004D79206865696768742085
:101F1000697320676F6F6421006865696768742062
:101F2000636865636B206F75743F00446F65732051
:101F30006D79206E6F7A7A6C650059657321004E59
:101F40006F00746F207472792061207072696E74F2
:101F50003F2020202000486F772764206974206785
:101F60006F3F20526561647920005765276C6C20B3
:101F70006B65657020676F696E672E2020204C6549
:101F800074732074727920746865206C656674209F
:101F9000202065787472756465722E2050757368A0
:101FA00020202020202066696C616D656E7420649D
:101FB0006F776E2E2E2E20202020004772656174D0
:101FC00021202049276C6C2073746F7020202072B0
:101FD000756E6E696E67206D7920657874727564B0
:101FE00065722E5072657373204D20746F20636F7D
:101FF0006E74696E75652E20202020202020202000
:102000002020202020202020202020005765276C21
:102010006C206B65657020676F696E672E202020CD
:10202000496620796F7527726520686176696E67E9
:102030002020202074726F75626C652C20636865A7
:10204000636B206F757420206D616B6572626F74B5
:102050002E636F6D2F68656C70202020004F4B2120
:102060002049276C6C206B656570206D79202020DD
:10207000206D6F746F722072756E6E696E672E20A0
:10208000596F7520206D6179206E65656420746FCD
:102090002070757368202020206861726465722E3C
:1020A0002E2E2020202020202020202020005768B5
:1020B000656E206D792066696C616D656E7420694E
:1020C000732072656C65617365642C20202020206C
:1020D000202020202020507265737320274D272058
:1020E000746F20657869742E202020202020202005
:1020F00020202020202020202020202020200057C9
:1021000068656E2066696C616D656E742069732008
:10211000202020657874727564696E67206F75740D
:10212000206F66207468656E6F7A7A6C652C20501B
:102130007265737320274D27202020746F206578E7
:102140006974202020202020202020202020200012
:102150005768656E2066696C616D656E7420697381
:1021600020202020657874727564696E67206F7511
:1021700074206F66207468656E6F7A7A6C652C20A7
:10218000507265737320274D27202020746F2073B1
:10219000746F7020657874727564696E672E202084
:1021A000007468726F75676820746865206772656F
:1021B000792020202072696E6720756E74696C200A
:1021C000796F75206665656C20746865206D6F7425
:1021D0006F722074756767696E6720202074686568
:1021E00020706C617374696320696E2E2E2E20201E
:1021F0002000477265617421204E6F772077652734
:102200006C6C202020206C6F616420746865206CE9
:102210006566742020202020202065787472756403
:1022200065722E205075736820202020202066695A
:102230006C616D656E7420646F776E2E2E2E20207B
:102240002020004F4B2049276D2072656164792161
:1022500020202020202020506F7020746865206787
:1022600075696465207475626520206F66662061FB
:102270006E642070756C6C20202020202020206649
:10228000696C616D656E742067656E746C792E2E55
:102290002E2020004F4B2049276D20726561647904
:1022A0002120202020202020506F7020746865207D
:1022B0006775696465207475626520206F666620A5
:1022C000616E64207075736820746865202020201A
:1022D00066696C616D656E7420646F776E2E2E2E4C
:1022E00020202020004F4B2049276D20726561641B
:1022F00079212020202020202046697273742077C5
:1023000065276C6C206C6F61642074686572696706
:1023100068742065787472756465722E20202020A0
:1023200020507573682066696C616D656E742069F4
:102330006E2E2E2E200049276D2068656174696E0F
:1023400067207570206D792020206578747275641F
:102350006572212020202020202020202020506C69
:102360006561736520776169742E2020202020200C
:10237000202020202020202020202020202020205D
:102380002020202020200048656174696E6720505D
:10239000726F67726573733A2020202020202020FE
:1023A000202020202020202020202020202020202D
:1023B000202020202020202020202020202020201D
:1023C000202020202020202020202020202020200D
:1023D000202020202020200054686973206D696728
:1023E00068742074616B6520612020206665772009
:1023F0006D696E757465732E2020202020202020AA
:10240000416E64207761746368206F75742C20744A
:10241000686520206E6F7A7A6C652077696C6C2015
:1024200067657420484F542100706F7073206F757A
:102430007420696E2066726F6E742E202049276D9D
:102440002068656174696E67207570206D79202041
:1024500020657874727564657220736F20776520CB
:1024600063616E20206C6F6164207468652066690A
:102470006C616D656E742E2E2E0067756964652023
:1024800074756265206F75742E20204E6F776665B7
:1024900065642066696C616D656E742066726F6D2F
:1024A0002020746865206261636B207468726F75A8
:1024B0006768207468657475626520756E74696CF0
:1024C0002069742E2E2E20202000507265737320F8
:1024D000646F776E206F6E207468652020206772AD
:1024E00065792072696E6720617420746F70206F47
:1024F0006620746865206578747275646572206101
:102500006E642020202070756C6C207468652062D9
:102510006C61636B2E2E2E20202000677569646528
:10252000207475626573206F75742E204E6F776608
:102530006565642066696C616D656E742066726F96
:102540006D2020746865206261636B207468726F0F
:1025500075676820746865747562657320756E743C
:10256000696C2069742E2E2E202020005072657315
:102570007320646F776E206F6E2074686520202052
:10258000677265792072696E677320617420746F59
:1025900070206F6674686520657874727564657202
:1025A0007320616E6420202070756C6C20746865E7
:1025B00020626C61636B2E2E2E202020004D79202E
:1025C000657874727564657273206172652020206D
:1025D000206E6F742068656174696E672075702E57
:1025E0002020202020436865636B206D7920202007
:1025F000202020202020202020636F6E6E656374D1
:10260000696F6E7321202020202020202000592077
:1026100041786973204C696E650058204178697370
:10262000204C696E6500446F6E65210053656C65D2
:1026300063742062657374206C696E65732E004745
:102640007265617421202049277665207361766563
:1026500064202074686573652073657474696E679F
:102660007320616E64202049276C6C20757365208F
:102670007468656D20746F202020206D616B65206B
:102680006E696365207072696E747321202020006A
:102690006C696E65206F6E65206973206578747251
:1026A000612020206C6F6E672E20546865205920B1
:1026B00061786973207365746973206C6566742032
:1026C0006F6E2074686520706C617465616E642043
:1026D0005820617869732069732072696768742E65
:1026E000004C6F6F6B20666F7220746865206265A6
:1026F00073742020206D617463686564206C696E5A
:102700006520696E2065616368617869732073650F
:10271000742E204C696E657320617265206E756D34
:10272000626572656420312D313320616E642E2E16
:102730002E0049276D20676F696E6720746F2070C7
:1027400072696E7420206120736572696573206FF1
:1027500066206C696E657320736F77652063616EA8
:102760002066696E64206D792020202020206E6F05
:102770007A7A6C6520616C69676E6D656E742E2067
:102780002020005765276C6C20676F20746F2074C1
:102790006865206D61696E6D656E752E20496620D5
:1027A000796F75206E65656420202068656C7020E7
:1027B000676F20746F3A2020202020202020206D79
:1027C000616B6572626F742E636F6D2F68656C70DC
:1027D00020202000417765736F6D65212020202027
:1027E00020202020202020205765276C6C20676F38
:1027F00020746F20746865205344202063617264E4
:10280000204D656E7520616E6420796F75202020E3
:1028100063616E2073656C656374206120707269FA
:102820006E742120005765276C6C206B65657020E5
:10283000676F696E6720202020616E64206C6F6175
:102840006420736F6D6520202020202020706C6133
:10285000737469632120466F722068656C7020670D
:102860006F746F206D616B6572626F742E636F6D34
:102870002F68656C70005765276C6C207472792026
:10288000616761696E2120202020202020202020E7
:102890002020202020202020202020202020202038
:1028A0002020202020202020202020202020202028
:1028B0002020202020202020202020202020202018
:1028C00020202020202000416161682C2074686154
:1028D00074206665656C73202020206D7563682008
:1028E0006265747465722E20202020202020204CE8
:1028F0006574277320676F206F6E20616E64206C93
:102900006F6164736F6D6520706C617374696321AE
:102910002020202020202000706C6174666F726D72
:1029200020736F2069742773202020206E696365EF
:1029300020616E64206C6576656C2E204974277367
:1029400070726F6261626C79206120626974206FBD
:102950006666202066726F6D207368697070696E9C
:10296000672E2E2E20202020004F7572206E657855
:10297000742073746570732077696C6C206765745C
:10298000206D652073657420757020746F20202081
:10299000207072696E74212046697273742C2077DE
:1029A00065276C6C20726573746F7265206D792079
:1029B0006275696C642E2E2E20004120736F6C6945
:1029C0006420274D27206D65616E732020204927E4
:1029D0006D20776F726B696E6720616E6420776916
:1029E0006C6C757064617465206D792073746174AA
:1029F0007573202020207768656E2049276D20663A
:102A0000696E69736865642E2E2E004120626C69C0
:102A10006E6B696E6720274D27206D65616E734967
:102A2000276D2077616974696E6720616E64207715
:102A3000696C6C636F6E74696E7565207768656E1E
:102A400020796F752020207072657373207468651B
:102A500020627574746F6E2E2E2E200057656C6385
:102A60006F6D652120202020202020202020202084
:102A700049276D20746865205265706C69636174C4
:102A80006F722E20507265737320746865207265B2
:102A900064204D20746F2020676574207374617208
:102AA0007465642120202020202020200045787497
:102AB000727564657200506C6174666F726D004C63
:102AC00065667420546F6F6C005269676874205497
:102AD0006F6F6C0053746F7020507265686561741D
:102AE00021005374617274205072656865617421AD
:102AF000004669726D776172652056657273696F01
:102B00006E20352E2000202020202D2D2D2D2D2D26
:102B10002D2D2D2D202020202020002020546865E0
:102B2000205265706C696361746F722020202000F0
:102B30002020202020202020202020202020202095
:102B40002020202000010049033600FF006B00D147
:102B500000A000B800D500A6000A0199003F018E30
:102B60000074018400A9017C00DE01740013026C72
:102B700000480265007D025D00B2025600E7024E89
:102B8000001C03460051033D0086033200BB0322B4
:102B900000F0030300001E25DB268E32EA3BEB3DEE
:102BA0005E45AB49F75BBB64588E11241FBECFEF67
:102BB000D1E2DEBFCDBF18E0A0E0B2E0EAE2F0E291
:102BC00001E00BBF02C007900D92AA39B107D9F7F7
:102BD00014E1AAE9B8E001C01D92A33AB107E1F7F8
:102BE0001BE2CAEADBE200E006C022970109FE010F
:102BF0000BBF0E941A8FC639D10780E00807A9F7DA
:102C00000E94CC320C9413900C940000EF92FF922F
:102C10000F931F937B018C0120E030E040E05FE4E4
:102C20000E94041987FD11C0C801B70120E030E0FF
:102C300040E05FE40E94A9170E9494199B01AC0137
:102C4000205030404040504806C0C801B7010E94A3
:102C500094199B01AC01B901CA011F910F91FF901A
:102C6000EF900895A0E0B0E0E8E3F6E10C94E78E81
:102C7000FC01EA018081823008F438C1DB019C91BB
:102C8000923008F430C1843059F4943009F02EC1E8
:102C9000918111968C911197981709F021C126C145
:102CA000943009F420C19230B1F4823009F01EC191
:102CB000CA01AF0128E0DA010D90AD01DC010D92EF
:102CC000CD012150C1F7DB0111968C9111979181B3
:102CD000892389830AC1823009F405C1C280D38067
:102CE000DB0112966D907C9013972481358146818B
:102CF00057811496ED90FD900D911C911797C60188
:102D0000861997095C0197FF04C0AA24BB24A81A5E
:102D1000B90AB0E2AB16B1040CF061C0181619067E
:102D20006CF5370148010A2C04C096948794779477
:102D300067940A94D2F781E090E0A0E0B0E00A2C1A
:102D400004C0880F991FAA1FBB1F0A94D2F70197CE
:102D5000A109B1098E219F21A023B123EE24FF24D4
:102D60008701E3940097A105B10519F4EE24FF242F
:102D70008701E628F728082919293CC00097D1F1D6
:102D8000CA0CDB1C39014A010A2C04C096948794B2
:102D9000779467940A94D2F781E090E0A0E0B0E0E5
:102DA0000A2C04C0880F991FAA1FBB1F0A94D2F7D0
:102DB0000197A109B10982239323A423B52321E01C
:102DC00030E040E050E00097A105B10519F420E0A3
:102DD00030E0A90126293729482959290BC06C144C
:102DE0007D0424F4EE24FF24870104C0630120E065
:102DF00030E0A9018181FB019181891709F445C067
:102E0000882349F0D801C701821B930BA40BB50B93
:102E10009C01AD0104C02E193F09400B510B57FD19
:102E200004C01982DB82CA820BC081E08983DB8205
:102E3000CA8250954095309521953F4F4F4F5F4F37
:102E40002C833D834E835F830DC0880F991FAA1F7B
:102E5000BB1F8C839D83AE83BF838A819B81019737
:102E60009B838A838C819D81AE81BF819C01AD0152
:102E700021503040404050402F3FEFEF3E07EFEFF2
:102E80004E07EFE35E0708F30BC08983DB82CA823B
:102E90002E0D3F1D401F511F2C833D834E835F83AA
:102EA00083E088832C813D814E815F8157FF1DC067
:102EB000DA01C90181709070A070B0705695479585
:102EC00037952795822B932BA42BB52B8C839D8331
:102ED000AE83BF838A819B8101969B838A8305C0D1
:102EE000ECEDF4E003C0FB0101C0FE01CF01CDB762
:102EF000DEB7EEE00C94038FA0E2B0E0E2E8F7E189
:102F00000C94EF8E69837A838B839C832D833E831D
:102F10004F83588789E0E82EF12CEC0EFD1ECE0180
:102F20000196B7010E94861B8E010F5E1F4FCE01D6
:102F30000596B8010E94861BC701B801AE01475E25
:102F40005F4F0E9432160E94B81AA096E6E00C94D9
:102F50000B8FA0E2B0E0EFEAF7E10C94EF8E69830B
:102F60007A838B839C832D833E834F8358878E0186
:102F7000075F1F4FCE010196B8010E94861B91E1A9
:102F8000E92EF12CEC0EFD1ECE010596B7010E9434
:102F9000861B8A8991E089278A8BC801B701AE0117
:102FA000475E5F4F0E9432160E94B81AA096E6E074
:102FB0000C940B8FA0E2B0E0E0EEF7E10C94E38E0E
:102FC00069837A838B839C832D833E834F835887C9
:102FD000CE010196BE01675F7F4F0E94861BCE0126
:102FE0000596BE016F5E7F4F0E94861B99859230C9
:102FF00078F089898230C0F0943019F4823041F43D
:10300000CBC0843019F4923079F4C6C0923051F4B8
:1030100081E02A859A89291709F480E08A87CE0100
:103020000996BCC0823051F481E02A859A8929171B
:1030300009F480E08A8BCE014196B0C06D847E8415
:103040008F849888ED88FE880F89188DE0E2F0E083
:1030500080E090E0DC01AA24BB24650120E030E0A0
:10306000A901B3016170707061157105D1F02E0D69
:103070003F1D401F511F15012601280E391E4A1EF3
:103080005B1E81E090E0A0E0B0E02E153F05400718
:10309000510718F080E090E0DC01820D931DA41D23
:1030A000B51DAA0CBB1CCC1CDD1C17FF09C061E0C0
:1030B000262E312C412C512CA228B328C428D528E7
:1030C000319749F0EE0CFF1C001F111F9694879456
:1030D00077946794C6CF6B897C89EB85FC856E0FEE
:1030E0007F1F6E5F7F4F7C8F6B8F61E0EA857A89EF
:1030F000E71709F460E06A8F6B8D7C8D10C0FC01CE
:10310000E170F070309729F05695479537952795DF
:103110005068B695A795979587956F5F7F4FB7FDD8
:10312000EECF0CC0880F991FAA1FBB1F57FD8160EF
:10313000220F331F441F551F615070408030E0E064
:103140009E07E0E0AE07E0E4BE0760F36B8F7C8F84
:103150006FE7E62EF12C012D112DE822F9220A232A
:103160001B2360E4E616F1040105110561F487FDF7
:103170000AC0211531054105510529F0805C9F4F9A
:10318000AF4FBF4F80788D8F9E8FAF8FB8A383E0F6
:10319000898FCE01499602C08CED94E00E94B81A46
:1031A000A096E2E10C94FF8EA8E1B0E0EAEDF8E130
:1031B0000C94EF8E69837A838B839C832D833E836B
:1031C0004F8358878E01075F1F4FCE010196B801CC
:1031D0000E94861B81E1E82EF12CEC0EFD1ECE0133
:1031E0000596B7010E94861B8985823040F0898947
:1031F000823028F0C801B7010E94EF1B01C081E0B6
:103200006896E6E00C940B8FA8E1B0E0EAE0F9E103
:103210000C94EF8E69837A838B839C832D833E830A
:103220004F8358878E01075F1F4FCE010196B8016B
:103230000E94861B81E1E82EF12CEC0EFD1ECE01D2
:103240000596B7010E94861B8985823040F08989E6
:10325000823028F0C801B7010E94EF1B01C08FEF38
:103260006896E6E00C940B8FA8E0B0E0EAE3F9E1A1
:103270000C94EF8E7B018C0183E08983D801C70118
:103280008827B7FD83959927AA27BB27282F8A83EC
:10329000E114F1040105110519F482E0898337C0B6
:1032A0008EE190E09C838B83222389F080E0E816F6
:1032B00080E0F80680E0080780E8180769F11095BB
:1032C0000095F094E094E11CF11C011D111DED82AC
:1032D000FE820F831887C801B7010E945E1A9C0105
:1032E000215030401216130694F4022E04C0EE0C46
:1032F000FF1C001F111F0A94D2F7ED82FE820F837C
:1033000018878EE190E0821B930B9C838B83CE0108
:1033100001960E94B81A04C060E070E080E09FEC63
:103320002896E6E00C940B8FACE0B0E0EAE9F9E116
:103330000C94F38E69837A838B839C83CE010196F0
:10334000BE016B5F7F4F0E94861B8D81823081F1B1
:10335000823070F1843021F48E81882369F10AC0B3
:103360002F81388537FD24C06E812F3131053CF027
:10337000662311F120E030E040E050E821C08EE10A
:1033800090E0821B930B29853A854B855C8504C0B0
:1033900056954795379527958A95D2F7662381F0FC
:1033A00050954095309521953F4F4F4F5F4F08C046
:1033B00020E030E0A90104C02FEF3FEF4FEF5FE7BF
:1033C000B901CA012C96E2E00C940F8FA8E0B0E09E
:1033D000ECEEF9E10C94ED8E7B018C011A82611503
:1033E00071058105910519F482E089835FC083E04E
:1033F00089838EE1C82ED12CDC82CB82ED82FE82C5
:103400000F831887C801B7010E945E1AFC0131972B
:10341000F7FF3AC0AA27BB27AE1BBF0B21E030E065
:1034200040E050E00A2E04C0220F331F441F551FF6
:103430000A94D2F721503040404050402E213F2185
:103440004023512361E070E080E090E021153105D8
:103450004105510519F460E070E0CB0104C01695F8
:103460000795F794E794AA95D2F7E62AF72A082B4E
:10347000192BED82FE820F8318878EE190E08E1B60
:103480009F0B9C838B8312C0309781F00E2E04C05B
:10349000EE0CFF1C001F111F0A94D2F7ED82FE8272
:1034A0000F831887CE1ADF0ADC82CB82CE01019609
:1034B0000E94B81A2896E8E00C94098FAF92BF9248
:1034C000CF92DF92EF92FF920F931F937B018C01BB
:1034D00080E0E81680E0F80681E0080780E0180741
:1034E00058F4EFEFEE16F1040105110509F090F420
:1034F00080E090E0DC0117C0F0E0EF16F0E0FF069E
:10350000F0E00F07F1E01F0750F480E190E0A0E049
:10351000B0E009C088E090E0A0E0B0E004C088E13D
:1035200090E0A0E0B0E020E230E040E050E0281B76
:10353000390B4A0B5B0B5701680104C0D694C79442
:10354000B794A7948A95D2F7D601C5018C519B4FA9
:10355000FC018081281B310941095109C9011F91D2
:103560000F91FF90EF90DF90CF90BF90AF900895B4
:10357000EF92FF920F931F93CF93DF93FC0124816F
:1035800035814681578161818081823020F440619C
:10359000EFEFF0E0A3C0843009F49BC0823009F45F
:1035A00092C0211531054105510509F48FC00280F3
:1035B000F381E02D8FEFE238F8070CF05AC0C2E833
:1035C000DFEFCE1BDF0BCA31D1056CF579018A0123
:1035D0000C2E04C016950795F794E7940A94D2F739
:1035E00081E090E0A0E0B0E00C2E04C0880F991FAD
:1035F000AA1FBB1F0A94D2F70197A109B109822320
:103600009323A423B52321E030E040E050E000976D
:10361000A105B10519F420E030E0A9012E293F29C8
:10362000402B512B03C020E030E0A901DA01C90191
:103630008F779070A070B07080349105A105B105AE
:1036400039F427FF09C0205C3F4F4F4F5F4F04C044
:10365000215C3F4F4F4F5F4FE1E0F0E0203080E0D2
:10366000380780E0480780E4580728F5E0E0F0E0FC
:1036700022C0E038F1056CF5E158FF4FDA01C901CD
:103680008F779070A070B07080349105A105B1055E
:1036900039F427FF09C0205C3F4F4F4F5F4F04C0F4
:1036A000215C3F4F4F4F5F4F57FF05C056954795E1
:1036B00037952795319687E0569547953795279505
:1036C0008A95D1F70BC0E0E0F0E005C0E0E0F0E063
:1036D00005C0EFEFF0E020E030E0A9018E2F8795E4
:1036E00088278795942F9F77679566276795E69536
:1036F000E22EA92FA82BFE2FF62B622F732F8A2FD5
:103700009F2FCDB7DEB7E6E00C940B8FDC01FB01F9
:103710002C9111963C91119712968C911297482FEB
:103720004F7750E0982F991F9927991F13966C9106
:103730001397862F880F892B90E0661F6627661FD8
:103740006183009739F5211531054105510511F4C3
:1037500082E029C082E89FEF9383828367E0220F93
:10376000331F441F551F6A95D1F783E0808309C03A
:10377000220F331F441F551F82819381019793832A
:103780008283203080E0380780E0480780E45807D3
:1037900078F320C08F3F910579F42115310541055B
:1037A000510519F484E08083089544FF03C081E04B
:1037B000808310C010820EC08F5790409383828305
:1037C00083E0808387E0220F331F441F551F8A95B3
:1037D000D1F7506424833583468357830895FC01D1
:1037E000DB019081923008F449C08C91823008F45A
:1037F00045C0943051F461818430B1F511962C911B
:10380000119730E0261B310941C0843021F09230FD
:1038100041F48230B1F111968C9111978823A1F176
:103820002DC06181823001F111968C91119768173A
:10383000D9F42281338112968D919C91139782172E
:10384000930794F028173907BCF02481358146810D
:10385000578114968D919D910D90BC91A02D82174A
:103860009307A407B50718F4662341F00DC0281785
:1038700039074A075B0728F4662331F021E030E07E
:1038800005C020E030E002C02FEF3FEFC9010895EE
:1038900010929C08E4E0F1E080818F718083E5E084
:1038A000F1E080818F71808308956F927F928F9273
:1038B0009F92AF92BF92CF92DF92EF92FF920F93BF
:1038C0001F93DF93CF93CDB7DEB7A8970FB6F894C9
:1038D000DEBF0FBECDBF8C01FC018181882309F0C2
:1038E000CDC08281882309F4BAC0C80102960E9423
:1038F000FB8C882309F4C2C0B2C080919A08882347
:10390000E9F4C8010C9640E856E968E970E00E94C5
:10391000DE8C81E080939A0811C07E010894E11C3E
:10392000F11CC7010E94DA8CD8011C96F7018AE0CD
:1039300001900D928150E1F710929A083CE0E32E3D
:10394000F12CE00EF11EC7010E94FB8C882399F038
:1039500085E0F801808381E081838E01055F1F4F40
:10396000C8010E94DA8CD701F8018AE001900D921B
:103970008150E1F783C0A1FC10C080919B0888238F
:10398000F1F4C801469640E856E968E970E00E9403
:10399000DE8C81E080939B0812C025E1E22EF12CA1
:1039A000EC0EFD1EC7010E94DA8CD8015696F70175
:1039B0008AE001900D928150E1F710929B0896E108
:1039C000E92EF12CE00EF11EC7010E94FB8C88232A
:1039D00099F086E0F801808381E081838E01015EA9
:1039E0001F4FC8010E94DA8CD701F8018AE00190CC
:1039F0000D928150E1F742C060909C08D61461F1AD
:103A00006D24EE24FF247724CC24C39493010E2C40
:103A100002C0359527950A94E2F720FF16C095015C
:103A20000E2C02C0359527950A94E2F720FD0DC0B3
:103A3000F8018181882349F4E082C182C40140E415
:103A400052E460E070E00E94DE8C0894E11CF11CFE
:103A5000F5E0EF16F104D1F6D0929C080FC082E099
:103A6000882E912C800E911EC4010E94218DD09031
:103A70000301AD2CBB24D0FE40CF4FCFA8960FB68C
:103A8000F894DEBF0FBECDBFCF91DF911F910F9194
:103A9000FF90EF90DF90CF90BF90AF909F908F906E
:103AA0007F906F900895FC01DB01F89481819081F3
:103AB00011827894882321F09C9311961C9211977F
:103AC00008958FE180939C08089580919F0A9091BA
:103AD000A00A009729F481E08093A60A80E0089567
:103AE0008091A10A9091A20A20919D0A30919E0A8C
:103AF000B9010E947F8EE091A30AF091A40AE80F19
:103B0000F91F8091A10A9091A20A0196B9010E9421
:103B10007F8E9093A20A8093A10A80919F0A909130
:103B2000A00A01979093A00A80939F0A808108952C
:103B3000462FFC0162816F700E94E25B0895F89449
:103B400080919F0A9091A00A20919D0A30919E0A2F
:103B5000281B390B7894C90108958093A80A089509
:103B600081E08093A90A08958091A80A0895209180
:103B70009F0A3091A00A81E02115310509F080E00B
:103B800008950E94651D08951F930E94651D182FBA
:103B90000E94651D982F812F1F9108951F93DF9319
:103BA000CF9300D0CDB7DEB70E94651D8A830E94F7
:103BB000651D89830E94651D182F0E94651D982F21
:103BC0006A817981812F0F900F90CF91DF911F91A2
:103BD00008951092A00A10929F0A1092A20A1092C1
:103BE000A10A1092A50A1092A60A1092AB0A10928E
:103BF000AA0A089581E02091AA0A3091AB0A2630E2
:103C0000310509F080E00895EF92FF920F931F9322
:103C1000DF93CF93CDB7DEB728970FB6F894DEBF0A
:103C20000FBECDBF0E94651D88870E94651D8F83D2
:103C30000E94651D9F812885993009F4A4C09A309F
:103C400090F4953009F49FC0963030F49330F1F041
:103C5000943009F09FC097C0973009F497C098300E
:103C600008F091C093C09C3061F19D3038F49A30D7
:103C700009F453C09B3009F08DC06CC09731D1F06E
:103C80009F31F1F19D3009F085C02FC0213019F02E
:103C9000222331F009C09DE6E92E9CE0F92E04C0F4
:103CA0008DEEE82E8BE0F82E0E94C41DBC01C701EA
:103CB000409630C08091A80A91E089278093A80A95
:103CC00067C0213019F0222321F005C00DE61CE069
:103CD00002C00DEE1BE00E94C11D682F70E06170F4
:103CE0007070C8010E94D02953C00E94C11D682F66
:103CF00070E06170707083E49BE00E94B43B48C048
:103D000083E49BE061E00E94AF3B0E94C41DBC01C4
:103D100089E79FE00E94F45E3BC080912A14909155
:103D20002B149A8389838B81807F81608B83CE0162
:103D3000019661E00E94981D0E94651D21E030E01F
:103D40003093AB0A2093AA0A682F70E061707070FC
:103D500084E016C080912A1490912B149D838C834B
:103D60008E81807F81608E83CE01049661E00E9407
:103D7000981D0E94651D682F70E06170707083E06F
:103D80000E94124905C00E94651D02C00E94CE1DFE
:103D900081E001C080E028960FB6F894DEBF0FBE28
:103DA000CDBFCF91DF911F910F91FF90EF900895BC
:103DB000FC01462F828193812081318182179307F4
:103DC000A0F46281738184819581860F971FB90168
:103DD0000E947F8EA681B781A80FB91F4C93828164
:103DE0009381019693838283089581E0808708956B
:103DF000682F8DE99AE00E94D81E08952F923F9275
:103E00004F925F926F927F928F929F92AF92BF92EA
:103E1000CF92DF92EF92FF920F931F93DF93CF9396
:103E2000CDB7DEB7CF5AD0400FB6F894DEBF0FBE85
:103E3000CDBF0E943F42882309F180919F0A909153
:103E4000A00A20919D0A30919E0A2817390709F48B
:103E5000CFC50E948C42882309F4CAC50E948F42B4
:103E6000682F8DE99AE00E94D81EE7CF80919F0AC3
:103E70009091A00A009711F40E949E420E940A4A63
:103E8000882309F180919F0A9091A00A20919D0AB0
:103E900030919E0A2817390709F4B0C50E94104ACC
:103EA000882309F4ABC50E941E4A682F8DE99AE069
:103EB0000E94D81EE7CF80919F0A9091A00A009798
:103EC00011F40E948C4A8091A80A882309F09CC5AD
:103ED0008091A90A882309F097C58091AA0A909138
:103EE000AB0A8330910581F40E946345882341F039
:103EF00086EB9AE00E94FB8C882331F00E94DF451C
:103F00001092AB0A1092AA0A8091AA0A9091AB0A69
:103F10008130910541F40E946345882321F4109279
:103F2000AB0A1092AA0A8091AA0A9091AB0A823039
:103F3000910551F48CEA9AE00E94FB8C882321F0D1
:103F40001092AB0A1092AA0A8091AA0A9091AB0A29
:103F500084309105E1F480EC9AE00E94FB8C882388
:103F600091F48091A70A813019F0882321F005C0CF
:103F70000DE61CE002C00DEE1BE0C80140960E9459
:103F80008E5F882321F01092AB0A1092AA0A8091CA
:103F9000AA0A9091AB0A8530910581F480EC9AE0F1
:103FA0000E94FB8C882331F489E79FE00E948E5F9A
:103FB000882321F01092AB0A1092AA0A8091AA0AD3
:103FC0009091AB0A8630910561F58AEC9AE00E94E7
:103FD000FB8C882351F08091D50A81FF1EC083E4B9
:103FE0009BE060E00E94ED381CC080E29DE00E94F2
:103FF000B3648823B1F08091D50A82FF04C080E2C7
:104000009DE00E94DF6283E49BE060E070E040E0BE
:1040100050E00E946F370E943F401092AB0A10920E
:10402000AA0A8091AA0A9091AB0A009709F0ECC401
:1040300080919F0A9091A00A009709F4E5C483E457
:104040009BE00E9406378091A10A9091A20A2091DC
:104050009D0A30919E0AE091A30AF091A40AB90149
:104060000E947F8E8E0F9F1FDC010C910138F1F5AD
:1040700080919F0A9091A00A8131910508F4C4C4EF
:104080000E94651D81E090E09093AB0A8093AA0A9C
:104090000E94CE1D6B017C010E94CE1D1B012C01D4
:1040A0000E94CE1D3B014C010E94CE1DCB55DF4F1F
:1040B000688379838A839B83C55AD04019E1A12EF6
:1040C000B12CAC0EBD1EC501B701A6019201810144
:1040D000740163010E94613EC501CB55DF4F4881E9
:1040E00059816A817B81C55AD04074C00B3809F070
:1040F00074C080919F0A9091A00A8931910508F4BB
:1041000083C40E94651D81E090E09093AB0A809388
:10411000AA0A0E94CE1D4B015C010E94CE1D8B019C
:104120009C01C255DF4F2883CE5AD040C155DF4F86
:104130003883CF5AD0400E94CE1D1B012C010E9413
:10414000CE1DCB55DF4F688379838A839B83C55A05
:10415000D0400E94CE1D6B017C010E94CE1DC75530
:10416000DF4F688379838A839B83C95AD04000D00C
:1041700000D0BDE26B2E712C6C0E7D1EEDB7FEB72C
:10418000C182D282E382F482C301B501A401C25587
:10419000DF4F2881CE5AD040C155DF4F3881CF5AEA
:1041A000D04072016101CB55DF4F88809980AA8091
:1041B000BB80C55AD0400E942D3E0F900F900F90AB
:1041C0000F90C301C755DF4F488159816A817B81B8
:1041D000C95AD0400E94DC4617C40E3809F082C08C
:1041E00080919F0A9091A00A8A31910508F40CC42D
:1041F0000E94651D81E090E09093AB0A8093AA0A2B
:104200000E94CE1D4B015C010E94CE1D8B019C01C2
:10421000C255DF4F2883CE5AD040C155DF4F388377
:10422000CF5AD0400E94CE1D1B012C010E94CE1DF2
:10423000CB55DF4F688379838A839B83C55AD040EF
:104240000E94CE1D6B017C010E94CE1DC755DF4F21
:10425000688379838A839B83C95AD0400E94C11D99
:10426000C355DF4F8883CD5AD04000D000D0A1E4A1
:104270006A2E712C6C0E7D1EADB7BEB71196CD9215
:10428000DD92ED92FC921497C301B501A401C255D1
:10429000DF4F2881CE5AD040C155DF4F3881CF5AE9
:1042A000D04072016101CB55DF4F88809980AA8090
:1042B000BB80C55AD0400E942D3E0F900F900F90AA
:1042C0000F90C301C755DF4F488159816A817B81B7
:1042D000C95AD040C355DF4F2881CD5AD0400E94E3
:1042E000A44792C3063889F480919F0A9091A00A4E
:1042F0008230910508F488C30E94651D0E94651DE7
:104300008093A70A0E9466467FC3093839F58091D9
:104310009F0A9091A00A8230910508F475C30E940B
:10432000651D0E94651DA82EAA1CAA24AA1C00E0D7
:1043300010E0C82EDD24C601002E02C09595879599
:104340000A94E2F780FF04C0802F6A2D0E94124970
:104350000F5F1F4F0530110571F756C3023821F565
:1043600080919F0A9091A00A8D30910508F44CC36A
:104370000E94651D0E94CE1D3B014C010E94CE1D76
:104380001B012C010E94CE1D6B017C01F5E5AF2EB7
:10439000B12CAC0EBD1EC501B401A3019201810177
:1043A0000E94613EC50148C00C3809F048C08091A8
:1043B0009F0A9091A00A8531910508F425C30E94B7
:1043C000651D0E94CE1D6B017C010E94CE1D1B014C
:1043D0002C010E94CE1D4B015C010E94CE1DCB55CD
:1043E000DF4F688379838A839B83C55AD0400E94BC
:1043F000CE1D00D000D0E9E66E2E712C6C0E7D1E15
:10440000EDB7FEB76183728383839483C301B701E1
:10441000A6019201810175016401CB55DF4F8880AF
:104420009980AA80BB80C55AD0400E942D3E0F9033
:104430000F900F900F90C3010E94E645E5C205382A
:10444000E9F480919F0A9091A00A8530910508F4C3
:10445000DBC282E090E09093AB0A8093AA0A0E94AC
:10446000651D0E94CE1D28EE33E040E050E00E9422
:10447000608EAB01BC018CEA9AE01CC10439B9F52D
:1044800080919F0A9091A00A8530910508F4BCC2E2
:104490000E94651D0E94651D8093D40A0E94C41D60
:1044A0008C010E94651D8093D50A0115110581F0CC
:1044B000B80180E090E020E432E44FE050E00E9458
:1044C000608EAB01BC018AEC9AE00E94DE8C80C059
:1044D0008E010B5F1F4FC8010E94DA8CAAECBAE074
:1044E000F8018AE001900D928150E1F771C0053921
:1044F00009F083C080919F0A9091A00A86309105AF
:1045000008F482C20E94651D0E94651DC82E0E948B
:10451000651D882E0E94651DA82E0E94651D082F0E
:10452000C0FC04C088EF9EE00E945B818092FA0E7E
:10453000A092FB0E41E0C1FE40E088EF9EE06DE9F5
:104540007AE00E941A85E0916E0DFF27E7FDF09555
:10455000EE0FFF1FE05AF24F20813181FEE0283F2D
:104560003F0731F080E29DE068EF7EE00E943A6212
:10457000002341F0C2FC06C088EF9EE0602F41E0BE
:104580000E949F81C2FE40C2002389F0602F70E02C
:1045900080E090E020E432E44FE050E00E94608E42
:1045A000AB01BC018AEC9AE00E94DE8C0EC08E0149
:1045B000015F1F4FC8010E94DA8CAAECBAE0F80133
:1045C0008AE001900D928150E1F781E08093D40A56
:1045D00083E49BE069E170E04FE050E00E946F37B8
:1045E00080E29DE06091D40A0E94AE6486E090E093
:1045F0009093AB0A8093AA0A07C2802F8358823017
:1046000090F580919F0A9091A00A8830910508F456
:10461000FBC10E94651D0E94C11DA82E0E94CE1DD7
:104620006B017C010E94C41D23E030E03093AB0A93
:104630002093AA0ABC0180E090E020E432E44FE03D
:1046400050E00E94608EAB01BC0186EB9AE00E94B4
:10465000DE8C81E0043809F080E06A2DA701960124
:104660000E94A148D1C1073841F580919F0A9091DD
:10467000A00A8630910508F4C7C184E090E09093C9
:10468000AB0A8093AA0A0E94651D0E94651D809353
:10469000A70A0E94C41D0E94C41DBC0180E090E0D6
:1046A00020E432E44FE050E00E94608EAB01BC0198
:1046B00080EC9AE00E94DE8CA7C10D3899F48091BD
:1046C0009F0A9091A00A8630910508F49DC185E06B
:1046D00090E09093AB0A8093AA0A0E94651D0E9405
:1046E000651DD7CF0F3809F047C080919F0A909180
:1046F000A00A8230910508F487C10E94651D0E94BE
:10470000C11D5EE0A52EB12C00E010E0882E99249A
:104710004DE7642E712C6C0E7D1E6E010894C11C39
:10472000D11CC401002E02C0959587950A94E2F72A
:1047300080FF18C0C3010E941146C301B8010E9446
:10474000833EFC0180819181A281B38189839A8318
:10475000AB83BC83F894C601B50144E050E00E94ED
:10476000EE8F78940F5F1F4F84E090E0A80EB91E83
:1047700005301105B1F648C1003909F03FC08091FC
:104780009F0A9091A00A8230910508F43DC10E94D1
:10479000651D0E94C11DC82E31E9A32EB12CAC0E9F
:1047A000BD1EC5010E9411462EE0622E712C00E054
:1047B00010E0DD248A2CAB2CC601002E02C095959A
:1047C00087950A94E2F780FF0CC0F894882D9A2D03
:1047D000B8010E948B3EB30144E050E00E94D88FA4
:1047E00078940F5F1F4FA4E0B0E06A0E7B1E053087
:1047F000110511F7CE018F569F4F1ECE0139C9F416
:1048000080919F0A9091A00A8230910508F4FCC023
:104810000E94651D0E94C11DC82E0E94C11D082F47
:104820008C2D602F0E9424498C2D602F0E942449DA
:10483000EBC0023989F580919F0A9091A00A8230DD
:10484000910508F4E1C00E94651D0E94C11D082F5A
:104850000E94C11DC155DF4F8883CF5AD0400E94AE
:10486000C11DC255DF4F8883CE5AD0400E94C11D62
:10487000C82E0E94C11D8C2D0E94CB40802FC15597
:10488000DF4F6881CF5AD040C255DF4F4881CE5AA2
:10489000D0400E942D40B8C0033909F580919F0A8D
:1048A0009091A00A8230910508F4AEC00E94651D67
:1048B0000E94C41D082F0E94C41DC155DF4F88836C
:1048C000CF5AD0400E94C11D802F90E0C155DF4FCC
:1048D0006881CF5AD04070E00E94313C95C00838C2
:1048E00019F580919F0A9091A00A8430910508F4EF
:1048F0008BC08091A10A9091A20A00919F0A109109
:10490000A00A0396B9010E947F8E8E0F9F1FFC01A3
:10491000808190E004960817190708F475C00E947A
:10492000651D0E94041E70C0063999F480919F0A8B
:104930009091A00A8230910508F466C00E94651D1E
:104940000E94C11D082F0E94C11D802F0E947E6100
:104950005BC00739C9F480919F0A9091A00A823008
:10496000910508F451C00E94651D0E94C11D882355
:1049700011F484E006C0813019F40E940F3D44C058
:1049800082E00E94F03C40C0083991F480919F0A77
:104990009091A00A0097C1F10E94651D0E94C11D5F
:1049A0000E94FB2783E49BE060E00E94ED382CC06E
:1049B000093979F480919F0A9091A00A009721F11A
:1049C0000E94651D0E94CE1D8DE99AE00E9426324C
:1049D0001BC00A39C9F480919F0A9091A00A0097E0
:1049E00099F00E94651D0E94651D0E949A2D0CC0C1
:1049F0000E948C42882309F439CA40CA0E94104A96
:104A0000882309F458CA5FCAC155DF4F0FB6F8941E
:104A1000DEBF0FBECDBFCF91DF911F910F91FF90F1
:104A2000EF90DF90CF90BF90AF909F908F907F904E
:104A30006F905F904F903F902F90089580E092E0AC
:104A400090939E0A80939D0A1092A00A10929F0A4A
:104A50001092A20A1092A10A8DE998E09093A40AFC
:104A60008093A30A1092A50A1092A60A8CEA9AE0F3
:104A70000E94DA8C86EB9AE00E94DA8C80EC9AE055
:104A80000E94DA8C8AEC9AE00E94DA8C0895462F14
:104A9000FC0162816F700E94C05B0895FC0162811D
:104AA0006F700E94D55B0895DF93CF9300D000D044
:104AB00000D0CDB7DEB780913414909135149A832D
:104AC00089838B81807F8B83CE0101960E944E2546
:104AD000882379F480913214909133149D838C83D0
:104AE0008E81807F84608E83CE0104960E944E2545
:104AF00001C081E026960FB6F894DEBF0FBECDBF91
:104B0000CF91DF9108950F931F93DF93CF93CDB78C
:104B1000DEB72C970FB6F894DEBF0FBECDBF8C0169
:104B200080913414909135149A8389838B81807F8E
:104B30008B83CE0101960E944E25882391F58091AA
:104B40003414909135149D838C838E81807F816095
:104B50008E83CE01049661E00E94981D80913214EC
:104B60009091331498878F838985807F84608987AB
:104B7000CE0107960E944E25882321F0C8010E948D
:104B8000DC250FC080913414909135149B878A875F
:104B90008C85807F81608C87CE010A9660E00E94C0
:104BA000981D2C960FB6F894DEBF0FBECDBFCF91E7
:104BB000DF911F910F9108950F931F93DF93CF9370
:104BC000CDB7DEB72C970FB6F894DEBF0FBECDBFC2
:104BD0008C0180913414909135149A8389838B8150
:104BE000807F8B83CE01019660E00E94981D8091AA
:104BF0003414909135149D838C838E81807F8E83B5
:104C0000CE01049661E00E944725F8011082809150
:104C100032149091331498878F838985807F8460C4
:104C20008987CE0107960E944E25882319F0C80176
:104C30000E94832580913414909135149B878A8734
:104C40008C85807F81608C87CE010A9660E00E940F
:104C5000981D2C960FB6F894DEBF0FBECDBFCF9136
:104C6000DF911F910F9108950F931F93DF93CF93BF
:104C7000CDB7DEB72C970FB6F894DEBF0FBECDBF11
:104C80008C0180913414909135149A8389838B819F
:104C9000807F81608B83CE01019660E00E94981D29
:104CA00080913414909135149D838C838E81807F04
:104CB00081608E83CE01049661E00E944725809139
:104CC00032149091331498878F838985807F846014
:104CD0008987CE01079660E00E94981D809132146A
:104CE000909133149B878A878C85807F84608C8722
:104CF000CE010A9660E00E944725C8010E94DC258B
:104D0000F8011182128213822C960FB6F894DEBF3E
:104D10000FBECDBFCF91DF911F910F910895CF931B
:104D2000DF93EC018B81882329F485E00E94F03C1D
:104D300081E08B83DF91CF9108950F931F93DF93D1
:104D4000CF9300D00F92CDB7DEB78C01FC018281EA
:104D5000853128F0C8010E948F2680E024C0809110
:104D60003414909135149A8389838B81807F8B834F
:104D7000CE0101960E944E25882331F0F801118260
:104D800082818F5F82830EC0F8018181863028F096
:104D9000C8010E948325F8011182F80181818F5F8B
:104DA0008183128281E00F900F900F90CF91DF915D
:104DB0001F910F91089586ED9AE00E9468870895EB
:104DC000DF93CF9300D0CDB7DEB7BC0181E08983FC
:104DD00082E38A83CE01019642E050E00E94EE8F8A
:104DE0000F900F90CF91DF910895CF93DF93EC0157
:104DF00040E050E060EE70E40E94835DCE010296D8
:104E000046E656E666EA7EE30E94835DCE0104969E
:104E100040E050E060E172E40E94835DDF91CF9159
:104E200008950F931F93CF93DF93EB018B01085EDF
:104E30001F4F009719F4CB0167E002C0CB0168E374
:104E40000E94F88FC80162E30E94F88FCE010A9693
:104E50000E94F526CE0140960E94F526CE014A9684
:104E60000E94E026CE01069664EF71E00E940E904B
:104E7000CE01029665E070E00E940E90CE0104968D
:104E800064EF71E00E940E90CE0108966CE271E032
:104E90000E940E90DF91CF911F910F910895CF93B3
:104EA000DF93EC0140EA56E861E070E00E94069072
:104EB000CE01049649E150E060E070E00E94069067
:104EC000CE01089643EE5FE060E070E00E9406903D
:104ED000BE01605F7F4F85E49BE240E550E00E94A9
:104EE000EE8FDF91CF9108950F931F93DF93CF93B0
:104EF00000D00F92CDB7DEB78C0160E00E94F88F32
:104F0000C801029661E00E94F88F8FEF89831B82AF
:104F10001A82B8016C5F7F4FCE01019643E050E0EA
:104F20000E94EE8F0F900F900F90CF91DF911F9105
:104F30000F9108950F931F93DF93CF9300D000D06C
:104F4000CDB7DEB7082F162F80E491E067E04C83E1
:104F50000E94F88F09831A834C814B83CE010196FE
:104F600064E471E043E050E00E94EE8F0F900F90F8
:104F70000F900F90CF91DF911F910F910895EF92B5
:104F8000FF920F931F93CF93DF937B018C01EA0174
:104F9000CA01B7010E940E90CE010496B8010E948A
:104FA0000E90DF91CF911F910F91FF90EF90089598
:104FB000AC016BE770E084EF91E00E94BF27089599
:104FC000CF93DF93EC016CED70E00E940E90CE0168
:104FD00002966CED70E00E940E90CE01049664E69D
:104FE00070E00E940E90CE01069665E00E94F88F58
:104FF000DF91CF910895DF93CF93CDB7DEB76D9753
:105000000FB6F894DEBF0FBECDBFDE011596E0E10E
:10501000F6E085E001900D928150E1F781EC93E29A
:105020009A83898384E193ED9C838B8380E092E073
:1050300062E270E044E150E00E94EE8FCE010596FE
:1050400066E070E045E050E00E94EE8F84E090E082
:105050006FE90E94F88F8CE090E06BE10E94F88F7E
:10506000DE011A96ECEFF5E084E101900D9281509B
:10507000E1F782E490E061E00E94E55C882341F082
:1050800085EE9BE2A0E0B0E08A879B87AC87BD8776
:10509000CE010A966EE070E044E150E00E94EE8F8F
:1050A00080E691E061E00E94F88F84E790E00E9442
:1050B0004F2788E591E00E94E027CE01019664E445
:1050C00070E044E050E00E94EE8F80E090E060E00D
:1050D00071E00E94112781E090E06CE171E00E9494
:1050E000112780E491E00E9474278AE491E00E94F5
:1050F000D82786E591E060E00E94F88F6D960FB6A4
:10510000F894DEBF0FBECDBFCF91DF9108951F93FE
:10511000DF93CF93CDB7DEB764970FB6F894DEBFB9
:105120000FBECDBF182F833008F011E082E490E06D
:10513000612F0E94F88FDE011196E8EEF5E084E120
:1051400001900D928150E1F7113041F485EE9BE220
:10515000A0E0B0E089839A83AB83BC83CE01019643
:105160006EE070E044E150E00E94EE8F64960FB66E
:10517000F894DEBF0FBECDBFCF91DF911F91089590
:1051800082E490E061E00E94E55C91E0813009F00A
:1051900090E0892F089580E491E00E9474278AE4CA
:1051A00091E00E94D82788E591E00E94E02780E600
:1051B00091E061E00E94F88F0895DF93CF93CDB71F
:1051C000DEB72C970FB6F894DEBF0FBECDBF1982A5
:1051D0001A821B821C821D821E821F8218861986DB
:1051E0001A861B861C86CE01019662E671E04CE0B1
:1051F00050E00E94EE8F2C960FB6F894DEBF0FBEE3
:10520000CDBFCF91DF91089582E090E06CE00E94E5
:10521000F88F82E490E061E00E94F88F0E94DD2820
:105220000E94FB2708956F927F928F929F92AF9278
:10523000BF92CF92DF92EF92FF920F931F93DF9373
:10524000CF93CDB7DEB72F970FB6F894DEBF0FBE62
:10525000CDBF3C01D62E2F8338874987EA86FB864F
:105260000C87AD86BE86CF8680912E1490912F1428
:105270009A8389832B81207F22602B839D838C835B
:105280008E81807F85608E83C301BE01635F7F4F07
:10529000AE014F5F5F4F9E012C5F3F4F0E94B78C66
:1052A00089E196E0F30196878587D78690E1A92E5C
:1052B000B12CA60CB71CA301435F5F4F8AE0E82E18
:1052C000F12CE80CF91CC501B30100E211EA27E05A
:1052D00030E0CC24C3940E94B45ED301A059BF4FE8
:1052E000FE01379683E001900D928150E1F7F301C2
:1052F000ED58FF4FD082A401465E5F4FC3018C582A
:105300009F4FB5010A851B852C850E94945CF30193
:10531000E258FF4F918280822F960FB6F894DEBF3D
:105320000FBECDBFCF91DF911F910F91FF90EF90F6
:10533000DF90CF90BF90AF909F908F907F906F90B5
:1053400008950F931F93CF93DF93EC018C010059C5
:105350001F4FC80160E00E94981DC80161E00E94D3
:105360004725CE0140960E94BE5DCE010E941C8C56
:10537000CE018C589F4F0E946A5CDF91CF911F91A4
:105380000F910895CF93DF93EC0140960E94166031
:10539000CE018C589F4F0E94485CDF91CF910895B9
:1053A0008C589F4F662319F00E943A5C08950E9422
:1053B000655C0895882321F080918000806803C097
:1053C000809180008F73809380000895882321F05E
:1053D0008091A000806803C08091A0008F738093AB
:1053E000A00008950F931F93DF93CF9300D000D0B8
:1053F00000D0CDB7DEB7062F1FB7F894FC0182812D
:10540000882309F5862F81508E3FA0F080E00E940E
:10541000E62980913414909135149A8389838B8185
:10542000807F83608B8361E00F3F09F060E0CE01F5
:10543000019622C070E07093A9006093A80081E0FB
:105440000E94E62924C0813011F5862F81508E3FBD
:10545000B0F080E00E94DA298091281490912914FC
:105460009D838C838E81807F85608E8361E00F3F7A
:1054700009F060E0CE0104960E94981D08C070E01B
:10548000709389006093880081E00E94DA291FBF31
:1054900026960FB6F894DEBF0FBECDBFCF91DF9139
:1054A0001F910F910895CF93DF93EC010E94B41DDB
:1054B00091E089270E94AD1DCE0161E80E94B0876E
:1054C000DF91CF910895FC0183A194A1009741F051
:1054D00023A134A181E02430310519F480E008953E
:1054E00080E00895CF92DF92EF92FF920F931F9387
:1054F000CF93DF93EC018B018881882399F17E01A2
:10550000DC2ECF2CCE0160E00E94508787FF2AC09E
:105510000E944242882321F0CE010E94454208C0E9
:105520000E943F42882321F40E940A4A882321F1E5
:10553000C80161E80E94B08713C08D2D9C2D6C2F8F
:105540000E9450870E94F81E2196CE15DF05ACF30D
:10555000C80161E802C0C80162E80E94B08778947F
:1055600081E001C080E0DF91CF911F910F91FF900A
:10557000EF90DF90CF900895F894E8800E949F1DEF
:10558000FF248E159F0538F3C0E0D0E0DECF0895EC
:10559000CF93DF93EB0161E00E9455878A3191053B
:1055A00040F4CE0161E80E94B087CE0160E070E077
:1055B00007C0CE0161E80E94B087CE0166EF71E0BE
:1055C0000E94B387DF91CF9108959F92AF92BF92CF
:1055D000CF92DF92EF92FF920F931F93DF93CF93BF
:1055E000CDB7DEB765970FB6F894DEBF0FBECDBF5F
:1055F0006B01F8948E010F5F1F4FC8010E94114686
:10560000C60161E80E94B087C80160E070E00E94B6
:10561000833EFC014081518162817381C6010E94F9
:10562000C987C80161E070E00E94833EFC014081AF
:10563000518162817381C6010E94C987C80162E0FD
:1056400070E00E94833EFC01408151816281738140
:10565000C6010E94C98702E010E060E08DE1A82E3B
:10566000B12C0A9D70010B9DF00C1A9DF00C1124B9
:1056700083E49BE0E80EF91E962E990C990CC70165
:105680000E94D189882311F022E001C020E0C701E7
:105690002D8B0E94ED892D89622F6929682B01507D
:1056A00010409FEF0F3F1907E1F6C6010E94B08737
:1056B000789465960FB6F894DEBF0FBECDBFCF913C
:1056C000DF911F910F91FF90EF90DF90CF90BF90EF
:1056D000AF909F9008959F92AF92BF92CF92DF922A
:1056E000EF92FF920F931F93DF93CF93CDB7DEB767
:1056F00065970FB6F894DEBF0FBECDBF8B01F8944F
:105700007E010894E11CF11CC7010E941146C801EA
:1057100061E80E94B087C70160E070E00E94833EAC
:10572000FC014081518162817381C8010E94C98757
:10573000C70161E070E00E94833EFC01408151811D
:1057400062817381C8010E94C987C70162E070E06D
:105750000E94833EFC014081518162817381C801B6
:105760000E94C987C70163E070E00E94833EFC018C
:105770004081518162817381C8010E94C987C7013C
:1057800064E070E00E94833EFC01408151816281AF
:105790007381C8010E94C98724E0C22ED12C60E029
:1057A0009DE1A92EB12CCA9C7001CB9CF00CDA9C17
:1057B000F00C112483E49BE0E80EF91E962E990C60
:1057C000990CC7010E94D189882311F022E001C001
:1057D00020E0C7012D8B0E94ED892D89622F692958
:1057E000682B0894C108D1089FEFC9169FEFD9060E
:1057F000D1F6C80170E00E94B387789465960FB621
:10580000F894DEBF0FBECDBFCF91DF911F910F91F6
:10581000FF90EF90DF90CF90BF90AF909F90089552
:105820000F931F93CF93DF93EB018C010D5F1F4FFD
:10583000CB0161E80E94B087C8010E946B43682FCA
:10584000CE010E94B087DF91CF911F910F910895F3
:105850006F927F928F929F92AF92BF92CF92DF9280
:10586000EF92FF920F931F93DF93CF930F92CDB7D9
:10587000DEB77C018B01CDB6DEB68DB69EB6ADB679
:10588000BEB6CB0161E80E94B087C70161E00E940B
:105890005087882379F00E94AE43BC01009751F0F5
:1058A000C8010E94B087C80160E00E94B0873C2D0B
:1058B000292D37C08DB79EB74F970FB6F8949EBF6E
:1058C0000FBE8DBFEDB6FEB60894E11CF11CC701FA
:1058D0006FE140E050E00E944641BC01F701808149
:1058E000882329F06115710511F48E3281F3C80106
:1058F0000E94B08720E0E22FF0E02F3161F0EE0D42
:10590000FF1D6081662339F0C80129830E94B0879A
:1059100029812F5FF0CFC80160E00E94B0873A2D47
:105920002B2D832F922F0FB6F8949EBF0FBE8DBFE5
:105930000FB6F894DEBE0FBECDBE0F90CF91DF91B3
:105940001F910F91FF90EF90DF90CF90BF90AF909D
:105950009F908F907F906F9008958F929F92AF92BB
:10596000BF92CF92DF92EF92FF920F931F93DF933C
:10597000CF93CDB7DEB7A82EE92E6B018DB69EB6BC
:1059800061E00E9455878C018A2D9E2D63E00E9464
:105990005087482FA82EBB248DB79EB78A199B0924
:1059A0000FB6F8949EBF0FBE8DBFEDB6FEB608943D
:1059B000E11CF11CC701B80150E00E94D88FC6015C
:1059C00061E80E94B08700E010E008C0F701619133
:1059D0007F01C6010E94B0870F5F1F4F0A151B058C
:1059E000ACF30FB6F8949EBE0FBE8DBECF91DF9183
:1059F0001F910F91FF90EF90DF90CF90BF90AF90ED
:105A00009F908F9008952F923F924F925F926F9246
:105A10007F928F929F92AF92BF92CF92DF92EF923E
:105A2000FF920F931F93DF93CF930F92CDB7DEB703
:105A3000C82EB92E4B012DB63EB661E00E945587A7
:105A4000A82E792E8C2D9B2D63E00E945087D82E96
:105A5000482E55248DB79EB7841995090FB6F89432
:105A60009EBF0FBE8DBF0DB71EB70F5F1F4F602EBD
:105A70001983C8016A2D772D4D2D50E00E94D88FD3
:105A8000E02EF12E00E010E00BC0602F6C5F8C2D3B
:105A90009B2D0E945087F70181937F010F5F1F4F5D
:105AA0000415150594F3862D99816A2D772D4D2DBA
:105AB00050E00E94EE8FC40161E80E94B087C401EB
:105AC0006D2D0E94B0870FB6F8943EBE0FBE2DBE5E
:105AD0000F90CF91DF911F910F91FF90EF90DF908A
:105AE000CF90BF90AF909F908F907F906F905F907E
:105AF0004F903F902F9008950F931F93CF93DF9374
:105B0000EB0161E00E945087082F80FF02C00E94D5
:105B1000DF4501FF02C00E94E91DCE0161E80E943D
:105B2000B087CE0160E00E94B087DF91CF911F91D6
:105B30000F9108951092400B10923F0B08950F9310
:105B40001F93CF93DF938091100B882379F400E1AA
:105B50001BE0C2E2D0E0CE0160E00E94E55CF8010B
:105B600081938F012196C233D105A9F78091100B43
:105B7000882369F4A0E1BBE080E090E0FC01EC59EF
:105B8000FE4FE491ED9301968E309105B9F780E1D7
:105B90009BE0DF91CF911F910F91089580E29BE0F0
:105BA000089580913F0B9091400B089580E29BE017
:105BB0000E9437439C01009731F482E090E090937B
:105BC000400B80933F0BC9010895CF92DF92EF9273
:105BD000FF920F931F93CF93DF936C017B01CB0157
:105BE00061E80E94B08700E21BE0C1E0D0E008C09D
:105BF000C6016C2F0E945087F80181938F01219676
:105C0000F601808190E0C817D90794F310923E0BFB
:105C10000E94D62D682FC7010E94B087DF91CF91D7
:105C20001F910F91FF90EF90DF90CF9008950E9409
:105C3000554A882331F085E090E09093400B8093A3
:105C40003F0B0E94E91D0E94DF45089580913F0BA4
:105C50009091400B8130910571F484E090E0909335
:105C6000400B80933F0B86E09BE040E452E46FE002
:105C700070E00E94DE8C81E08093410B08952F92AA
:105C80003F924F925F927F928F929F92AF92BF927C
:105C9000CF92DF92EF92FF920F931F93DF93CF93F8
:105CA000CDB7DEB72C970FB6F894DEBF0FBECDBFD1
:105CB0008C017C876B87FC018081882309F4A9C152
:105CC000702E812EC80161E00E945087982EC80175
:105CD00062E00E945087E82FF0E0E632F10508F01C
:105CE00098C1EE58FF4FEE0FFF1F0590F491E02D85
:105CF00009948B859C8561E80E94B0878B859C8583
:105D000066EF71E083C18B859C8561E80E94B08756
:105D10000FE012E0F801E1908F018B859C856E2DDC
:105D20000E94B087EE2009F476C1F2E00E321F0720
:105D300089F771C181E08093410B30C08B859C85D0
:105D400061E80E94B087892D813019F0992031F0E7
:105D500009C01DE6E12E1CE0F12E04C0BDEEEB2EC5
:105D6000BBE0FB2EC701409676C0992D913019F00B
:105D7000992031F009C0ADE6CA2EACE0DA2E04C09D
:105D8000FDEECF2EFBE0DF2E872D982D62E00E94E6
:105D90005587BC01C60140960E94F45E8B859C85A8
:105DA00061E8C8C0C8016B857C850E94AD2C33C1F9
:105DB000C8016B857C850E94032D2DC18B859C8538
:105DC0000E94532A28C1E92DE13019F0992031F0C1
:105DD00009C0EDE6AE2EECE0BE2E04C07DEEA72E8F
:105DE0007BE0B72E872D982D62E00E945087682FA8
:105DF00070E061707070C5010E94D029CFCF802FF4
:105E0000912F63E00E945087682F70E0617070707E
:105E100083E49BE00E94B43BFEC08B859C8561E8D7
:105E20000E94B087F92DF13019F0992031F009C0A6
:105E30006DE6462E6CE0562E04C05DEE452E5BE00E
:105E4000552EC201409632C08B859C8561E80E9428
:105E5000B08789E79FE00E94B05FD5C08B859C85A5
:105E600061E80E94B087892D813019F0992031F0C6
:105E700009C04DE6242E4CE0342E04C03DEE232E06
:105E80003BE0332EC101409607C08B859C8561E8BD
:105E90000E94B08789E79FE00E94AA5FB4C08B850B
:105EA0009C8561E80E94B08789E79FE00E948E5F31
:105EB000682F3EC08B859C8561E80E94B087992D34
:105EC000913019F0992031F009C0EDE6FCE0FA8339
:105ED000E98304C08DEE9BE09A83898389819A814E
:105EE00040960E942561882311F000E801C000E07F
:105EF00089E79FE00E942561882311F080E401C0BA
:105F000080E0082B992D913019F0992031F009C0CB
:105F1000EDE6FCE0FC83EB8304C08DEE9BE09C830C
:105F20008B838B819C8140960E948E5F602F682BB3
:105F30008B859C850E94B0876EC08B859C8561E8AF
:105F40000E94B087992D913019F0992031F009C045
:105F5000EDE6FCE0FE83ED8304C08DEE9BE09E83C6
:105F60008D838D819E8140960E94B55FBC018B859B
:105F70009C850E94B387992D913019F0992031F0BA
:105F800009C0EDE6FCE0F887EF8304C08DEE9BE0EE
:105F900098878F838F81988540960E94B95FBC0156
:105FA0008B859C850E94B387992D913019F099209B
:105FB00031F009C0EDE6FCE0FA87E98704C08DEE18
:105FC0009BE09A87898789859A8540960E94BD5F64
:105FD000BC018B859C850E94B38789E79FE00E9466
:105FE000B55FBC018B859C850E94B38789E79FE0E4
:105FF0000E94B95FBC018B859C850E94B38789E7AD
:106000009FE00E94BD5FBC018B859C850E94B38789
:1060100002C080E001C081E02C960FB6F894DEBF8C
:106020000FBECDBFCF91DF911F910F91FF90EF90E9
:10603000DF90CF90BF90AF909F908F907F905F90B8
:106040004F903F902F900895EF92FF920F931F93E0
:10605000CF93DF938C01EB01FC018081882309F44D
:10606000CBC0C80160E00E94508787FDC5C0E82F03
:10607000F0E0EA31F10508F0BFC0E856FF4FEE0F3F
:10608000FF1F0590F491E02D0994C801BE010E9404
:10609000C82AB4C0CE0161E80E94B08700E2E02EB9
:1060A0000BE0F02E8701CE01F70161917F010E9484
:1060B000B087F8018081882309F4A0C0FFE3EF16C0
:1060C000FBE0FF0679F79AC080913F0B9091400B5F
:1060D0009C01215030402230310518F08530910567
:1060E00031F483E49BE064E070E00E94393781E0A2
:1060F0008093410BCE0161E80E94B0877FC0CE0142
:1061000061E80E94B0870E949F1DAC0160E070E0D2
:1061100017C0C801BE010E94E52A70C0C801BE01B7
:106120000E946B2B6BC0C801BE010E94102C66C080
:10613000CE0161E80E94B0870E94E042AB01BC0141
:10614000CE0157C0C801BE010E94E52D57C0C8014D
:10615000BE010E94282C52C0CE010E94532A4EC07C
:10616000C801BE010E943F2E49C0CE0161E80E94D5
:10617000B087F8940E946345882321F40E94B71DDC
:10618000882311F460E001C061E0CE010E94B08775
:10619000789434C0C801BE010E94AD2C2FC0C80144
:1061A000BE010E94032D2AC0C801BE010E947C2DA1
:1061B00025C0CE0161E80E94B087CE0140E050E0EA
:1061C000BA010E94C987CE0140E050E0BA010E94A6
:1061D000C987CE0140E050E0BA010E94C987CE01D4
:1061E00040E050E0BA010E94C987CE0140E050E093
:1061F000BA010E94C98702C080E001C081E0DF913E
:10620000CF911F910F91FF90EF9008950F931F93DF
:10621000DF93CF93CDB7DEB72A970FB6F894DEBFE2
:106220000FBECDBF8DE794E10E94632A882309F059
:10623000DBC08091060B882309F4D4C086E09BE084
:106240000E94FB8C882309F0CDC08E010F5F1F4F89
:10625000C8010E94DA8CA6E0BBE0F8018AE0019058
:106260000D928150E1F78FEF99E6A8E181509040BF
:10627000A040E1F700C0000001E08091410B8823BD
:1062800099F0002389F41092410B8091420B0E94F7
:1062900097321092420B8CEF9AE00E941E8D109262
:1062A000100B1092200B99C080917A1490917B145E
:1062B000009709F180917A1490917B1484309105B4
:1062C000D1F08091FC0A882349F48CEF9AE040E2F7
:1062D0005EE460E070E00E94DE8C0DC08CEF9AE01E
:1062E0000E94FB8C882339F087E594E10E94ED86BB
:1062F00084E08093791480917914882399F08091B7
:106300007914843029F483E49BE060E070E004C0F9
:1063100083E49BE063E070E00E94393787E594E115
:106320000E94FB8680917A1490917B1484309105B1
:10633000D1F58CEF9AE00E941E8D8DE794E10E94CA
:10634000708780913F0B9091400B86309105F1F062
:10635000002361F08DE794E169E80E94B08783E44F
:106360009BE066E070E00E94393715C087E594E154
:106370006DE774E10E94722A882369F487E594E14D
:106380006DE774E10E942430882329F48DE794E1BD
:1063900065E80E94B08787E594E10E94FB8683E56B
:1063A00094E10E94818D80913F0B9091400B82304F
:1063B000910541F40E943F42882321F41092400B42
:1063C00010923F0B80913F0B9091400B85309105CF
:1063D00059F40E940A4A882339F41092400B109213
:1063E0003F0B02C000E049CF2A960FB6F894DEBFFB
:1063F0000FBECDBFCF91DF911F910F910895CF9325
:10640000DF93FC0182819381009721F481E08187F1
:1064100080E019C08481958120813181B9010E9479
:106420007F8EC681D781C80FD91F8481958101963F
:10643000B9010E947F8E9583848382819381019725
:10644000938382838881DF91CF910895DF92EF92C9
:10645000FF920F931F93DF93CF93CDB7DEB76F9764
:106460000FB6F894DEBF0FBECDBF7C0180913F0B0D
:106470009091400B8130910591F1823091051CF48F
:10648000009739F13DC08230910521F085309105AA
:10649000B9F525C0DD248E010F5F1F4FC7010E9493
:1064A000FF31F801ED0DF11D8083D394FE01ED0D58
:1064B000F11D8081882391F7C80168E172E00E9494
:1064C000A08F0097E9F080E29BE0B8010E94A98FBD
:1064D00017C081E090E09093400B80933F0B00E069
:1064E000C7010E94FF31E02FF0E0E05EF44F8083AF
:1064F0000F5FE02FF0E0E15EF44F8081882381F7A9
:106500006F960FB6F894DEBF0FBECDBFCF91DF916F
:106510001F910F91FF90EF90DF9008958CEF9AE01C
:106520000E94DA8C86E09BE00E94DA8C0895DF936B
:10653000CF930F92CDB7DEB7682FF89484B7662358
:10654000A1F088E10FB6F89480936000109260008B
:106550000FBE14BE89E228E130E00FB6F894A8958A
:10656000209360000FBE8093600069830E94AF4259
:106570000E940D4A0E94DF450E94E91D0E94B65C00
:106580000E94158C83E49BE069810E94ED38789429
:106590000F90CF91DF91089583E49BE00E947246B3
:1065A00081E00E94973278940E9406310E94FE1E7C
:1065B00083E49BE00E94B137A895F6CFCF93DF9399
:1065C000EC010E94B05B8A81807F8A83CE010396B2
:1065D0000E94B05B8D81807F8D83CE0106960E94E4
:1065E000B05B8885807F8887CE0109960E94B05B6A
:1065F0008B85807F8B87CE010C960E94B05B8E8549
:10660000807F8E87CE010F960E94B05B8989807F44
:10661000898BDF91CF910895CF93DF93EC0187E6CB
:1066200097E099838883FE01EA5AFF4F1082CE01DA
:10663000865A9F4F0E94DA8CCE018C599F4F0E9440
:10664000A3821C82DF91CF910895CF93DF93EC0159
:1066500002960E94DA8CCE010C960E94DA8CCE0152
:1066600046960E94DA8CDF91CF910895CF93DF9305
:10667000EC0125EF37E0FC0121933193CF010E941B
:106680000E81CE010A960E94A382CE014B960E94F3
:10669000DA8CDF91CF910895CF93DF93EC0181E401
:1066A00098E099838883CE0105960E947783CE0176
:1066B0000E960E943633CE01C9960E94FA80CE0112
:1066C0008F5B9F4F0E940481DF91CF9108952F929D
:1066D0003F924F925F926F927F928F929F92AF9272
:1066E000BF92CF92DF92EF92FF920F931F93DF93AF
:1066F000CF93CDB7DEB7CE50D1400FB6F894DEBF02
:106700000FBECDBF3C0100E010E0C301800F911F20
:106710000E94DE32035E1F4F01391105B1F7C3013C
:106720008B569F4F0E94DA8CC30181569F4F0E9467
:10673000DA8C8091341490913514282F89839A83B0
:106740004B81407F43604B83E82E8C839D830E8179
:10675000007F04600E8380912E1490912F14A82E38
:106760008F8398875985507F53605987C301865519
:106770009F4F60E03A81F32EB884C52E812C71E0E2
:10678000972E0E9413298091281490912914282F64
:106790008A879B874C85407F45604C87E82E8D8794
:1067A0009E870F85007F06600F8780912E14909141
:1067B0002F14A82E888B998B5A89507F54605A8B3E
:1067C000C301865D9E4F61E03B85F32EB988C52EDF
:1067D0005CE1852E51E0952E0E9413291AEAA12E24
:1067E00011E0B12EA60CB71CC5010E942533BAECEE
:1067F0008B2EB1E09B2E860C971C80912A149091D1
:106800002B14482F8B8B9C8B6D89607F64606D8B04
:10681000082F8E8B9F8B288D207F2360288FC82E7A
:10682000898F9A8F3B8D307F32603B8FC4015C89AA
:10683000152FD52EE32E0E94176580912A14909172
:106840002B149D8F8C8F2E8D207F25602E8F98A3EB
:106850008F8F89A1807F866089A3C3018B549C4F51
:10686000C35FDE4F99838883CD50D140A6E34A2E83
:10687000A2E05A2E460C571CF8E52F2EF3E03F2ECF
:10688000260C371CC30183529E4FB501A4019E0103
:10689000245E3F4F8E01015E1F4F72016101C35F95
:1068A000DE4FA880B980CD50D1400E94B261C201B4
:1068B0000E945883F301EA5AFC4F87E798E09183DE
:1068C000808385E297E0F10191838083C301865A3A
:1068D0009C4F0E94A382C30185599C4F0E944C3358
:1068E000C35FDE4F88819981CD50D1400E940C3327
:1068F00083010E5D1B4FC8016FE040E00E94648B76
:10690000A3014C5C5B4F8FE196E0FA019183808399
:10691000C3018A5C9B4FB80100E513EC20E030E036
:10692000E0E1EE2EE1E0FE2ECC240E94B45EF30105
:10693000EA56FB4F81E080838091301490913114AE
:106940009BA38AA32CA1207F2CA39EA38DA32FA160
:10695000207F21602FA399A788A72AA5207F2260E6
:106960002AA720913A1430913B143CA72BA74DA5A0
:10697000407F41604DA73FA72EA728A9207F28ABC5
:106980009AAB89AB8BA9807F83608BABBCE78B2EE6
:10699000912C8C0E9D1EC401BE016E5D7F4FAE0119
:1069A0004B5D5F4F9E01285D3F4F8E01055D1F4F80
:1069B000AEE2EA2EF12CEC0EFD1EF1E3CF2ED12C2F
:1069C000CC0EDD1EE2E0AE2EB12C0E946689D30112
:1069D000F4018DE101900D928150E1F78091301426
:1069E000909131149DAB8CAB2EA9207F24602EABEF
:1069F00098AF8FAB29AD207F256029AF9BAF8AAFC1
:106A00002CAD207F26602CAF20913A1430913B149E
:106A10003EAF2DAF4FAD407F43604FAFDE01A05C76
:106A2000BF4F11963C932E93FE01EE5BFF4F2081EA
:106A3000207F22602083FE01ED5BFF4F91838083E6
:106A40008281807F8760828319E9812E912C8C0E50
:106A50009D1EC401BE016C5C7F4FAE01495C5F4F5F
:106A60009E01265C3F4F8E01035C1F4F7D016F012D
:106A7000E2E0AE2EB12C0E946689D3015D96F4014E
:106A80008DE101900D928150E1F7BE016A5B7F4F6D
:106A90008091381490913914FB0191838083228175
:106AA000207F2283AE01475B5F4FFA019183808391
:106AB0002281207F216022832CE4A22EB12CAC0EF7
:106AC000BD1EF501918380832281207F2260228375
:106AD000DE01A15BBF4F20913A1430913B14119617
:106AE0003C932E9312960C911297007F076012969A
:106AF0000C93129702E5E02EF12CEC0EFD1EF7012F
:106B0000318320832281207F2660228315E5C12ED8
:106B1000D12CCC0EDD1EF601918380838281807F93
:106B200083608283F6EB8F2E912C8C0E9D1EC40108
:106B300095018D01E2E0AE2EB12C0E946689D30151
:106B4000DA96F4018DE101900D928150E1F78E010A
:106B5000085A1F4F8091261490912714F8019183B1
:106B600080832281207F226022833BE5E32EF12C6B
:106B7000EC0EFD1EF701918380832281207F23602C
:106B800022832EE5C22ED12CCC0EDD1EF601918380
:106B900080838281807F8460828381E6A82EB12CED
:106BA000AC0EBD1EC5010E94B05BF5018281807FE5
:106BB0008283B4E68B2E912C8C0E9D1EC4010E9404
:106BC000B05BF4018281807F8283FE01E959FF4F2F
:106BD0008091261490912714918380838281807FF5
:106BE00085608283A3ED4A2E512C4C0E5D1EC2019E
:106BF000B801A7019601850174016F01E2E0AE2E94
:106C0000B12C0E946689D301A95ABF4FF2018DE1D0
:106C100001900D928150E1F78E0106591F4F80912E
:106C2000261490912714F801918380832281207F7C
:106C3000266022832DE6E22EF12CEC0EFD1EF701DC
:106C4000918380838281807F8760828390E7C92ED1
:106C5000D12CCC0EDD1E8091321490913314F601AC
:106C6000918380838281807F8260828383E7A82EE4
:106C7000B12CAC0EBD1EC5010E94B05BF501828136
:106C8000807F8283B6E78B2E912C8C0E9D1EC401D3
:106C90000E94B05BF4018281807F8283FE01E7580D
:106CA000FF4F8091361490913714918380838281B5
:106CB000807F86608283A0EF4A2E512C4C0E5D1E91
:106CC000C201B801A7019601850174016F01E2E0DC
:106CD000AE2EB12C0E946689D301AC58BF4FF20191
:106CE0008DE101900D928150E1F7C25FDE4F0FB64A
:106CF000F894DEBF0FBECDBFCF91DF911F910F91F2
:106D0000FF90EF90DF90CF90BF90AF909F908F90CB
:106D10007F906F905F904F903F902F9008956FB746
:106D2000F8948F569F4FFC0120813181428153811D
:106D30006FBFB901CA0108950F931F93CF93DF93DB
:106D4000EC01FC01EF56FF4F80819181A281B3815C
:106D500080589F4FAF4FBF4F80839183A283B383EF
:106D60000E94B41D8823D1F40E9436498E01095631
:106D70001B4FC8010E945425882381F0C8010E943E
:106D80009D26882359F4FE01E556FB4F81E0808360
:106D9000C356DB4F83E090E099838883DF91CF91E6
:106DA0001F910F910895CF93DF93EC01FC01E356FF
:106DB000FB4F7183608361307105E1F48A5C9B4F06
:106DC0000E9425618823D9F40E94C0288823B9F045
:106DD000CE0186549F4F0E9425618823A1F0CE01E9
:106DE000865C9E4F0E942561882369F008C081E07F
:106DF0008093E20FC556DB4F81E0888304C0809109
:106E0000E20F8823A1F3DF91CF91089581569F4F20
:106E100040E05CE866E877E40E94DE8C08951F920B
:106E20000F920FB60F920BB60F9211242F933F9330
:106E30004F935F936F937F938F939F93AF93BF9382
:106E4000EF93FF9383E49BE00E949C36FF91EF91C8
:106E5000BF91AF919F918F917F916F915F914F9172
:106E60003F912F910F900BBE0F900FBE0F901F9070
:106E700018950F931F93DF93CF9300D00F92CDB748
:106E8000DEB78B0161157105A1F41092E80F109225
:106E9000E70F80912814909129149A8389838B811C
:106EA000807F87608B83CE01019660E00E94981DF1
:106EB0000CC08091E40F90E08617970731F082E0D4
:106EC00090E09093E80F8093E70F0093E40F0F900A
:106ED0000F900F90CF91DF911F910F910895411561
:106EE000510531F41092EA0F1092E90F81E008C0C9
:106EF0006115710541F41092EA0F1092E90F80E0DC
:106F00000E949E6108956093E50F4093E60F81E033
:106F100090E09093EA0F8093E90F0895CF93DF9369
:106F2000EC0169E170E04FE050E00E946F37CE0164
:106F300083529E4F6FEF0E94AE64C456DB4F81E0D8
:106F40008883DF91CF910895CF93DF93EC01835233
:106F50009E4F0E948262CE010E948E37DF91CF91B8
:106F60000895EF92FF920F931F93CF93DF938C01BD
:106F7000FC01E755FF4F80818823E1F0FDEDEF2E06
:106F8000F1E0FF2EE00EF11EC7010E941E62E80133
:106F9000CB56DF4FCE010E94FB8C882359F0C701EE
:106FA0000E941D63C7010E942462AB01BC01CE0197
:106FB0000E94DE8CF801EA56FB4F8081882329F07D
:106FC000C8018A5C9B4F0E941660ECE9EE2EE4E05B
:106FD000FE2EE00EF11EF70180818823C1F0E8014A
:106FE000C352DE4FCE010E94B364882381F0C801F2
:106FF00060E070E040E050E00E946F370E943F4048
:10700000F7011082CE010E94DF621092E30FE801C7
:10701000C156DF4FCE010E94FB8C882309F446C085
:10702000F801E556FB4F8081882309F03FC0CE016F
:107030000E94218DE801C654DF4FCE010E94AA5F55
:107040001816190684F0C801865C9E4F0E94AA5F3C
:107050001816190644F0C8018A5C9B4F0E94AA5F6B
:107060001816190684F4C80183529E4F63E272E039
:107070000E948262C8010E948E3780E060E04FEF7C
:1070800021E00E94513FCE0160E070E00E94F45E7A
:10709000C801865C9E4F60E070E00E94F45EC8010B
:1070A0008A5C9B4F60E070E00E94F45EE801C55688
:1070B000DB4F8881882309F47FC08091E30F882308
:1070C00009F07AC00E94EF3B882309F075C081E087
:1070D0008093E30FC8016AE070E04AE050E00E944C
:1070E0006F37C80186549F4F60E070E00E94F45EE5
:1070F000C801865C9E4F60E070E00E94F45EC801AB
:107100008A5C9B4F60E070E00E94F45EF801E356F9
:10711000FB4F8081918183309105B9F084309105D6
:107120003CF48130910529F18230910571F507C059
:107130008430910591F08530910539F514C0C8016E
:1071400083529E4F69E472E005C0C80183529E4F8E
:1071500069E972E00E94826218C0C80183529E4FA2
:1071600069EE72E0F7CFC80183529E4F6AE373E085
:10717000F1CFC80183529E4F6CE873E00E94826297
:10718000C8010E948E37188221C00E94443F0E948D
:10719000C72A0E94B01DF801EB5CFD4F81E080839F
:1071A0000E94DF45C0E0D0E08C2F60E00E941249D1
:1071B0002196C530D105C1F7C80186559F4F0E9461
:1071C000C229C801865D9E4F0E94C229DF91CF91DE
:1071D0001F910F91FF90EF900895BF92CF92DF9291
:1071E000EF92FF920F931F93DF93CF93CDB7DEB74C
:1071F0002F970FB6F894DEBF0FBECDBF8C01B62E11
:1072000060E070E00E94393782E090E060E00E9428
:10721000E55CE82E83E890E10E9466448E2D80951F
:10722000881F8827881F0E946346EE24FF248DE173
:10723000C82ED12CEC9CC001ED9C900DFC9C900DB7
:107240001124800F911F6E2D0E944F8A0894E11C1B
:10725000F11C85E0E816F10469F783E594E161E04B
:107260000E94A18D87E594E10E94FB86C8018655A6
:107270009F4F0E94A129C801865D9E4F0E94A129AF
:10728000C80186549F4F60E070E00E94F45EC80120
:10729000865C9E4F60E070E00E94F45EB6E3CB2E09
:1072A000B4E0DB2EC00ED11EC60160E070E00E948B
:1072B000F45E21E024BD25BD17BC18BC10926E0001
:1072C0001092900089E0809391001092920080E0EB
:1072D00098E0909399008093980082E080937100E9
:1072E0001092B00097E09093B1002093700010923C
:1072F00020018093210110922901109228011092FF
:107300002B0110922A011092730093E09093800059
:1073100083E180938100109289001092880010927E
:107320008B0010928A0010926F009093A0008093BF
:10733000A1001092A9001092A8001092AB00109228
:10734000AA00109272000E942A61F801E755FF4FCF
:1073500080838823A9F1ADEDEA2EA1E0FA2EE00E9C
:10736000F11EC7010E94A06286E591E060E00E94E4
:10737000E55C882321F4B80165597C4F03C0B8014E
:107380006A5A7C4FC7010E943A62BB2049F08FEFD6
:107390009BE7A2E981509040A040E1F700C00000C7
:1073A000B80166537E4FC7010E948661C7010E94E3
:1073B0002462AB01BC01C8018B569F4F0E94DE8C3A
:1073C000C80160E070E040E050E00E946F37BB20F1
:1073D00009F44DC080912814909129149A838983CF
:1073E0008B81807F87608B83CE01019661E00E9454
:1073F000472580912A1490912B149D838C838E8134
:10740000807F81608E83CE01049661E00E944725D3
:1074100080912A1490912B1498878F838985807F7F
:107420008987CE01079661E00E944725809132143A
:10743000909133149B878A878C85807F81608C87AD
:10744000CE010A9661E00E9447250E94D0400E942A
:107450004C3DF801E556FB4F1082F801E356FB4F17
:1074600011821082C80189569B4F0E9434260E94C7
:107470003F4080913A1490913B149E878D878F8571
:10748000807F84608F87CE010D9661E00E94472542
:10749000C8018E5D9B4F0E945D8BC6010E94BE5D40
:1074A000F801E456FB4F10822F960FB6F894DEBF1A
:1074B0000FBECDBFCF91DF911F910F91FF90EF9045
:1074C000DF90CF90BF9008951F920F920FB60F924A
:1074D0000BB60F9211242F933F934F935F936F93AB
:1074E0007F938F939F93AF93BF93EF93FF93DF931C
:1074F000CF93CDB7DEB72997DEBFCDBF8091EB0F1D
:107500009091EC0F1816190614F401973FC0809162
:10751000E70F9091E80F8130910519F58091ED0FFB
:107520009091EE0F01969093EE0F8093ED0F82E015
:1075300090E09093E80F8093E70F82E190E09093C2
:10754000EC0F8093EB0F80912814909129149A836B
:1075500089838B81807F87608B83CE01019660E079
:1075600053C08230910581F58091E40F90E0209125
:10757000ED0F3091EE0F281739076CF083E090E0A3
:107580009093E80F8093E70F80E590E09093EC0FE5
:107590008093EB0F3BC081E090E09093E80F8093E5
:1075A000E70F82E190E09093EC0F8093EB0F8091D6
:1075B0002814909129149D838C838E81807F87600D
:1075C0008E83CE0104961FC083309105F9F410928A
:1075D000EE0F1092ED0F81E090E09093E80F809312
:1075E000E70F82E190E09093EC0F8093EB0F809196
:1075F00028149091291498878F838985807F8760CC
:107600008987CE01079661E00E94981D8091EF0F57
:107610009091F00F1816190634F401979093F00F1B
:107620008093EF0F27C08091E90F9091EA0F81308E
:10763000910571F482E090E09093EA0F8093E90F56
:107640008091E50F8093EF0F1092F00F81E010C052
:107650008230910579F481E090E09093EA0F809375
:10766000E90F8091E60F8093EF0F1092F00F80E00A
:107670000E949E612996DEBFCDBFCF91DF91FF9121
:10768000EF91BF91AF919F918F917F916F915F919A
:107690004F913F912F910F900BBE0F900FBE0F9007
:1076A0001F9018951F920F920FB60F920BB60F9264
:1076B00011242F933F934F935F936F937F938F93F7
:1076C0009F93AF93BF93EF93FF930E94973DFF91DA
:1076D000EF91BF91AF919F918F917F916F915F914A
:1076E0004F913F912F910F900BBE0F900FBE0F90B7
:1076F0001F901895882321F080912001806203C09B
:10770000809120018F7C8093200108950F931F9317
:10771000DF93CF9300D00F92CDB7DEB7062F1FB700
:10772000F89480E00E947A3B80913A1490913B1447
:107730009A8389838B81807F84608B8361E00023BF
:1077400009F460E0CE0101960E94981D1FBF0F90C2
:107750000F900F90CF91DF911F910F910895FC0131
:10776000EA56FB4F608308950F931F93DF93CF93E7
:1077700000D000D000D0CDB7DEB7062F1FB7F894E9
:1077800080913A1490913B149A8389838B81807FF6
:1077900085608B83CE01019661E00E944725809130
:1077A0003A1490913B149D838C838E81807F8560F9
:1077B0008E83CE010496602F0E94981D1FBF2696CF
:1077C0000FB6F894DEBF0FBECDBFCF91DF911F91F2
:1077D0000F91089583E49BE00E94673308958091A0
:1077E000FF0F0895FC019B0182819381608171816B
:1077F00086179707B8F44281538184819581840F5D
:10780000951F0E947F8E880F991FA681B781A80FB0
:10781000B91F11963C932E93828193810196938395
:107820008283089581E080870895CF93DF939C0140
:10783000EB0180915F109091601040915D1050912C
:107840005E104817590751F08DE590E1B9010E948B
:10785000F23B87E690E1BE010E94F23BDF91CF91BF
:1078600008950F931F93CF93DF93EC018B018091C9
:10787000FE0F882321F0CE010E94153CACC08AE4A3
:1078800091E061E00E94E55C882309F4A4C081E0F6
:107890008093FF0F8093FE0F81EF9FE060E00E94D6
:1078A000981D81EF9FE061E00E9447259E0140E026
:1078B00050E060E072E18AE790E00E94A68EDA0173
:1078C000C901B695A795979587950197A109B10923
:1078D0008093041090930510A0930610B0930710A6
:1078E0008F3F9105A105B10509F008F444C0DA0104
:1078F000C901F4E0B695A79597958795FA95D1F7C4
:107900000197A109B1098F3F9105A105B105A9F121
:10791000A0F1DA01C901E7E0B695A795979587959B
:10792000EA95D1F70197A109B1098F3F9105A1050A
:10793000B10529F120F1DA01C90179E0B695A795E1
:10794000979587957A95D1F70197A109B1098F3F4E
:107950009105A105B105A9F0A0F0DA01C9016BE01C
:10796000B695A795979587956A95D1F70197A1093F
:10797000B10925E007C021E005C022E003C023E0F3
:1079800001C024E0285F25BD87BD88BD82E08093CB
:107990006E00BE0180E090E0660F771F881F991F80
:1079A000980140E050E00E94608E28EE33E040E015
:1079B00050E00E94C88E2093001030930110409335
:1079C0000210509303101092081010920910109298
:1079D0000A1010920B10DF91CF911F910F91089513
:1079E0000F931F93CF93DF9300E010E0C82FD0E0F8
:1079F0000EC08EEE91E06CE271E00E94313C88EBAB
:107A000091E06CE271E00E94313C0F5F1F4F0C1758
:107A10001D077CF3DF91CF911F910F91089580E7AF
:107A200093E06CEB70E00E94313C80E090E06CEB06
:107A300070E00E94313C80EE96E06CEB70E00E94BA
:107A4000313C80E090E06CEB70E00E94313C88EBD0
:107A500097E06CEB70E00E94313C80E090E06CEBD2
:107A600070E00E94313C8DE298E06CEB70E00E9487
:107A7000313C89EA98E06CEB70E00E94313C80E098
:107A800090E06CEB70E00E94313C80EC9DE06DE496
:107A900071E00E94313C089580EC9DE060E271E06D
:107AA0000E94313C80E090E06CEB70E00E94313C41
:107AB00083E591E16CEB70E00E94313C80E090E066
:107AC0006CEB70E00E94313C8BE592E161EB71E080
:107AD0000E94313C0895CF93DF93FC018281938112
:107AE000009729F481E0818720E030E01CC0848188
:107AF000958120813181B9010E947F8E880F991F65
:107B0000C681D781C80FD91F848195810196B9019B
:107B10000E947F8E958384838281938101979383D2
:107B2000828328813981C901DF91CF910895CF9354
:107B3000DF938091001090910110A0910210B091FC
:107B400003100097A105B10511F160910C1081E0BF
:107B5000682760930C1081EF9FE00E94981D809130
:107B6000001090910110A0910210B09103100097A5
:107B7000A105B10569F10197A109B1098093001030
:107B800090930110A0930210B093031021C01092A3
:107B90006E0018BC17BC81EF9FE060E00E94981D4A
:107BA0001092FE0F80915F1090916010009771F01D
:107BB0008DE590E10E946B3DEC0187E690E10E942B
:107BC0006B3DBC01CE010E94313C02C01092FF0F00
:107BD000DF91CF9108958091321490913314909356
:107BE000F20F8093F10F8091F30F807F8560809377
:107BF000F30F84EF9FE00E94DA8C84E190E0909391
:107C00005E1080935D101092601010925F101092C1
:107C10006210109261102DE030E1309364102093D7
:107C20006310109265101092661090936810809304
:107C3000671010926A101092691010926C101092D6
:107C40006B1085E390E190936E1080936D1010920D
:107C50006F1010927010089508958F929F92AF92B6
:107C6000BF92CF92DF92EF92FF920F931F93DF9319
:107C7000CF93CDB7DEB7FC0140835183628373831A
:107C80000483158326833783C086D186E286F386F4
:107C900084869586A686B7868F859889A989BA89AC
:107CA000808B918BA28BB38BCF91DF911F910F9122
:107CB000FF90EF90DF90CF90BF90AF909F908F900C
:107CC0000895CF92DF92EF92FF920F931F93FC01E2
:107CD00040835183628373830483158326833783B0
:107CE000C086D186E286F3861486158616861786A8
:107CF000108A118A128A138A1F910F91FF90EF90B8
:107D0000DF90CF900895660F771F660F771F680F7B
:107D1000791FCB010895660F771F660F771F680FD5
:107D2000791FCB010895DF93CF9300D000D0CDB75A
:107D3000DEB795E099836C83882349F481E08B83D7
:107D4000842F80959091711089234A7A09C08130DF
:107D500011F583E08B83842F809590917110892396
:107D6000842B8A8384ECBE016F5F7F4F42E00E94C8
:107D7000C54985E08A95F1F7000084ECBE016D5F8E
:107D80007F4F42E00E94C54985E08A95F1F70000E7
:107D90008A81809371100F900F900F900F90CF9168
:107DA000DF910895DF93CF9300D0CDB7DEB795E094
:107DB0009983262F209590917110882321F092238A
:107DC0006575962B01C092239A8384ECBE016F5F88
:107DD0007F4F42E00E94C5498A81809371100F90C5
:107DE0000F90CF91DF910895DF93CF9300D000D013
:107DF000CDB7DEB795E099831A821C821B826C8313
:107E0000882349F482E08B83842F809590917110B0
:107E100089234A7A09C0813019F584E08B83842F45
:107E20008095909171108923842B8A8384ECBE0104
:107E30006F5F7F4F42E00E94C54985E08A95F1F768
:107E4000000084ECBE016D5F7F4F42E00E94C54997
:107E500085E08A95F1F700008A818093711007C050
:107E600081E0662309F480E0642F0E94D23E0F90E7
:107E70000F900F900F90CF91DF91089583E060E015
:107E80004FE30E94F43E08950E943E3F81E068EC7B
:107E900043E00E94F43E81E062E843E00E94933EAA
:107EA0000895CF92DF92EF92FF920F931F93DF938B
:107EB000CF930F92CDB7DEB7F82E162F042F2223C3
:107EC00021F099830E943E3F99812F2D2F3F09F485
:107ED00093E01F3F09F49C600F3F09F4906383E037
:107EE00061E0492F0E94F43E9F2D915081E09E3F1A
:107EF00008F080E0282F30E0912F91509E3F10F441
:107F00002F5F3F4FE02EEA944E2D4E3F18F4223063
:107F10003105A1F1882389F080E06091721043E07F
:107F200099830E94933E80E06F2D43E00E94F43ECF
:107F300081E0C82ED12C998102C0CC24DD249E3F43
:107F400078F4FC2C8C2D609172104CE00E94933ED2
:107F50000894C11CD11C8F2D612F4CE00E94F43E6F
:107F60008E2D8E3F08F06FC08C2D6091721040E313
:107F70000E94933E8C2D602F40E363C0EF2DF0E014
:107F8000202F30E0DF01A21BB30BB7FF03C0B09579
:107F9000A195BF4F812F90E0E81BF90BF7FF03C0BD
:107FA000F095E195FF4F281B390B37FF03C0309543
:107FB00021953F4FAE17BF07C4F4A217B3076CF566
:107FC00080E0609172104CE00E94933E80E0612F4F
:107FD0004CE00E94F43E81E06091721043E30E9405
:107FE000933E81E06F2D43E32CC0E217F307ACF41E
:107FF00080E06091721040E30E94933E80E0602F29
:1080000040E30E94F43E81E0609172104FE00E94D4
:10801000933E81E0612F4FE014C080E060917210C8
:1080200043E00E94933E80E06F2D43E00E94F43EC7
:1080300081E0609172104CE30E94933E81E0612FD9
:108040004CE30E94F43E0F90CF91DF911F910F916E
:10805000FF90EF90DF90CF900895FF920F931F93C2
:10806000F82E062F142F0E949A278F2D602F412F54
:1080700021E00E94513F1F910F91FF900895EF92D0
:10808000FF920F931F930E943E3F80E491E061E0D6
:108090000E94E55C182F84E491E04FEF5FEF6FEFF3
:1080A0007FEF0E941F5D133009F44EC0143028F496
:1080B000113011F1123098F50BC0153099F01530D0
:1080C00020F1163009F449C0173009F05FC051C0E3
:1080D00081E0609172104FE30E94933E81E064E67C
:1080E0004FE344C081E06091721040E30E94933EF0
:1080F00081E064E640E33AC081E06091721043E0C1
:108100000E94933E81E064E61DC081E060917210A0
:108110004CE00E94933E81E064E64CE027C081E0A1
:10812000609172104CE00E94933E81E062E34CE06B
:108130000E94F43E80E06091721043E00E94933E02
:1081400080E068EC43E012C081E06091721043E38C
:108150000E94933E81E066E408C081E06091721065
:1081600043E30E94933E81E068EC43E30E94F43EC7
:108170000DC07C0100271127272F382F492F5527A5
:10818000892F6E2D422F21E00E94513F1F910F91A8
:10819000FF90EF900895809372100E943F400895E1
:1081A0000E94044A0E943F4008950F938FE298E591
:1081B00062ED78E540E05AE527EC3AE500E00E9400
:1081C000B3569093741080937310009779F48FE2F4
:1081D00098E562ED78E540E05AE527EC3AE50FEFE7
:1081E0000E94B356909374108093731081E0209195
:1081F0007310309174102115310509F480E00F914E
:10820000089580917310909174100E94DF4F9C012B
:10821000909376108093751081E02115310509F453
:1082200080E008950F931F93DF93CF93CDB7DEB710
:10823000AB970FB6F894DEBF0FBECDBF809175101F
:10824000909176106DED73E08E010F5F1F4FA801C6
:108250000E9436558091751090917610B8010E9459
:1082600022549C01909378108093771081E021151F
:10827000310509F480E0AB960FB6F894DEBF0FBE6F
:10828000CDBFCF91DF911F910F9108958F929F9253
:10829000BF92CF92DF92EF92FF920F931F93DF93E3
:1082A000CF93CDB7DEB7AB970FB6F894DEBF0FBE56
:1082B000CDBF7C014A0185E0B82E6E010894C11C37
:1082C000D11C062F10E00150104080917710909142
:1082D0007810B6010E9465548823E1F0D701F601B9
:1082E00080E090E08017910734F42191222319F067
:1082F0002D930196F7CFF701E80FF91F1082009731
:1083000031F08114910441F0F401808305C0BA94E6
:10831000E1F602C0F701108280E090E0AB960FB664
:10832000F894DEBF0FBECDBFCF91DF911F910F91AB
:10833000FF90EF90DF90CF90BF909F908F90089527
:108340000F931F93CF93DF938C01EB010EC0CE01EF
:10835000B8010E94A08F009741F48091771090910E
:1083600078100E94C15581E009C0809177109091EA
:108370007810BE010E946554882349F7DF91CF91A0
:108380001F910F910895EF92FF920F931F93DF9328
:10839000CF93CDB7DEB7AB970FB6F894DEBF0FBE65
:1083A000CDBF7B018E010F5F1F4FB8010E94A0411E
:1083B000882361F08091751090917610B8010E9429
:1083C0008451F7019183808381E001C080E0AB9606
:1083D0000FB6F894DEBF0FBECDBFCF91DF911F91D6
:1083E0000F91FF90EF9008950F931F93DF93CF931A
:1083F000CDB7DEB7AB970FB6F894DEBF0FBECDBFDB
:108400008E010F5F1F4FB8010E94A041882349F0E1
:108410008091751090917610B8010E94315681E0DC
:1084200001C080E0AB960FB6F894DEBF0FBECDBFA3
:10843000CF91DF911F910F910895DF93CF93CDB727
:10844000DEB7AB970FB6F894DEBF0FBECDBFBC0151
:108450008091771090917810AE014F5F5F4F0E942E
:10846000CE5591E0882309F490E0892FAB960FB6A2
:10847000F894DEBF0FBECDBFCF91DF9108958091FC
:108480007C10089580917B100895CF93DF93EC01C9
:108490008091791090917A100097E1F0BE016E5FA3
:1084A0007F4F488150E00E94DE52288180917D10EC
:1084B00090917E10A0917F10B0918010820F911D3D
:1084C000A11DB11D80937D1090937E10A0937F100D
:1084D000B0938010DF91CF9108950E94DD578823DB
:1084E00091F08091791090917A1061E870E141E00B
:1084F00050E00E94CF5121E0181619060CF020E040
:1085000020938210089583E49BE06FED73E00E9456
:10851000A437109282100895809182100895DF93FD
:10852000CF930F92CDB7DEB78091811089830E94DF
:108530006D4289810F90CF91DF91089510927C1048
:108540008091791090917A10009721F00E94BC518F
:108550000E94135810927A10109279100895809109
:108560007C10882311F00E949E4280917B1088230A
:1085700011F00E94E042809177109091781000975E
:1085800031F00E945F541092781010927710809111
:10859000751090917610009731F00E947E511092E4
:1085A000761010927510809173109091741000974E
:1085B00031F00E9485571092741010927310089534
:1085C00080917B10882381F08091791090917A10AE
:1085D000009721F00E94BC510E94135810927A100B
:1085E0001092791010927B100E94AF4260917D1022
:1085F00070917E1080917F109091801008950E945C
:108600004259882371F40E94DD57882329F40E947F
:10861000AF4221E030E029C00E94AF4222E030E0CA
:1086200024C00E94D540882329F40E94AF4223E051
:1086300030E01BC00E940141882329F40E94AF4210
:1086400024E030E012C00E941241882329F40E94E5
:10865000AF4225E030E009C00E94F957882319F0A5
:1086600026E030E002C020E030E0C9010895CF9359
:10867000DF93EC010E94AF420E94FF429C010097F1
:1086800019F086309105D9F410927D1010927E1069
:1086900010927F101092801010927A101092791020
:1086A000CE0169E770E10E94C341882331F08091D7
:1086B000791090917A10009731F427E030E0C901E9
:1086C000DF91CF91089581E080937C100E946D42EC
:1086D00020E030E0F4CFEF92FF920F931F93CF93FF
:1086E000DF938C010E94AF420E94FF42EC01009791
:1086F00069F510927D1010927E1010927F101092EA
:10870000801010927A1010927910C8010E94F441E2
:10871000C8010E941D42882389F0C80169E770E101
:108720000E94C341882369F08091791090917A105A
:10873000009751F081E080937B1008C0C7E0D0E043
:1087400005C0C3E0D0E002C0C8E0D0E0CE01DF91B8
:10875000CF911F910F91FF90EF9008950E94AF422B
:108760000E94FF429C01009719F08630910541F468
:1087700080917710909178100E94C15520E030E0F0
:10878000C9010895CF92DF92EF92FF920F931F934A
:10879000DF93CF93CDB7DEB72F970FB6F894DEBF38
:1087A0000FBECDBF8C01EE24FF246801CE0CDF1C70
:1087B000C6010E94B05BF6018281807F828383E0E4
:1087C00090E0E80EF91E9FE0E916F10471F7809140
:1087D000361490913714F801908B87878189807FB8
:1087E0008560818B85E0828B80913014909131146B
:1087F0009A838983D801FE01319683E001900D921E
:108800008150E1F7F8018281807F836082838091CB
:108810003014909131149D838C83D8011396FE01FE
:10882000349683E001900D928150E1F7F801858143
:10883000807F876085838091381490913914988760
:108840008F83D8011696FE01379683E001900D9232
:108850008150E1F7F8018085807F83608087809177
:108860002614909127149B878A87D8011996FE01B8
:108870003A9683E001900D928150E1F7F8018385EB
:10888000807F8560838780913614909137149E870E
:108890008D87D8011C96FE013D9683E001900D92D4
:1088A0008150E1F7F8018685807F866086872F9664
:1088B0000FB6F894DEBF0FBECDBFCF91DF911F91F1
:1088C0000F91FF90EF90DF90CF900895FF920F935C
:1088D0001F93CF93DF938C01FF2412C08F2D90E064
:1088E000EC01CC0FDD1FC80FD91FC00FD11FCE0167
:1088F00061E00E944725CE0161E00E94981DF3943B
:10890000F8018289F81650F3015F1F4FC80161E03A
:108910000E944725C80161E00E94981DDF91CF9118
:108920001F910F91FF9008951F93CF93DF93EC0158
:1089300085E18A95F1F70000CE010F9661E00E9473
:10894000981D85E18A95F1F7000010E00DC0212FF8
:1089500030E0C901880F991F820F931F8C0F9D1F54
:1089600061E00E94981D1F5F8A89181780F385E1D6
:108970008A95F1F70000DF91CF911F910895AF9292
:10898000BF92CF92DF92EF92FF920F931F93DF93EC
:10899000CF9300D00F92CDB7DEB7B62E29833A839E
:1089A0004B8378E0C72ED12C60E8A62E8E010F5F96
:1089B0001F4F5FE0E52EF12CE80EF91E8A2D8B216A
:1089C00061E009F460E0C8010E94981DC70161E000
:1089D0000E94981D85E18A95F1F70000C70160E0CB
:1089E0000E94981DA6940894C108D108C114D1040E
:1089F00029F7C80161E00E94981DC80160E00E944B
:108A00004725C70161E00E94981DC8010E944E25BC
:108A1000C82EC70160E00E94981DC80161E00E9455
:108A2000472581E0C11080E00F900F900F90CF910B
:108A3000DF911F910F91FF90EF90DF90CF90BF904B
:108A4000AF900895EF92FF920F931F93DF93CF9310
:108A500000D00F92CDB7DEB78C01F62E29833A8372
:108A60004B83EE240DC02E2D30E0C901880F991FD5
:108A7000820F931F800F911F60E00E94981DE39466
:108A8000F8018289E81678F3F5E1FA95F1F700002C
:108A9000C8010F9660E00E94981DC8016F2D2981C2
:108AA0003A814B810E94BF440F900F900F90CF915D
:108AB000DF911F910F91FF90EF90089583E890E16F
:108AC0000E94C243089580919610882319F48091E2
:108AD0002611089581E008955F926F927F928F92A0
:108AE0009F92AF92BF92CF92DF92EF92FF920F933D
:108AF0001F93CF93DF935FB6F89407E211E17801FB
:108B0000C2E6D1E09AE0A92EB12CC12CD12C82E092
:108B1000682E712C812C912CCE0140E050E0BA01DE
:108B20000E941F5DA60195010E94C88ECA01B9016D
:108B3000A40193010E94C88EF701219331934193C0
:108B400051937F012496F1E0CE36DF0729F710928A
:108B50003311109234111092351110923611109277
:108B60003711109238111092391110923A11EBE32B
:108B7000F1E1E80189919991A991B9918E01B0959E
:108B8000A095909581959F4FAF4FBF4F8193919343
:108B9000A193B19381E1CB33D80759F75FBEDF9141
:108BA000CF911F910F91FF90EF90DF90CF90BF90EA
:108BB000AF909F908F907F906F905F9008951092EC
:108BC0009610109226110E946C450895EF92FF9224
:108BD0000F931F93CF93DF938C01C0E0D0E02BE184
:108BE000E22EF12CC801BE010E94833EFC01CE9D05
:108BF000C001CF9D900DDE9D900D112440815181CB
:108C00006281738181569F4E0E946D882196C53086
:108C1000D10541F7DF91CF911F910F91FF90EF9018
:108C200008958F929F92AF92BF92CF92DF92EF9270
:108C3000FF920F931F93CF93DF93EC014091A1100C
:108C40005091A2106091A3107091A4100091BC10DB
:108C50001091BD102091BE103091BF10C090D71060
:108C6000D090D810E090D910F090DA108090F210E7
:108C70009090F310A090F410B090F51080910D1129
:108C800090910E11A0910F11B091101100D000D051
:108C9000EDB7FEB781839283A383B483CE010E9494
:108CA0002D3E0F900F900F900F90CE01DF91CF913E
:108CB0001F910F91FF90EF90DF90CF90BF90AF90FA
:108CC0009F908F900895809351110895813019F4E9
:108CD0008BE391E102C087E291E190935011809380
:108CE0004F1108958F929F92AF92BF92CF92DF92D1
:108CF000EF92FF920F931F93DF93CF93CDB7DEB721
:108D00006B970FB6F894DEBF0FBECDBF5C0110921B
:108D100096104FE9E42E40E1F42E00E010E03DE132
:108D2000832E912C6E010894C11CD11C089DB001AA
:108D3000099D700D189D700D11246A0D7B1DC601D3
:108D40000E94F787D701F6018BE101900D928150C7
:108D5000E1F70F5F1F4F8BE190E0E80EF91E053041
:108D6000110521F782E691E04FEF5FEF6FEF7FE7AC
:108D70000E941F5D6F3F2FEF72072FEF82072FE7D3
:108D8000920711F40E94DD280E946C4580E00E9449
:108D900066466B960FB6F894DEBF0FBECDBFCF917F
:108DA000DF911F910F91FF90EF90DF90CF90BF90D8
:108DB000AF909F908F9008952F923F924F925F9225
:108DC0006F927F928F929F92AF92BF92CF92DF92DB
:108DD000EF92FF920F931F93CF93DF931C012A0111
:108DE0003B01CC24DD248824992454018BE190E0BC
:108DF000C89EE001C99ED00DD89ED00D1124C15649
:108E0000DF4EC101B6010E94833EFC0140815181C9
:108E100062817381CE0120E00E941388EE88FF8872
:108E2000088D198DF2E0CF16D10469F480915111AB
:108E3000882349F461E0E114F1040105110509F406
:108E400060E0CE0107C0E114F1040105110521F035
:108E5000CE0161E00E9473888E149F04A006B106C3
:108E600014F4470158010894C11CD11C85E0C816B0
:108E7000D10409F0BBCFC501B401A30192010E9446
:108E8000608E20E830E040E050E00E94C88E2093E1
:108E90009710309398104093991050939A10209304
:108EA0009B1030939C1040939D1050939E10CA01CC
:108EB000B90122E030E040E050E00E94C88E5095B9
:108EC0004095309521953F4F4F4F5F4F2093B11004
:108ED0003093B2104093B3105093B4102093CC1041
:108EE0003093CD104093CE105093CF102093E710C5
:108EF0003093E8104093E9105093EA102093021148
:108F000030930311409304115093051120931D11C8
:108F100030931E1140931F115093201181E08093D4
:108F20009610DF91CF911F910F91FF90EF90DF90FE
:108F3000CF90BF90AF909F908F907F906F905F90F9
:108F40004F903F902F9008952F923F924F925F92B3
:108F50006F927F928F929F92AF92BF92CF92DF9249
:108F6000EF92FF920F931F93CF93DF935C012A013F
:108F70003B0188249924C0E0D0E0222E33240BE169
:108F800010E0C501BE010E94833EC1010C2E02C04B
:108F9000959587950A94E2F780FD23C0C501BE012F
:108FA0000E94833EDC01C09FC001C19F900DD09FF5
:108FB000900D1124E0914F11F0915011E80DF91D21
:108FC0004D915D916D917C911397C080D180E2802D
:108FD000F3804C0D5D1D6E1D7F1D81569F4E20E060
:108FE00013C0C501BE010E94833EFC01C09FC001A9
:108FF000C19F900DD09F900D1124408151816281BD
:10900000738181569F4E21E00E941388C09FF0011A
:10901000C19FF00DD09FF00D1124E156FF4E8689BF
:109020009789A08DB18DC230D10569F4209151117D
:10903000222349F461E00097A105B10509F460E03D
:1090400085ED90E10EC00097A105B10561F0C09FCC
:10905000C001C19F900DD09F900D112481569F4E4D
:1090600061E00E947388219624E030E0820E931E16
:10907000C530D10509F085CFC301B20120E830E049
:1090800040E050E00E94C88E2093971030939810D3
:109090004093991050939A1020939B1030939C10FA
:1090A00040939D1050939E10CA01B90122E030E018
:1090B00040E050E00E94C88E509540953095219533
:1090C0003F4F4F4F5F4F2093B1103093B2104093FA
:1090D000B3105093B4102093CC103093CD10409324
:1090E000CE105093CF102093E7103093E8104093A8
:1090F000E9105093EA10209302113093031140932A
:1091000004115093051120931D1130931E114093AB
:109110001F115093201181E080939610DF91CF9121
:109120001F910F91FF90EF90DF90CF90BF90AF9085
:109130009F908F907F906F905F904F903F902F9077
:1091400008959F92AF92BF92CF92DF92EF92FF92DB
:109150000F931F93CF93DF93982E162FCA01B90157
:109160002FEF3FEF4FEF5FE720939B1030939C1062
:1091700040939D1050939E10E7E0969587957795C4
:109180006795EA95D1F76093971070939810809344
:10919000991090939A1022E030E040E050E00E9455
:1091A000C88ECC24DD247601C21AD30AE40AF50A5B
:1091B000C0E0D0E05BE1A52EB12C012F10E0CA9DEC
:1091C000C001CB9D900DDA9D900D112481569F4ECC
:1091D000FC01C28AD38AE48AF58A98010C2E02C067
:1091E000359527950A94E2F720FF04C0692D0E9467
:1091F000598805C0FC01168A178A108E118E219697
:10920000C530D105E1F681E080932611DF91CF9141
:109210001F910F91FF90EF90DF90CF90BF90AF9094
:109220009F900895853078F4482F50E02BE130E08E
:10923000429FC001439F900D529F900D1124815673
:109240009F4E0E9473880895853078F4482F50E02F
:109250002BE130E0429FC001439F900D529F900D43
:10926000112481569F4E0E94798808950F931F9371
:10927000CF93DF93809196108823D9F180919B1032
:1092800090919C10A0919D10B0919E109C01AD01F9
:10929000215030404040504020939B1030939C1010
:1092A00040939D1050939E100097A105B10519F4AD
:1092B000109296101BC0C0E0D0E00BE110E0C09F00
:1092C000C001C19F900DD09F900D11244091971027
:1092D000509198106091991070919A1081569F4EFC
:1092E0000E947F882196C530D10549F7809196105C
:1092F0002DC080912611882341F110922611C0E0E3
:10930000D0E00BE110E0C09FC001C19F900DD09F45
:10931000900D1124409197105091981060919910E0
:1093200070919A1081569F4E0E94F088882319F4FC
:109330008091261101C081E0809326112196C530CD
:10934000D10509F78091261101C080E0DF91CF910E
:109350001F910F910895CF93DF93CFE9D0E1CE0114
:109360000E94F387CE014B960E94F387CE01C696EA
:109370000E94F38780EF90E10E94F3878BE091E1F8
:109380000E94F387DF91CF91089594EA9093BC00F7
:109390009091BC0097FFFCCF9091B900987F9830D6
:1093A00069F58093BB0084E88093BC008091BC0089
:1093B00087FFFCCF8091B900887F883109F5862F1F
:1093C000972FFC0180E090E050E034E80FC021913D
:1093D0002093BB003093BC002091BC0027FFFCCF42
:1093E0002091B900287F283269F4019684179507E7
:1093F00074F384E98093BC0080E0089581E00895CF
:1094000082E0089583E008951092B90080E280938D
:10941000B800089580915211089510925211089544
:1094200081E0409153115091541120915511309188
:109430005611421753070CF080E0089580915311A4
:109440009091541120915511309156118217930724
:109450006CF4E0915711F0915811E80FF91F019643
:1094600090935411809353118491089580E008954E
:1094700020915711309158118091531190915411AE
:1094800040E0682F592FF901E80FF91FE491019688
:10949000E539B9F7862F952F01964F5F453089F74B
:1094A0006093531150935411089591E09093521189
:1094B00010925411109253118130A1F0813028F094
:1094C000823099F0833031F503C023E731E00FC0DB
:1094D0008EEB91E090935811809357110E94384A77
:1094E00081E009C02EEB31E002C021E639E0309383
:1094F000581120935711E82FF0E0EE0FFF1FEC59A1
:10950000F44E25913491209355113093561180914A
:109510005211089580E00895109252110895DF933A
:10952000CF9300D0CDB7DEB7FC01009769F1623070
:10953000710550F1A081B181660F771F80E090E046
:109540002681378140855185620F731F841F951FC7
:10955000ED91FC91AE014F5F5F4F22E030E0099545
:10956000882391F029813A812115310579F08FEF17
:10957000273F380749F0C90140968730910520F010
:109580008FEF283F380710F020E030E0C9010F903E
:109590000F90CF91DF9108954F925F926F927F92DB
:1095A0008F929F92AF92BF92CF92DF92EF92FF92F3
:1095B0000F931F93DF93CF9300D0CDB7DEB75C013D
:1095C0008B01009709F449C06230710508F445C069
:1095D000DC0116964D905D906D907C9019974E0130
:1095E0000894811C911C000F111F6801EE24FF24B8
:1095F000C40CD51CE61CF71CD501ED91FC91019023
:10960000F081E02DC701B601A40122E030E0099508
:10961000882319F109811A8101151105E1F0C801AA
:10962000409688309105C8F0BFEF083F1B0710F047
:1096300000E010E01A821982D501ED91FC910480BE
:10964000F581E02DC701B601A40122E030E00995C3
:109650000115110541F681E001C080E00F900F90E7
:10966000CF91DF911F910F91FF90EF90DF90CF90FE
:10967000BF90AF909F908F907F906F905F904F9032
:1096800008952F923F924F925F926F927F928F92A6
:109690009F92AF92BF92CF92DF92EF92FF920F9381
:1096A0001F93DF93CF93CDB7DEB72E970FB6F89405
:1096B000DEBF0FBECDBF6C017A876987009709F4C2
:1096C000A4C0DC01ED91FC911197208131813C8790
:1096D0002B87848195819C838B8316968D919D9198
:1096E0000D90BC91A02D8D839E83AF83B887F6012A
:1096F000028D138D428453846484758476946794B8
:10970000579447945E864D86138E128E642E752E66
:10971000EE24FF241E010894211C311C4CC0023091
:10972000110528F02D853E850217130710F002E081
:1097300010E04801880C991CAA24BB248D819E81CD
:10974000AF81B885880E991EAA1EBB1EC501B40143
:10975000A10122E030E0AB85BC85FD01099588239D
:1097600009F453C089819A81009701F5611471044D
:1097700021F4F601138F028F25C0E114F10429F4BE
:109780002FEF3FEF3A83298302C0FA82E982C501B5
:10979000B401A10122E030E0AB81BC81FD0109955B
:1097A000882379F1089461087108780108944108C8
:1097B00051080F5F1F4F4114510409F0B0CF6114DD
:1097C0007104F9F4E985FA85E230F10500F1FA82D5
:1097D000E982BF01660F771F80E090E02D813E8116
:1097E0004F815885620F731F841F951FAE014F5F15
:1097F0005F4F22E030E0AB81BC81FD0109958823F9
:1098000031F4C601B7010E94CC4AEE24FF24C701FF
:109810002E960FB6F894DEBF0FBECDBFCF91DF916D
:109820001F910F91FF90EF90DF90CF90BF90AF907E
:109830009F908F907F906F905F904F903F902F9070
:10984000089580E190E00895CF93DF93EC010097B5
:10985000C1F062307105A8F06250704080E090E085
:109860002889398940E050E00E94608E9B01AC015C
:109870008A899B89AC89BD89280F391F4A1F5B1FC4
:1098800003C020E030E0A901B901CA01DF91CF9106
:109890000895FC0181914AE0282F30E05191C901DF
:1098A0009695982F88279795879535952795822B9C
:1098B000850F415089F70895EF92FF920F931F9300
:1098C000DF93CF93CDB7DEB760970FB6F894DEBFC6
:1098D0000FBECDBF8C0162307105D8F00E94244CC0
:1098E000AE014F5F5F4F20E1DA011D922A95E9F743
:1098F000D801ED91FC91119750962D913C91519783
:109900000680F781E02D01E21CE4EE24FF24099596
:1099100001C080E060960FB6F894DEBF0FBECDBFE9
:10992000CF91DF911F910F91FF90EF9008958F924B
:109930009F92AF92BF92CF92DF92EF92FF920F93DE
:109940001F93DF93CF93CDB7DEB72D970FB6F89463
:10995000DEBF0FBECDBF8C014A015B016901D90199
:10996000ED90FC90119712968D919C911397809693
:1099700013969C938E931297F8018081853E11F087
:10998000882329F4D60114961C921497D0C0F801AC
:1099900083858F3009F04AC0D90114968C911497B1
:1099A000882319F09585891779F08BE2D7011D92EC
:1099B0008A95E9F7F8018585D60114968C93F7010D
:1099C00087A290A6A1A6B2A6D8012C9130E02F7351
:1099D0003070215030404DE050E0249FC001259F61
:1099E000900D349F900D1124DE011196E1E2F6E016
:1099F0002DE001900D922150E1F7DE011196E80E65
:109A0000F91E9C01235F3F4F8F31910508F08FC0F5
:109A10004D91F801E40FF11D4081F70141937F0161
:109A200001968217930709F482C0EECFD7018C917B
:109A3000882341F0C8010E94494CF601948198178F
:109A400009F458C08BE2D7011D928A95E9F7F70116
:109A500087A290A6A1A6B2A6B801D701C80140E08E
:109A6000FC015191CF015032A1F05C93F8012485A3
:109A700023FF0BC09C0121503040F901208121348B
:109A800020F02B3510F4505E5C934F5F11964830F8
:109A900039F7D7018C91853011F485EE8C93F8015C
:109AA0008085803219F1D701A40FB11D8EE28C930D
:109AB000242F2C5F4F5FDB0118968C911897803212
:109AC000A9F0D701A40FB11D8C93F801948594FFE0
:109AD00008C0FB019085913420F09B3510F4805E26
:109AE0008C934F5F6F5F7F4F421729F7F701E40FA9
:109AF000F11D1082D8011B968C911B97F70180A352
:109B00005A968D919C915B9792A381A35C968D91BF
:109B10009D910D90BC91A02D83A394A3A5A3B6A362
:109B200081E0D60115968C93159780E001C081E005
:109B30002D960FB6F894DEBF0FBECDBFCF91DF914B
:109B40001F910F91FF90EF90DF90CF90BF90AF905B
:109B50009F908F9008952F923F924F925F926F92B5
:109B60007F928F929F92AF92BF92CF92DF92EF92AD
:109B7000FF920F931F93DF93CF93CDB7DEB7A097DC
:109B80000FB6F894DEBF0FBECDBF8B01009709F46E
:109B900018C16115710509F414C1DC01ED91FC9146
:109BA00024803580FB0187A090A4A1A4B2A46B01FE
:109BB000DB010D900020E9F71197FA2EF61A8F2D90
:109BC00090E00C966DE070E00E94938EE62ECE0140
:109BD000019660E270E04BE050E00E948E8FC80179
:109BE0006EE270E00E94CD8F0097F9F09C012F5F2C
:109BF0003F4FDC0111968C9111978823B1F0F90148
:109C000001900020E9F73197E21BF30B8E2F80952E
:109C1000F80EBE01675F7F4F4E2FE43008F043E03F
:109C2000CB01B90150E00E94858FCE010196BF2D76
:109C3000B93080F4B6014F2D50E00E94858FF801B5
:109C400080818E3281F581818E3209F48281882370
:109C500049F129C0FC018C2D9D2DDC0188E00D907F
:109C600001928150E1F7D80191962C919197822F22
:109C700090E0203A38F444E0959587954A95E1F7CD
:109C8000805D06C034E0959587953A95E1F78F5948
:109C90008F83822F8F708A3010F4805D01C08F59BE
:109CA000888701C0EE248981853E11F485E089838F
:109CB00085E1FE013C96DF011D928A95E9F7F801E6
:109CC00080A18C8781A192A19C8F8B8F83A194A16D
:109CD000A5A1B6A18D8F9E8FAF8FB8A36E2D70E01A
:109CE00095E0660F771F9A95E1F780E090E0680DA8
:109CF000791D8A1D9B1D6E010894C11CD11CA601F3
:109D000020E230E0F1010995882309F45AC0C60128
:109D10000E94494C482EFE2C8DE0682E712CBFE02D
:109D20005B2E4AC0C6016FEF70E040E250E00E9437
:109D30008E8F8F2D90E00197869DF001879DF00D0D
:109D4000969DF00D1124E00FF11F21E0CF01D60107
:109D5000A20FB11D30813C932F5FD601A20FB11D20
:109D60001C922F5F2B3019F02A3121F402C02EE013
:109D700001C02CE13196DC018C91882311F02F3148
:109D800028F3F982FE1419F48F2D806489835C8690
:109D90004E861D861B8E1C8EC501B401A60120E2D5
:109DA00030E0F101099580E290E0A0E0B0E0880E9B
:109DB000991EAA1EBB1EFA94FF2009F0B3CF81E0C2
:109DC00001C080E0A0960FB6F894DEBF0FBECDBFF5
:109DD000CF91DF911F910F91FF90EF90DF90CF9087
:109DE000BF90AF909F908F907F906F905F904F90BB
:109DF0003F902F9008952F923F924F925F926F92D3
:109E00007F928F929F92AF92BF92CF92DF92EF920A
:109E1000FF920F931F93DF93CF9300D00F92CDB794
:109E2000DEB74C019B01009709F4AEC04115510506
:109E300009F4AAC0FA0101900020E9F7CF01841BC0
:109E4000950B0B966DE070E00E947F8E6F5F6B83C9
:109E5000D9016D907C9011976114710451F4F40153
:109E6000A688B788C08CD18C2288338844885588CE
:109E700006C0222433242101AA24BB2465018601C3
:109E800075011A82A214B304C404D50409F04CC0AD
:109E90006114710409F478C0A114B104C104D1049F
:109EA00079F1C401B3010E948F4A009741F5C401C2
:109EB000B30141E050E00E94414B5C01009709F47E
:109EC00063C0BC016250704080E090E0D4015096C5
:109ED0002D913C91519740E050E00E94608E7B01B3
:109EE0008C01F40182899389A489B589E80EF91E51
:109EF0000A1F1B1FC401B5010E945C4C48C03C01F5
:109F0000C401B3010E94244C5B016C01D401509642
:109F10002D903C90519744245524260E371E481E00
:109F2000591E7B018C011A82D401ED91FC910190A4
:109F3000F081E02DC601B501AE014F5F5F4F21E01A
:109F400030E00995882301F18981853E11F088234D
:109F500079F4BA81BF5FBA83EB81BE17C0F480E2A7
:109F600090E0A0E0B0E0A80EB91ECA1EDB1E8ACFAA
:109F700050E2E52EF12C012D112DEA0CFB1C0C1DDD
:109F80001D1D570168017DCFEE24FF248701B70115
:109F9000C8010F900F900F90CF91DF911F910F91FB
:109FA000FF90EF90DF90CF90BF90AF909F908F90F9
:109FB0007F906F905F904F903F902F9008952F92D9
:109FC0003F924F925F926F927F928F929F92AF9249
:109FD000BF92CF92DF92EF92FF920F931F93DF9386
:109FE000CF93CDB7DEB7AC970FB6F894DEBF0FBEF8
:109FF000CDBF6C01009709F45EC1DC0114968D9110
:10A000009C911597009709F456C116968D919C91D5
:10A010001797009709F44FC16AC1EFEEF1E18CE1A7
:10A02000DF011D928A95E9F7D092F011C092EF11ED
:10A03000D6011996ED90FD900D911C911C9789E029
:10A04000EE0CFF1C001F111F8A95D1F7EA8EFB8EC4
:10A050000C8F1D8FC801B701655F7F4F8F4F9F4FDA
:10A06000ED91FC91AE014F5F5F4F29E130E0099522
:10A07000882309F41CC129803A804C815D81BB8111
:10A08000BAA32E81EF81F885FCA3EBA389859A857D
:10A090006C857D85EE88FF88088D198DEE8EFF8E8C
:10A0A00008A319A3E114F1040105110551F4009767
:10A0B00009F4FDC07C0100E010E0EE8EFF8E08A3E5
:10A0C00019A36115710509F4F2C0CA01A0E0B0E05E
:10A0D0008DA39EA3AFA3B8A780E090E030E040E05E
:10A0E00050E00E94608E69A77AA78BA79CA7EE8C90
:10A0F000FF8C08A119A18DA19EA1AFA1B8A5E81A56
:10A10000F90A0A0B1B0B89A59AA5ABA5BCA5E81AF1
:10A11000F90A0A0B1B0BC10101972BA13CA1F5E029
:10A12000220F331FFA95E1F7820F931FB1010E94AE
:10A130007F8E80E090E0E61AF70A080B190B9AA1CF
:10A14000292F30E040E050E0C801B7010E94A68E00
:10A1500029013A01253FAFE03A07A0E04A07A0E015
:10A160005A0708F4A4C0253FBFEF3B07B0E04B07F8
:10A17000B0E05B0720F486E0F601808704C08BE046
:10A18000D60118968C9388E1E1EFF1E1DF011D9291
:10A190008A95E9F74101AA24BB246E8D7F8D88A1A1
:10A1A00099A1A50194010E94608E6093F1117093B2
:10A1B000F2118093F3119093F411C501B4012DA114
:10A1C0003EA14FA158A50E94608E7B018C018A8D13
:10A1D0009B8DAC8DBD8DE80EF91E0A1F1B1FE092F2
:10A1E000F511F092F6110093F7111093F811A301F5
:10A1F00092012E5F3F4F4F4F5F4FD60118968C91C3
:10A200001897863029F462E070E080E090E004C0A6
:10A2100064E070E080E090E00E94608E6093F9114D
:10A220007093FA118093FB119093FC113092FE1100
:10A230002092FD11BAA12B2F30E0229DC001239D59
:10A24000900D329D900D1124909300128093FF1178
:10A2500069A57AA58BA59CA5A50194010E94608E95
:10A260006E0D7F1D801F911F609305127093061263
:10A270008093071290930812EBA1FCA19F0140E08C
:10A2800050E0E5E0220F331F441F551FEA95D1F738
:10A29000260F371F481F591F2093011230930212B7
:10A2A00040930312509304122FEE31E106C0109236
:10A2B000F0111092EF1120E030E0C901AC960FB61A
:10A2C000F894DEBF0FBECDBFCF91DF911F910F91EC
:10A2D000FF90EF90DF90CF90BF90AF909F908F90C6
:10A2E0007F906F905F904F903F902F900895809156
:10A2F000EF119091F0110097F1F68FCE009719F0C1
:10A30000FC01118210820895CF93DF93FB01009727
:10A3100029F1309719F120A124FD20C025C0CDEBF3
:10A32000D1E1DF012BE20D9009922150E1F79093EA
:10A33000BC118093BB111092E8111092E911109298
:10A34000EA111092EB1181A192A19093ED118093EB
:10A35000EC111092EE112BEB31E102C020E030E065
:10A36000C901DF91CF9108952091BB113091BC11AB
:10A370002115310599F7D3CFCF93DF93EC010097E7
:10A3800059F08BA9813031F4FE0181919191BF0187
:10A390000E94AB4D19821882DF91CF9108952F92C0
:10A3A0003F924F925F926F927F928F929F92AF9265
:10A3B000BF92CF92DF92EF92FF920F931F93DF93A2
:10A3C000CF9300D000D000D0CDB7DEB79E838D8371
:10A3D0007C836B833A01009709F4D4C06115710541
:10A3E00009F4D0C04115510509F4CCC0DC019D969B
:10A3F000CD90DD90ED90FC90D09795962D913D916C
:10A400004D915C919897C301A0E0B0E08C0D9D1D2B
:10A41000AE1DBF1D281739074A075B0728F439010D
:10A420006C187D0809F4ABC0AD81BE81ED91FC9143
:10A430001197208931893A832983D1960D911C91F6
:10A44000D2970115110579F593960D911C9194976A
:10A450000115110539F4C114D104E104F10409F422
:10A460008EC090C0C114D104E104F104E1F04601B2
:10A47000570189819A811C01442455240FC0AD8164
:10A48000BE818D919C91B8010E948F4A8C010097EA
:10A4900009F478C082189308A408B50882149304BC
:10A4A000A404B50460F789809A8008948108910813
:10A4B0008C209D207301ED81FE8120803180C101BF
:10A4C000B8010E94244C9B01AC01C980DA80C818F5
:10A4D000D908EC14FD0408F46701D101ED91FC9159
:10A4E000B40180E090E0620F731F841F951F0190FC
:10A4F000F081E02D4B815C8196010995882349F11B
:10A50000EC18FD08960140E050E0ED81FE8185A544
:10A5100096A5A7A5B0A9820F931FA41FB51F85A755
:10A5200096A7A7A7B0ABC601880D991D29813A81CE
:10A5300082179307A0F080819181B8010E948F4A11
:10A540008C01009751F4AD81BE81D2961C921E926F
:10A55000D19793012E193F0917C088249924ED81C2
:10A56000FE8112AB01ABE114F10439F02B813C8187
:10A570002C0D3D1D3C832B839ECF930105C020E015
:10A5800030E002C02FEF3FEFC90126960FB6F894D6
:10A59000DEBF0FBECDBFCF91DF911F910F91FF9016
:10A5A000EF90DF90CF90BF90AF909F908F907F9073
:10A5B0006F905F904F903F902F9008952F923F9211
:10A5C0004F925F926F927F928F929F92AF92BF92C3
:10A5D000CF92DF92EF92FF920F931F93DF93CF936F
:10A5E00000D000D000D0CDB7DEB79E838D831B0195
:10A5F0005C834B83009709F409C16115710509F467
:10A6000005C14115510509F401C1DC019D968D90EC
:10A610009D90AD90BC90D097FC0185A196A1A7A17B
:10A62000B0A588159905AA05BB0508F4EFC080817F
:10A630009181DC0150960D90BC91A02DBA83A98325
:10A6400001A912A90115110509F052C003A114A115
:10A6500001151105A1F481149104A104B10409F0BC
:10A66000D5C060E070E041E050E00E94414B8C01B9
:10A67000ED81FE8194A383A3009709F4C7C0AD8147
:10A68000BE819D96CD90DD90ED90FC90D097C11449
:10A69000D104E104F10461F121C0C418D508E60831
:10A6A000F708ED81FE8180819181B8010E948F4A77
:10A6B000009791F4C114D104E104F10409F0A6C09B
:10A6C000AD81BE818D919C91B80141E050E00E9426
:10A6D000414B009709F49AC08C0105C0E981FA81C9
:10A6E0002F0166247724C414D504E604F704A8F6E1
:10A6F000C980DA800894C108D108C820D920AB806D
:10A70000BC80AD81BE818D909C90C401B8010E9437
:10A71000244C9B01AC01E980FA80EC18FD08AE14D2
:10A72000BF0408F47501D401ED91FC91B60180E0FD
:10A7300090E0620F731F841F951F0480F581E02D48
:10A74000A10197010995882309F444C0AE18BF08F8
:10A75000970140E050E0ED81FE8185A596A5A7A573
:10A76000B0A9820F931FA41FB51F85A796A7A7A7FF
:10A77000B0ABC7018C0D9D1D29813A8182179307CB
:10A78000E8F080819181B8010E948F4A009799F486
:10A79000A114B10459F0AD81BE818D919C91B80195
:10A7A00041E050E00E94414B009729F4ED81FE8189
:10A7B00012AA11AA0FC08C01CC24DD24AD81BE8168
:10A7C000D2961C930E93D197A114B10419F02E0CBC
:10A7D0003F1C97CFED81FE8185A596A5A7A5B0A9C1
:10A7E00025A136A147A150A5281739074A075B07BD
:10A7F00040F421E023ABED81FE8185A396A3A7A3BE
:10A80000B0A72B813C812A193B0902C02FEF3FEFF3
:10A81000C90126960FB6F894DEBF0FBECDBFCF910B
:10A82000DF911F910F91FF90EF90DF90CF90BF903D
:10A83000AF909F908F907F906F905F904F903F90E0
:10A840002F900895CF93DF93DB01009791F110973C
:10A8500081F190962C91909724FF2BC02091591153
:10A8600030915A112115310551F020918A11309102
:10A870008B1121153105E9F4EAE8F1E102C0E9E5BF
:10A88000F1E19F012E5F3F4FBD014BE2EB010990CB
:10A89000BE01E90109929E014150C1F79183808375
:10A8A00091968D919C91929796A785A710AA17A62D
:10A8B00002C0E0E0F0E0CF01DF91CF910895009772
:10A8C00019F0FC011182108208952F923F924F924D
:10A8D0005F926F927F928F929F92AF92BF92CF9230
:10A8E000DF92EF92FF920F931F93DF93CF93CDB739
:10A8F000DEB7A6970FB6F894DEBF0FBECDBF5C01E2
:10A90000009709F499C06115710509F495C0DC013F
:10A910006D907C901197F301208831889D964D9021
:10A920005C909E979F968D909C90D09782149304F4
:10A9300068F093968D919C9194979E969C938E939C
:10A940009D97D0961C921E929F9776C0FE013196DD
:10A9500086E0DF011D928A95E9F78BE2DB011D920B
:10A960008A95E9F77A8369834114510409F055C047
:10A97000F3012288338886899789281A390A4DC0BD
:10A980006101C818D908740100E010E041145104B5
:10A9900041F4D30156966D917D918D919C9159977B
:10A9A00004C0C301B2010E94244C6E0D7F1D801FA4
:10A9B000911F1C821B82D301ED91FC910280F381D7
:10A9C000E02DAE01495F5F4F20E230E08601A7E94C
:10A9D000EA2EACE4FA2E6E010894C11CD11C099534
:10A9E000882351F18B819C81880E991E82149304D7
:10A9F000A0F0C301B2010E948F4A2C01009759F4C4
:10AA00008E81882371F4F50183A194A196A785A76F
:10AA100010AA17A611C0882499248E81882309F4CE
:10AA2000AFCFD5019E965C924E929D97D0969C9208
:10AA30008E929F978E8101C080E0A6960FB6F89403
:10AA4000DEBF0FBECDBFCF91DF911F910F91FF9061
:10AA5000EF90DF90CF90BF90AF909F908F907F90BE
:10AA60006F905F904F903F902F9008958F929F929C
:10AA7000AF92BF92CF92DF92EF92FF920F931F930C
:10AA8000CF93DF934C01EB018A01009709F464C076
:10AA9000209709F461C08881882309F45DC04115BD
:10AAA000510509F459C08F3209F421968BE2D8017F
:10AAB0001D928A95E9F780E1F80180A301C0E501C4
:10AAC0008881882309F44AC0C401B8010E94225435
:10AAD0007C01009709F440C0CE016FE270E00E9453
:10AAE000958F009739F0A82FAC1B5C010894A11C2E
:10AAF000B11C29C0DE010D900020E9F71197AC1BB5
:10AB00005E01AA0EB11C1FC0F80101900020E9F7F8
:10AB10003197E01BF10BEC15FD05B9F4CE01B8013E
:10AB2000A6010E94B08F009781F4D70111961C9264
:10AB30001E92CC0DDD1D8881882381F0F80180A153
:10AB400084FDBDCF09C0CA2EDD24C701B8010E9413
:10AB500065548823C9F610C080E001C081E0DF9110
:10AB6000CF911F910F91FF90EF90DF90CF90BF900A
:10AB7000AF909F908F900895D70111961C921E92CE
:10AB80009FCFFC01009741F083A194A196A785A7D0
:10AB900010AA17A681E0089580E00895AF92BF92B1
:10ABA000CF92DF92EF92FF920F931F93CF93DF9399
:10ABB0008C017B01EA01009709F446C0611571051B
:10ABC00009F442C0DB018C918823F1F12097E1F177
:10ABD000C801BE010E946554882371F0C701BE01FF
:10ABE0000E94A08F0097A1F7F80183A194A196A7D6
:10ABF00085A710AA17A628C0D801CD90DC905E01C9
:10AC0000EC2FFB2D8BE2DF011D928A95E9F7CE0137
:10AC1000B7014FE150E00E94BE8FB8016D5D7F4FDC
:10AC2000C601AE010E94FB4E6FA378A789A79AA721
:10AC3000611571058105910539F0C601BE010E94BB
:10AC4000AB4D91E0882309F490E0892FDF91CF91FB
:10AC50001F910F91FF90EF90DF90CF90BF90AF903A
:10AC600008957F928F929F92AF92BF92CF92DF9280
:10AC7000EF92FF920F931F93DF93CF93CDB7DEB781
:10AC80002C970FB6F894DEBF0FBECDBF6C015B01F1
:10AC9000009709F453C06115710509F44FC0DB0139
:10ACA0009796ED90FD900D911C919A97E114F10407
:10ACB0000105110509F442C04E010894811C911C44
:10ACC000B5EE7B2ED601ED91FC910190F081E02D47
:10ACD000C801B701A4012CE030E00995882371F187
:10ACE0007982D601ED91FC910480F581E02DC801B7
:10ACF000B701A4012CE030E009958823F9F08C8598
:10AD00008F3049F480E290E0A0E0B0E0E80EF91E58
:10AD10000A1F1B1FD7CFD50191966D917C919297F9
:10AD20006115710541F0C6010E94CC4A91E088236B
:10AD300019F490E001C091E0892F01C080E02C96C9
:10AD40000FB6F894DEBF0FBECDBFCF91DF911F913C
:10AD50000F91FF90EF90DF90CF90BF90AF909F90BA
:10AD60008F907F9008958F929F92AF92BF92CF92D3
:10AD7000DF92EF92FF920F93DF93CF93CDB7DEB7C1
:10AD800060970FB6F894DEBF0FBECDBF7C016B019C
:10AD90005A014901009709F4A3C06115710509F42E
:10ADA0009FC004300CF09CC007FD1DC0602F7727AA
:10ADB00067FD709584E0660F771F8A95E1F762540E
:10ADC0007E4F882777FD8095982FAE014F5F5F4FAC
:10ADD00020E130E0F7010995882309F481C08D81D5
:10ADE000882309F47DC080911312882309F078C06C
:10ADF000EBE0F2E181E1DF011D928A95E9F7F09243
:10AE00000C12E0920B12D0920E12C0920D12B09260
:10AE10001012A0920F12909212128092111207FD3E
:10AE20005AC08D81809313128A8590E0A0E0B0E033
:10AE3000BA2FA92F982F88272B8530E040E050E0CB
:10AE4000A90133272227822B932BA42BB52B2985ED
:10AE500030E040E050E0822B932BA42BB52B2C85C7
:10AE600030E040E050E0522F442733272227822B46
:10AE7000932BA42BB52B81879287A387B4878E85CC
:10AE800090E0A0E0B0E0BA2FA92F982F88272F8557
:10AE900030E040E050E0A90133272227822B932B9A
:10AEA000A42BB52B2D8530E040E050E0822B932B76
:10AEB000A42BB52B288930E040E050E0522F4427E6
:10AEC00033272227822B932BA42BB52B858796879C
:10AED000A787B08B03C08FEF809313129F0102C02E
:10AEE00020E030E0C90160960FB6F894DEBF0FBED7
:10AEF000CDBFCF91DF910F91FF90EF90DF90CF907A
:10AF0000BF90AF909F908F900895009721F0FC0123
:10AF1000108681E0089580E008958EBD0DB407FE8F
:10AF2000FDCF8DB58F778DBD08958FEF8EBD0DB49C
:10AF300007FEFDCF8DB58F778DBD8EB508951F931C
:10AF4000DF93CF9300D000D0CDB7DEB7182F4C835E
:10AF50005B836A8379830E949557812F80640E9466
:10AF60008D577981872F0E948D576A81862F0E9485
:10AF70008D575B81852F0E948D574C81842F0E94B5
:10AF80008D57112319F0183041F405C085E90E944E
:10AF90008D571AE004C087E8FACF8FEFF8CF0E94F0
:10AFA00095578F3F11F41150D1F70F900F900F90DC
:10AFB0000F90CF91DF911F910895DF93CF9300D031
:10AFC0000F92CDB7DEB780913414909135149A83E7
:10AFD00089838B81807F86608B83CE0101960E945E
:10AFE0004E2591E089270F900F900F90CF91DF9120
:10AFF0000895DF93CF9300D00F92CDB7DEB7809145
:10B000003414909135149A8389838B81807F856075
:10B010008B83CE0101960E944E250F900F900F90CA
:10B02000CF91DF91089580911C128823A1F4609143
:10B030001D1270911E1280911F129091201241E2F8
:10B0400052E120E032E00E94005A882331F081E092
:10B0500080931C12089581E0089580E008952F9256
:10B060003F924F925F926F927F928F929F92AF9298
:10B07000BF92CF92DF92EF92FF920F931F93CF93E5
:10B08000DF931B012C018A01790172C09FEFA92E69
:10B0900091E0B92EA220B320C501A0E0B0E04201AA
:10B0A0003101681A790A8A0A9B0AC0E0D2E0CA19FB
:10B0B000DB09EC16FD0608F4E70180911D12909162
:10B0C0001E12A0911F12B0912012681679068A06EE
:10B0D0009B06D9F10E941358882309F44FC0289881
:10B0E00081E1B401A3010E949F57882311F0289A9F
:10B0F00045C00E9495578E3FE1F781E2C82E82E15C
:10B10000D82E0E949557F60181936F01F1E2CF1678
:10B11000F4E1DF06B1F760921D1270921E12809268
:10B120001F129092201295012F5D3D4EC801B9016A
:10B13000AE010E94858F0C0F1D1F0E9495570E9423
:10B140009557289A0E9495570AC095012F5D3D4E4C
:10B15000C801B901AE010E94858F0C0F1D1FEC1AAA
:10B16000FD0ACE01A0E0B0E0280E391E4A1E5B1E8B
:10B17000E114F10409F08ACF81E001C080E0DF91A1
:10B18000CF911F910F91FF90EF90DF90CF90BF90E4
:10B19000AF909F908F907F906F905F904F903F9077
:10B1A0002F9008952F923F924F925F926F927F92CD
:10B1B0008F929F92AF92BF92CF92DF92EF92FF92C7
:10B1C0000F931F93DF93CF9300D000D0CDB7DEB79E
:10B1D0004B015C013A013C832B8341155105C1F1C0
:10B1E00021153105A9F10217130790F1E114F104BB
:10B1F00079F1309521953F4F3A8329832B813C810A
:10B20000021B130B190144245524C501B401A301E9
:10B210002B813C810E942F588823D1F0C301B501B6
:10B22000A4019601F70109958823A1F089819A81EB
:10B23000080F191F8B819C81800F911FEB81FC816E
:10B240008E179F0738F0820C931CA41CB51CDDCF11
:10B2500080E001C081E00F900F900F900F90CF9190
:10B26000DF911F910F91FF90EF90DF90CF90BF90F3
:10B27000AF909F908F907F906F905F904F903F9096
:10B280002F9008950F931F93DF93CF9300D000D09A
:10B2900000D0CDB7DEB780913414909135149A83E5
:10B2A00089838B81807F86608B83CE01019660E0ED
:10B2B0000E94472580913414909135149D838C838E
:10B2C0008E81807F85608E83CE01049660E00E942F
:10B2D0004725229A219A209A2398289A83E58CBDA3
:10B2E0008DB58E7F8DBD109221140E94DD5788236D
:10B2F00009F479C000E00E9495570F5F0A30D9F732
:10B30000289800E010E080E040E050E0BA010E94A0
:10B310009F57813041F081E00F3F180709F43FC08B
:10B320000F5F1F4FF0CF87E340E050E0BA010E946B
:10B330009F5789E240E050E0BA010E949F5782FD8A
:10B3400005C08091211481608093211400E010E0F9
:10B350008091211490E083709070009741F087E312
:10B3600040E050E0BA010E949F5789E201C081E0AD
:10B3700040E050E0BA010E949F5780FF07C08FE76E
:10B380000F3F180761F00F5F1F4FE2CF80E140E0F1
:10B3900052E060E070E00E949F57882311F0289AE5
:10B3A00022C0289A8CB58C7F8CBD8DB581608DBDF7
:10B3B0008FEF9FEFAFEFBFEF80931D1290931E12A0
:10B3C000A0931F12B093201281E080931C1260E0C2
:10B3D00070E0CB0141E252E120E032E00E942F58C0
:10B3E00091E0882309F490E0892F26960FB6F8940F
:10B3F000DEBF0FBECDBFCF91DF911F910F9108959A
:10B400002F923F924F925F926F927F928F929F9274
:10B41000AF92BF92CF92DF92EF92FF920F931F9362
:10B42000CF93DF932B013C014A0189010E94F95718
:10B43000882309F48EC095C04FEFA42E41E0B42EAE
:10B44000A420B520C501A0E0B0E073016201C81AD4
:10B45000D90AEA0AFB0AE101CA19DB090C171D0720
:10B4600008F4E80180911D1290911E12A0911F1204
:10B47000B0912012C816D906EA06FB06F9F00E9420
:10B480001358882309F46DC0A114B10421F422E0FB
:10B49000C030D20759F0C701B60141E252E120E0C5
:10B4A00032E00E942F58882309F45BC0C0921D121D
:10B4B000D0921E12E0921F12F092201231E28316F7
:10B4C00032E1930671F095012F5D3D4EC901B40143
:10B4D000AE010E94858F10921C120C171D0709F4F3
:10B4E00042C0289888E1B701A6010E949F5788238F
:10B4F00011F0289A36C08EEF0E948D5731E2C32E8C
:10B5000032E1D32EF60181916F010E948D57F1E255
:10B51000CF16F4E1DF06B1F78FEF0E948D578FEF62
:10B520000E948D570E9495578F3FE1F70E949557D3
:10B53000289A8C0E9D1ECE01A0E0B0E0480E591E48
:10B540006A1E7B1E0C1B1D0BAA24A394A0921C1226
:10B5500003C0212C22E0322E0115110509F06CCF19
:10B5600002C080E001C081E0DF91CF911F910F9177
:10B57000FF90EF90DF90CF90BF90AF909F908F9013
:10B580007F906F905F904F903F902F9008954F92D3
:10B590005F926F927F928F929F92AF92BF92CF9263
:10B5A000DF92EF92FF920F931F93CF93DF934B01A4
:10B5B0005C013A01690128014115510571F101153C
:10B5C000110559F111E021153105C1F010E016C047
:10B5D000112319F4CC16DD0600F1C501B401A30155
:10B5E0009E010E94005A8823C1F0CE01A0E0B0E085
:10B5F000880E991EAA1EBB1ECC1ADD0A112319F44F
:10B60000C114D10461F0C301B501A4019701F20195
:10B610000995EC010097E1F602C080E001C081E0ED
:10B62000DF91CF911F910F91FF90EF90DF90CF901E
:10B63000BF90AF909F908F907F906F905F904F9052
:10B640000895883098F490B321E030E0082E02C0CD
:10B65000220F331F0A94E2F72095922390BB91B3F7
:10B66000922391BB90917B00977F17C08850909157
:10B67000070121E030E0082E02C0220F331F0A9498
:10B68000E2F720959223909307019091080192236D
:10B690009093080190917B00986090937B00805C70
:10B6A00080937C0080917A008F6880937A0008955F
:10B6B00090917A0096FD23C02FB7F89470932314CD
:10B6C000609322145093251440932414FA0110829D
:10B6D000883020F490917B00977F04C0885090912F
:10B6E0007B00986090937B00805C80937C008091CD
:10B6F0007A00806480937A002FBF81E0089580E013
:10B7000008951F920F920FB60F920BB60F9211244D
:10B710002F933F938F939F93EF93FF9380917800A4
:10B7200090917900E0912214F0912314392F20E0B8
:10B7300090E0822B932B91838083E0912414F091ED
:10B74000251481E08083FF91EF919F918F913F912C
:10B750002F910F900BBE0F900FBE0F901F9018955A
:10B760002FEF3FEFFC01318320830895FC0181E03E
:10B77000208131819FEF2F3F390709F080E0089544
:10B78000DC01ED91FC911197318181E090E002C0E4
:10B79000880F991F6A95E2F7282F209523234423C9
:10B7A00009F480E0822B81830895DC01ED91FC9106
:10B7B0001197808190E002C0959587956A95E2F790
:10B7C00081700895DC01ED91FC911197328181E047
:10B7D00090E002C0880F991F6A95E2F7282F209504
:10B7E0002323442309F480E0822B8283089580E29E
:10B7F00090E0909327148093261483E290E0909336
:10B8000029148093281486E290E090932B1480935F
:10B810002A1489E290E090932D1480932C148CE2EA
:10B8200090E090932F1480932E148FE290E09093E9
:10B8300031148093301482E390E09093331480931A
:10B84000321480E091E0909335148093341483E0B7
:10B8500091E0909337148093361486E091E09093B2
:10B8600039148093381489E091E090933B148093CD
:10B870003A14089521E0FC0125830895029661E0C1
:10B880000E94981D0895029660E00E94981D0895F8
:10B89000CF93DF93EC018D818823A1F0888199817A
:10B8A0000E94B05F2E813F812817390744F424E0BD
:10B8B0008030920721F0CE010E943E5C03C0CE0191
:10B8C0000E94435CDF91CF910895FC0115820E9494
:10B8D000435C08950F931F93CF93DF93EC0188850A
:10B8E0009985019662E30E94E55C8E831F828E013A
:10B8F0000E5F1F4FC80160E00E94981DC80161E003
:10B900000E9447258885998561E00E94E55C813029
:10B9100011F48D8304C01D82CE010E94435CDF912F
:10B92000CF911F910F9108950F931F93DF93CF93A2
:10B9300000D00F92CDB7DEB709831A832B83FC01A9
:10B9400061937193DE01119623E00D9001922150D5
:10B95000E1F7FC01518740870E946A5C0F900F90CD
:10B960000F90CF91DF911F910F910895DF93CF93A7
:10B9700000D0CDB7DEB7CE01019660E070E042E0C6
:10B9800050E00E94D88F2A8184E6289FC0011124AC
:10B990003981830F911D31E0863F930789F0225052
:10B9A0002D3F10F00E94042982E0898385E08A837C
:10B9B000CE01019660E070E042E050E00E94EE8F20
:10B9C0000F900F90CF91DF9108951F93DF93CF9346
:10B9D0000F92CDB7DEB79C01162FCE010196B901AB
:10B9E00041E050E00E94D88F89818F3F09F419838C
:10B9F00089810F90CF91DF911F9108950F931F932D
:10BA0000DF93CF9300D0CDB7DEB79C018B01CE0181
:10BA10000196B90142E050E00E94D88F89819A8155
:10BA20002FEF8F3F920711F41A83098389819A813E
:10BA30000F900F90CF91DF911F910F910895EF928A
:10BA4000FF920F931F93142FE52EF62E072F0E94BF
:10BA5000E88F9B01AC012F3F8FEF38078FEF48072E
:10BA60008FEF580721F4212F3E2D4F2D502FB90174
:10BA7000CA011F910F91FF90EF900895EF92FF92EE
:10BA80000F931F93DF93CF9300D0CDB7DEB79C0108
:10BA9000F42E052F162FE72ECE010196B90142E0B4
:10BAA00050E00E94D88F69816F3F19F48A818F3FDF
:10BAB000E9F070E080E090E00E94E6197B018C01E3
:10BAC0006A8170E080E090E00E94E61920E030E0BA
:10BAD00040E85BE30E94DA179B01AC01C801B701A3
:10BAE0000E947C17F62E072F182FE92E6F2D702F2E
:10BAF000812F9E2D0F900F90CF91DF911F910F916D
:10BB0000FF90EF900895CF92DF92EF92FF920F9304
:10BB10001F93DF93CF9300D0CDB7DEB76C017A01CE
:10BB20008B01CB01BA010E940616698370E0882759
:10BB300077FD8095982F0E9434199B01AC01C801B4
:10BB4000B7010E94A91720E030E040E853E40E94CA
:10BB5000DA170E9494196A83CE010196B60142E079
:10BB600050E00E94EE8F0F900F90CF91DF911F91C8
:10BB70000F91FF90EF90DF90CF9008952F923F921A
:10BB80004F925F926F927F928F929F92AF92BF92ED
:10BB9000CF92DF92EF92FF920F931F93DF93CF9399
:10BBA000CDB7DEB764970FB6F894DEBF0FBECDBF3A
:10BBB0008C01FC01158E148E178E168EEB5BFF4FD9
:10BBC0001082FC01EA5BFF4F1082FC01E85BFF4F33
:10BBD00011821082FC01E95BFF4F10826E01089414
:10BBE000C11CD11CC6010E94DA8CD801A65BBF4FD4
:10BBF000F6018AE001900D928150E1F79BE0C92E99
:10BC0000D12CCC0EDD1EC6010E94DA8CD801AC5AB4
:10BC1000BF4FF6018AE001900D928150E1F7F801E3
:10BC2000E25AFF4F1082F80110A281A192A140E0D8
:10BC300050E060EE70E40E943E5D6B017C01F80113
:10BC400081A192A1029646E656E666EA7EE30E944C
:10BC50003E5D4B015C01F80181A192A1049640E098
:10BC600050E060E172E40E943E5D2B013C0183E202
:10BC7000282E312C200E311EC1010E948A85C70159
:10BC8000B60120E030E0A9010E94D418882381F594
:10BC9000C501B40120E030E0A9010E94D418882336
:10BCA00039F5C301B20120E030E0A9010E94D418A7
:10BCB0008823F1F40F2EF0E04F2EF0E05F2EF0E13C
:10BCC0006F2EF2E47F2EF02D0F2EF6E68F2EF6E685
:10BCD0009F2EF6EAAF2EFEE3BF2EF02D0F2EF0E0E2
:10BCE000CF2EF0E0DF2EF0EEEF2EF0E4FF2EF02D61
:10BCF000F801C3A2D4A2E5A2F6A287A290A6A1A6AB
:10BD0000B2A643A654A665A676A6C10160E070E07F
:10BD10000E94AE86C801049640E251EA67E070E0F6
:10BD20000E94DE8CF801408D518D628D738DC801AB
:10BD30000E960E94DE8C64960FB6F894DEBF0FBE9E
:10BD4000CDBFCF91DF911F910F91FF90EF90DF90CA
:10BD5000CF90BF90AF909F908F907F906F905F90AB
:10BD60004F903F902F9008958F929F92AF92BF92E5
:10BD7000CF92EF92FF920F931F93CF93DF93EC013B
:10BD800048015901798368835B834A8304960E9442
:10BD9000DA8CCE010E960E94DA8C888E998EAA8E4D
:10BDA000BB8EFAA2E9A2CE0183960E949F85CE01A6
:10BDB000865B9F4F0E94DA8CCE018C5A9F4F0E9467
:10BDC000DA8CFE01E15AFF4FC082CE010E94BE5DB7
:10BDD000DF91CF911F910F91FF90EF90CF90BF9087
:10BDE000AF909F908F900895AF92BF92CF92DF92C5
:10BDF000EF92FF920F931F93DF93CF93CDB7DEB7F0
:10BE00006E970FB6F894DEBF0FBECDBF8C01E62E45
:10BE1000F72E85E0E81681E0F80624F054E0E52EE0
:10BE200051E0F52EF80110A2E15AFF4F80818823DE
:10BE300009F45EC0F801848D958D978F868FE25A44
:10BE4000FF4F1082F801E95BFF4F1082FFE1EF1610
:10BE5000F10460F1F801868D978D0A9644E5C42EB1
:10BE6000D12CC00ED11E8E159F0540F4C60140E0B6
:10BE70005AE562E672E00E94DE8C0EC05E01089414
:10BE8000A11CB11CC5010E94DA8CD601F5018AE023
:10BE900001900D928150E1F7C801865B9F4F40E011
:10BEA00053EA61EE71E10E94DE8C22C03BE0C32EBA
:10BEB000D12CCC0EDD1EC6010E94DA8CD801A65B07
:10BEC000BF4FF6018AE001900D928150E1F725E124
:10BED000C22ED12CCC0EDD1EC6010E94DA8CD801F8
:10BEE000AC5ABF4FF6018AE001900D928150E1F704
:10BEF000C8018396B7010E94AE866E960FB6F8947D
:10BF0000DEBF0FBECDBFCF91DF911F910F91FF908C
:10BF1000EF90DF90CF90BF90AF900895FC0180A18B
:10BF20008823B1F4448D558DDF01A05CBF4F8D9106
:10BF30009C9111979C01225030404217530740F0CA
:10BF4000248D358D02968217930710F081E080A32F
:10BF500080A10895FC01E05CFF4F808191810895EC
:10BF6000FC01248D358DC901089583960E94C386F6
:10BF7000089583960E94C786089583960E94D0866E
:10BF80000895CF93DF93EC01FC01E05CFF4F8081CB
:10BF90009181181619065CF4CE010E948E5F8823E9
:10BFA00031F4CB5BDF4F888191E0892701C080E0CD
:10BFB000DF91CF910895FC01E05CFF4F208131813A
:10BFC000DC01ED91FC911197828193818217930797
:10BFD00018F4281B390B04C0AC01421B530B9A0107
:10BFE000C9010895DC0112968D919C911397DC0193
:10BFF000ED91FC910190F081E02D09950895CF938A
:10C00000DF93EC01FC01EB5BFF4F81E08083CE010D
:10C0100060E00E94F25FC85BDF4F6881798183E452
:10C020009BE00E94D336DF91CF9108950F931F9329
:10C03000CF93DF93EC018C01025F1F4FC8010E9478
:10C04000FB8C882309F4A0C0488D598D6A8D7B8DA7
:10C05000C8010E94DE8C88819981DC01ED91FC9100
:10C060000280F381E02D0995009741F097FD17C0FC
:10C0700083309105A4F482E090E025C0FE01EA5BE4
:10C08000FF4F1082E881F981828193819D8F8C8F8F
:10C090008C8D9D8DB1E08D329B07C0F425C0FE01D3
:10C0A000EA5BFF4F80818F5F8083863050F0FE0116
:10C0B000E85BFF4F81E090E091838083CE010E9496
:10C0C000FF5F83E090E09D8F8C8FBAC0FE01E95B3B
:10C0D000FF4F80818F5F8083863030F0FE01E85B08
:10C0E000FF4F82E090E04AC08E01025A1F4FF801D4
:10C0F0008081882321F5CE018C5A9F4F0E94FB8CB2
:10C100008823E9F0D8018C918823C9F42C8D3D8DCA
:10C110008E8D9F8D0A962817390770F4FE01E95B12
:10C12000FF4F80818F5F8083863048F0FE01E85B9F
:10C13000FF4F84E090E022C081E0F8018083CE01CF
:10C14000865B9F4F0E94FB8C8823F1F02C8D3D8DE8
:10C15000FE01E05CFF4F808191814E9728173907DF
:10C1600098F4FE01E95BFF4F80818F5F808386300A
:10C1700058F0FE01E85BFF4F85E090E091838083FB
:10C18000CE010E94FF5F5CC0FE01EB5BFF4F808130
:10C19000882309F055C08E010C5F1F4FC8010E9413
:10C1A000FB8C882309F44CC0C80140E251EA67E0E7
:10C1B00070E00E94DE8C2C8D3D8DFE01E05CFF4F17
:10C1C00080819181821B930BFE01EC5BFF4F2081EC
:10C1D000222349F08F3091055CF41082CE018396C2
:10C1E0000E94698505C08A31910514F081E0808341
:10C1F000FE01EC5BFF4F8081882319F0CE016FEFC9
:10C200001DC06C8D7D8DCE0183960E94B485BC01CE
:10C2100097FD05C08F3F910509F024F405C060E04B
:10C2200070E002C06FEF70E0FE01E05CFF4F8081C4
:10C230009181009711F460E070E0CE010E94F25FFE
:10C24000DF91CF911F910F910895FC01EB5BFF4FA0
:10C2500080810895DF93CF93CDB7DEB729970FB6CE
:10C26000F894DEBF0FBECDBF80912A1490912B149D
:10C270009A8389838B81807F87608B83CE0101962F
:10C2800060E00E94981D80912A1490912B149D8348
:10C290008C838E81807F87608E83CE01049660E0E0
:10C2A0000E94472580912A1490912B1498878F83A0
:10C2B0008985807F87608987CE0107960E944E25F9
:10C2C000882391F080913E1490913F1461E040E00A
:10C2D0000E949F6480913E1490913F1460E040E082
:10C2E0000E949F6481E001C080E029960FB6F89417
:10C2F000DEBF0FBECDBFCF91DF910895682F809133
:10C300003E1490913F140E94DA62089590933F1476
:10C3100080933E1470933D1460933C140895BC01C7
:10C3200080913E1490913F140E943A62089580914A
:10C330003E1490913F140E94DF6208951F93182FBE
:10C3400080913E1490913F1460E0412F0E949F64C1
:10C3500080913E1490913F1461E0412F0E949F64B0
:10C360001F9108956F927F928F929F92AF92BF928A
:10C37000CF92DF92EF92FF920F931F93DF93CF93B1
:10C3800000D0CDB7DEB73C014801FC0151834083AA
:10C39000738362838BE397E0938782878301015BDA
:10C3A0001F4FC80129833A830E94B05BF301EF5A03
:10C3B000FF4F8081807F8083C3018E5A9F4F0E94F0
:10C3C000B05BF301EC5AFF4F8081807F8083F301E3
:10C3D000E95AFF4F1082F301D582C482F782E682C8
:10C3E000B186A086D80129813A81822F932FFC0142
:10C3F00083E001900D928150E1F7D301AE5ABF4F17
:10C40000882D992DFC0183E001900D928150E1F778
:10C41000F301EA5AFF4F85E680830F900F90CF918A
:10C42000DF911F910F91FF90EF90DF90CF90BF9021
:10C43000AF909F908F907F906F900895FC018281C4
:10C4400093810E94551C0895FC01E25BFF4FE0813F
:10C45000FF27E7FDF095B096EE0FFF1FE80FF91FDD
:10C4600080819181DC01ED91FC910190F081E02DC2
:10C47000099508950F931F93CF93DF93EC01DC018F
:10C48000A25BBF4FEC91E63064F4EF5FEC93FF27C3
:10C49000E7FDF095B096EE0FFF1FE80FF91F7183CF
:10C4A00060838E01025B1F4FD801EC91FF27E7FDEF
:10C4B000F095B096EE0FFF1FEC0FFD1F808191816C
:10C4C000DC01ED91FC910480F581E02D0995D80106
:10C4D000EC91FF27E7FDF095B096EE0FFF1FEC0FF4
:10C4E000FD1F80819181DC01ED91FC916881798152
:10C4F0000280F381E02D41E00995DF91CF911F91FA
:10C500000F9108950F931F93CF93DF93EC018B014D
:10C51000888599850E945B81E885F985128213825E
:10C5200088859985B80141E00E942B8168857985CD
:10C53000CE010E943A62DF91CF911F910F91089531
:10C54000CF93DF93EC018A819B810E94481C8881F4
:10C55000998164E144E020E00E94696788819981C3
:10C560000E944A67888199810E944067CE01815B61
:10C570009F4F61E00E944725CE018E5A9F4F61E098
:10C580000E944725FE01EB5AFF4F1082FE01E25B3D
:10C59000FF4F8FEF8083FE01E95AFF4F10826E81BB
:10C5A0007F81CE010E943A62C85ADF4F1882DF9124
:10C5B000CF910895FC01EA5AFF4F608308950F93CD
:10C5C0001F93CF93DF93EC018C01025B1F4FD801C7
:10C5D000EC91FF27E7FDF095B096EE0FFF1FEC0FF3
:10C5E000FD1F80819181DC01ED91FC910088F18932
:10C5F000E02D0995F8018081181614F4815080838C
:10C60000FE01E25BFF4FE081FF27E7FDF095B0966A
:10C61000EE0FFF1FEC0FFD1F80819181DC01ED917A
:10C62000FC91688179810280F381E02D41E00995D8
:10C63000DF91CF911F910F910895EF92FF920F9389
:10C640001F93CF93DF93EC010E94D12D8130910590
:10C650000CF464C0833091053CF08530910509F0FD
:10C660005DC081E080934A14FE01EB5AFF4F808148
:10C67000882309F093C0FE01E25BFF4FE081FF27B2
:10C68000E7FDF095B096EE0FFF1FEC0FFD1F8081C8
:10C690009181DC01ED91FC910484F585E02D0995F3
:10C6A000882329F40E94FA1D882309F432C1FE016F
:10C6B000E25BFF4FA081A630A4F4AF5FA083BB274D
:10C6C000A7FDB095FD01B096EE0FFF1FEC0FFD1F0B
:10C6D0005F96AA0FBB1FAC0FBD1F8D919C919183DC
:10C6E00080838C819D81FE01E25BFF4FE081FF270B
:10C6F000E7FDF0957F96EE0FFF1FEC0FFD1F918376
:10C700008083DC01ED91FC910480F581E02D099599
:10C71000FE01EB5AFF4F81E0808340C0E5E5EE2E3D
:10C72000F12CEC0EFD1EF70180818823B9F18E01FA
:10C73000025B1F4FD801EC91FF27E7FDF095B09603
:10C74000EE0FFF1FEC0FFD1F80819181DC01ED9149
:10C75000FC910484F585E02D09958823F9F4CE0138
:10C760000E94DF62F7011082D801EC91FF27E7FDFC
:10C77000F095B096EE0FFF1FEC0FFD1F2081318169
:10C780008C819D812817390749F480914A148823A8
:10C7900029F0CE010E94DF6210924A14FE01E85A8D
:10C7A000FF4F8081882309F0C3C08A819B816BE49D
:10C7B00074E10E94531D882309F46CC020914B142E
:10C7C00030914C142530310519F40E94262EB0C04A
:10C7D0008E01095A1F4FF801808190E002C09595A3
:10C7E00087952A95E2F780FF9AC0FE01E25BFF4F32
:10C7F000E081FF27E7FDF095B096EE0FFF1FEC0FED
:10C80000FD1F80819181DC01ED91FC910684F7850B
:10C81000E02D0995882309F082C0F80110823AC002
:10C82000BE01665F7F4FCE010E943A6233C08E0127
:10C83000025B1F4FD801EC91FF27E7FDF095B09602
:10C84000EE0FFF1FEC0FFD1F80819181DC01ED9148
:10C85000FC910680F781E02D0995D801EC91FF2726
:10C86000E7FDF095B096EE0FFF1FEC0FFD1F8081E6
:10C870009181DC01ED91FC910084F185E02D099519
:10C88000882341F080E494E140E452E460E070E009
:10C890000E94DE8C80E494E10E94FB8C882341F0AE
:10C8A0008A819B810E94611D80E494E10E94218D18
:10C8B0008E01025B1F4FD801EC91FF27E7FDF09539
:10C8C000B096EE0FFF1FEC0FFD1F80819181DC0100
:10C8D000ED91FC91DE01AA5ABF4F0284F385E02D51
:10C8E0006C910995D801EC91FF27E7FDF095B09682
:10C8F000EE0FFF1FEC0FFD1F80819181DC01ED9198
:10C90000FC91688179810280F381E02D40E00995F6
:10C910000FC06C817D81CE010E943A62F9CE609198
:10C920004B1470914C146630710509F080CF78CFAC
:10C93000DF91CF911F910F91FF90EF900895E62F17
:10C94000F0E09F01220F331F2E0F3F1F215B3F4F4F
:10C95000820F931F642F0E94981D0895FC01E95ACD
:10C96000FF4F60830895FC01E95AFF4F81E09081F9
:10C97000911180E0089580E494E10E94DA8C08959A
:10C98000AF92BF92CF92DF92EF920F931F93DF93FC
:10C99000CF93CDB7DEB729970FB6F894DEBF0FBEA1
:10C9A000CDBF5C0149835A836B830C831D832E8327
:10C9B000CF82D886E986DC011296FE01319683E0AB
:10C9C00001900D928150E1F7D5011596FE01349644
:10C9D00083E001900D928150E1F7D5011896FE0198
:10C9E000379683E001900D928150E1F7C5010296E0
:10C9F00061E00E944725C501059661E00E94472538
:10CA0000C501089661E00E944725F5011386299625
:10CA10000FB6F894DEBF0FBECDBFCF91DF911F914F
:10CA20000F91EF90DF90CF90BF90AF900895AF92AD
:10CA3000BF92CF92DF92EF920F931F93DF93CF932A
:10CA4000CDB7DEB729970FB6F894DEBF0FBECDBFC6
:10CA50005C0149835A836B830C831D832E83CF82B1
:10CA6000D886E98622E336E0FC0121933193CF0199
:10CA70000E94B05BF5018481807F8483C5010596A7
:10CA80000E94B05BF5018781807F8783C50108968E
:10CA90000E94B05BF5018285807F8287C501498154
:10CAA0005A816B810C811D812E81CF80D884E984CD
:10CAB0000E94C06429960FB6F894DEBF0FBECDBFAA
:10CAC000CF91DF911F910F91EF90DF90CF90BF90AA
:10CAD000AF9008958F929F92AF92BF92CF92DF92C4
:10CAE000FF920F931F93DF93CF930F92CDB7DEB7D3
:10CAF0004C015B01423099F0433018F44130A1F50C
:10CB000005C0433031F0443079F506C02AE030E00A
:10CB100008C028EE33E005C020E137E202C024E679
:10CB200030E010E08AE0C82ED12C1CC0C901B6014B
:10CB30000E947F8EF62E072FD401ED91FC91C50146
:10CB4000B9010E947F8E6F2D702F0E947F8E605DD5
:10CB50000190F081E02DC401498309951F5F2F2DBD
:10CB6000302F4981141710F30F90CF91DF911F914F
:10CB70000F91FF90DF90CF90BF90AF909F908F90DC
:10CB80000895CF92DF92EF92FF920F931F93DF935E
:10CB9000CF9300D00F92CDB7DEB77C01062F172FB1
:10CBA0006E010894C11CD11CD8018C918823E1F03E
:10CBB0008A30D1F080912A1490912B149A83898322
:10CBC0008B81807F86608B83C60161E00E94981D07
:10CBD000D701ED91FC910190F081E02DC701D801C2
:10CBE0006D918D010995E0CFC8010F900F900F90C6
:10CBF000CF91DF911F910F91FF90EF90DF90CF9039
:10CC000008950F931F93CF93DF93EC01062F172FF7
:10CC100007C0E881F9810190F081E02DCE010995EE
:10CC2000F80161918F016623A1F7DF91CF911F91E8
:10CC30000F9108950F931F93CF93DF93EC018B0116
:10CC400006C0A881B981ED91FC91CE010995F8014A
:10CC50000F5F1F4F64916623A1F7DF91CF911F9162
:10CC60000F910895AF92BF92CF92DF92EF92FF9211
:10CC70000F931F93CF93DF938C01C7E0D0E028E0A0
:10CC8000E22EF12CE80EF91E95E0C92ED12CC00E33
:10CC9000D11EA62EBB24C70160E00E94981DB501DD
:10CCA0000C2E02C0759567950A94E2F7617070705A
:10CCB000C6010E94981DC70161E00E94981D95E081
:10CCC0009A95F1F7000021978FEFCF3FD80719F71A
:10CCD0000E5F1F4FC80161E00E94981D95E09A9574
:10CCE000F1F70000C80160E00E94981DDF91CF912C
:10CCF0001F910F91FF90EF90DF90CF90BF90AF907A
:10CD000008951F93CF93DF93EC01162F85E08A954A
:10CD1000F1F700001860CE01612F0E94326685E0B5
:10CD20008A95F1F70000612F677FCE010E9432667D
:10CD300085E08A95F1F70000DF91CF911F9108956A
:10CD40001F93CF93DF93EC01162F0E943266CE0122
:10CD5000612F0E948166DF91CF911F9108950F93FB
:10CD60001F93CF93DF93EC01162F442311F002E0C1
:10CD700001C000E0612F607F600FCE010E94A066BD
:10CD8000612F6295607F600FCE010E94A066DF91E7
:10CD9000CF911F910F91089540E00E94AF660895D2
:10CDA000CF92DF92EF92FF920F931F93DF93CF9377
:10CDB00000D0CDB7DEB76C016770660F660F660FE7
:10CDC000606449835A830E94CC6649815A81E42E6B
:10CDD000F52E00E010E0D7016D917D01D601ED91B7
:10CDE000FC910190F081E02DC60109950F5F1F4F66
:10CDF0000830110581F70F900F90CF91DF911F91AF
:10CE00000F91FF90EF90DF90CF900895FC01648523
:10CE1000262F246024876C600E94CC660895DF93DF
:10CE2000CF93CDB7DEB728970FB6F894DEBF0FBE0D
:10CE3000CDBFFE013196A4E3B6E028E00D9001924B
:10CE40002150E1F7FC012189241710F4422F4150B1
:10CE5000FC016787408BE42FF0E0EE0FFF1FEC0F23
:10CE6000FD1F2181260F2068622F0E94CC66289624
:10CE70000FB6F894DEBF0FBECDBFCF91DF910895FE
:10CE800062E00E94CC668FE39FE10197F1F700C05A
:10CE90000000089561E00E94CC668FE39FE1019756
:10CEA000F1F700C000000895CF93DF93EC0141E05B
:10CEB0000E94AF668F858F5F8F879A89891730F0C0
:10CEC00048894F5FCE0160E00E940F67DF91CF91EC
:10CED0000895EF92FF920F931F93DF93CF93CDB7F7
:10CEE000DEB72F970FB6F894DEBF0FBECDBF7C0123
:10CEF000423040F0DC011B968C911B9788601B969A
:10CF00008C931B97F701418B628B222329F04130D0
:10CF100019F48385846083878FEF90E7A2E08150C6
:10CF20009040A040E1F700C00000C70160E00E940F
:10CF30003266D7011B966C911B9764FD23C0C70115
:10CF400060E30E94A066EFE4F6E43197F1F700C0D9
:10CF50000000C70160E30E94A0668FE496E4019799
:10CF6000F1F700C00000C70160E30E94A066A7E5DA
:10CF7000B2E01197F1F700C00000C70160E20E9423
:10CF8000A0661EC06062C7010E94CC66EFE4F6E4B2
:10CF90003197F1F700C00000D7011B966C916062D9
:10CFA000C7010E94CC66E7E5F2E03197F1F700C0D7
:10CFB0000000D7011B966C916062C7010E94CC668D
:10CFC000F70163856062C7010E94CC6684E0D701E7
:10CFD0001C968C93C7010E940667C7010E944A678E
:10CFE00082E0F7018587C70166E00E94CC66DE011A
:10CFF0001196E4E4F6E087E001900D928150E1F7AC
:10D00000DE011896ECE3F6E088E001900D92815085
:10D01000E1F7C70160E08E010F5F1F4FA8010E947A
:10D02000D066C70160E0A8010E94D0668E01085F4B
:10D030001F4FC70161E0A8010E94D066C70161E0EF
:10D04000A8010E94D0662F960FB6F894DEBF0FBEDF
:10D05000CDBFCF91DF911F910F91FF90EF90089579
:10D0600080E00895089580E0089580E0089508958F
:10D0700060E271EA87E090E0089560E271EA87E09B
:10D0800090E0089560E573EC80E090E0089581E021
:10D09000089560E573EC80E090E0089560E573EC3E
:10D0A00080E090E0089581E00895FC016281738141
:10D0B00084819581089581E0089560E573EC80E0B6
:10D0C00090E0089560E573EC80E090E0089560E5FD
:10D0D00073EC80E090E0089560E271EA87E090E010
:10D0E00008950895FC01623029F0633041F1613008
:10D0F000B1F503C082A1882389F0878D442311F004
:10D100008F5F01C08150878F878D823014F0178E1A
:10D11000089587FF24C081E0878F089580A144236C
:10D1200011F08F5F01C0815080A380A1823014F084
:10D1300010A2089587FF13C081E080A3089581A104
:10D14000442311F08F5F01C0815081A381A18230FF
:10D1500014F011A2089587FF02C081E081A3089511
:10D16000FC0181E08483878382E0838787E0848772
:10D1700085870895FC01613019F0623019F511C0FE
:10D180008485442311F08F5F01C08150848784859A
:10D190008E3014F08DE003C01816A4F081E084876F
:10D1A00008958585442311F08F5F01C081508587E4
:10D1B00085858E301CF08DE085870895181614F053
:10D1C00081E085870895FC0182E084838783089548
:10D1D000FC0182E0848387830895FC0182E08483DC
:10D1E00087830895FC01E65AFF4F2081222329F40A
:10D1F000895A9F4FFC018081089581E00895089528
:10D20000FC0181E090E0938382831582148217826F
:10D2100016820895FC0164870895CF93DF93EC0193
:10D220001F821C828FEF8D831B82E881F981028827
:10D23000F389E02DCE0109951A82DF91CF910895EF
:10D24000FC0110868FEF818712868387CF010E94B1
:10D250000D690895FC01623029F0633071F161308D
:10D26000F1F503C082898823A1F084859585442344
:10D2700011F0019601C00197958784878485958573
:10D2800021E08530920758F184E091E0958784870A
:10D29000089586859785442311F0019601C0019772
:10D2A000978786878685978521E085309207B8F035
:10D2B00084E091E097878687089580899189442347
:10D2C00011F0019601C00197918B808B8089918923
:10D2D0008937910520F088E790E0918B808B089545
:10D2E000FC0182E0848387830895FC0181E08483CC
:10D2F00087830895EF92FF92CF93DF93EC01623022
:10D30000710571F16330710524F46115710549F0FF
:10D3100058C063307105E9F16430710509F051C0FE
:10D3200025C09C818A85981740F09C818B85891740
:10D3300020F0888591E0892788878885882319F0DF
:10D340008C8189870AC08FEF89876C81E881F98198
:10D350000688F789E02DCE01099581E08B8331C0E5
:10D360008885882371F50E9497612BC08885882362
:10D3700049F06C81E881F981028CF38DE02DCE01BA
:10D3800041E012C09C818F818917D8F48C81815033
:10D3900017C08885882351F06C81E881F981028C5F
:10D3A000F38DE02DCE0140E00995D7CF2C8130E000
:10D3B0008E8190E00197281739071CF48C818F5FCC
:10D3C0008C83DF91CF91FF90EF900895DC01623064
:10D3D0007105C1F06330710524F46115710541F0E8
:10D3E00008956330710509F16430710589F50DC048
:10D3F00014966C911497ED91FC910688F789E02DB5
:10D40000099508950E949761089514969C91149728
:10D4100017968C9117978917D8F414968C911497B6
:10D42000815014968C931497089514962C91149708
:10D4300030E016968C91169790E0019728173907DF
:10D440003CF414968C9114978F5F14968C931497D8
:10D4500008950E9497610895FC0162307105B9F04A
:10D46000633071053CF461157105C9F061307105D7
:10D47000C1F412C06330710521F06430710589F484
:10D4800003C082E090E005C012AA11AA089583E0CB
:10D4900090E092AB81AB089572AB61AB08950E94AE
:10D4A00097610895623019F0633089F405C01092D5
:10D4B0004F140E949761089580914F14813011F4A8
:10D4C00082E001C081E080934F140E94976108952B
:10D4D000623019F0633089F405C010924E140E9436
:10D4E0009761089580914E14813011F482E001C05B
:10D4F00081E080934E140E9497610895623019F084
:10D50000633049F403C00E949761089581E08093DD
:10D510004D140E94976108956115710511F40E94E0
:10D5200097610895CF93DF93EC010E94D12D9C0168
:10D53000215030402230310518F08530910511F42A
:10D5400081E001C082E08C838F831886DF91CF91C8
:10D550000895CA01613051F0613028F0623049F01D
:10D56000633081F40BC06DE07DE105C06DEF7CE1BF
:10D5700002C06AEF7CE10E941A66089566EF7CE1C2
:10D580000E941A660895CA01613051F0613028F096
:10D59000623049F0633081F40BC060EE7EE105C07B
:10D5A0006FEC7EE102C067EC7EE10E941A6608958E
:10D5B0006CEC7EE10E941A660895CA01613051F058
:10D5C000613028F0623049F0633081F40BC06BE2C7
:10D5D0007FE105C069E17FE102C066E07FE10E9472
:10D5E0001A66089565EF7EE10E941A660895CA01E1
:10D5F000613051F0613028F0623049F0633081F4DD
:10D600000BC066E57FE105C062E47FE102C06AE32A
:10D610007FE10E941A6608956FE37FE10E941A6617
:10D620000895FC016230C1F1633030F4662359F093
:10D63000613009F063C018C0633009F43EC0643043
:10D6400009F05CC04BC08585442311F08F5F01C099
:10D65000815085878585823014F01586089587FF6F
:10D660004DC081E0858708958685442311F08F5F42
:10D6700001C0815086878685873014F0168604C0E5
:10D6800087FF02C086E0868780E491E066850E947D
:10D69000F88F0E943F4008958485442311F08F5FE6
:10D6A00001C0815084878485833014F081E003C0F9
:10D6B000181624F182E0848708958785442311F0A9
:10D6C0008F5F01C0815087878785823014F017866D
:10D6D000089587FF13C081E08787089580894423D8
:10D6E00011F08F5F01C08150808B8089823014F0EF
:10D6F000108A089587FF02C081E0808B08951F93F0
:10D70000CF93DF93EC01162F6230C9F0633028F419
:10D71000662341F0613059F509C06330E9F06430A7
:10D7200031F51EC08AE491E06D851DC080E491E072
:10D730006E850E94F88F0E943F401B8318C08C8525
:10D740000E9487288C85882381F08DE79CE060E02B
:10D7500070E00E94F45E09C082E491E06F8503C02E
:10D7600080E691E068890E94F88F81E08B83DF91E9
:10D77000CF911F9108950F931F93CF93DF938C0147
:10D78000EA01623009F481C0633030F4662359F055
:10D79000613009F0EAC026C0633009F49EC06430ED
:10D7A00009F0E3C0B9C0CA016AEA7BE10E941A66C7
:10D7B000CE016BE040E00E940F67F801818588236D
:10D7C00021F4CE016FEE73E003C0CE0163EF73E08E
:10D7D0000E940166CE016EE040E00E940F67F801F2
:10D7E0008585B8C0CA016BE97BE10E941A66CE014B
:10D7F0006BE041E00E940F67F8018185813021F4E0
:10D80000CE016FEE73E003C0CE0163EF73E00E94C0
:10D810000166CE016EE041E00E940F67F801868547
:10D820008330D9F084303CF4813079F082308CF44C
:10D83000882319F19AC08530C1F0853094F0863084
:10D84000C1F0873009F091C01CC0CE016FEF73E0CA
:10D850008AC0CE0166E074E086C0CE016EE074E05E
:10D8600082C0CE0165E174E07EC0CE016CE174E05F
:10D870007AC0CE0163E274E076C0CE016AE274E061
:10D8800072C0CE0161E374E06EC0CA0160EB7BE15F
:10D890000E941A66CE016BE042E00E940F67F80119
:10D8A0008185823021F4CE016FEE73E003C0CE019A
:10D8B00063EF73E00E940166CE016EE042E00E94D9
:10D8C0000F67F8018485813021F4CE0168E374E0AC
:10D8D0004AC0CE016FE374E046C0CA0161E97BE152
:10D8E0000E941A66CE016BE043E00E940F67F801C8
:10D8F0008185833021F4CE016FEE73E003C0CE0149
:10D9000063EF73E00E940166CE016EE043E00E9487
:10D910000F67F80187851EC0CA0165E87BE10E9498
:10D920001A66CE016BE040E00E940F67F801818526
:10D93000843021F4CE016FEE73E003C0CE0163EFBB
:10D9400073E00E940166CE016EE040E00E940F6726
:10D95000F8018089882321F0CE0167EF73E003C0CE
:10D96000CE016BEF73E00E940166DF91CF911F91B2
:10D970000F9108950F931F93CF93DF938C01EA01CA
:10D980006130B1F0613030F0623091F1633009F014
:10D9900089C063C0FC0183A1882321F0CA0164ED22
:10D9A0007AE203C0CA0162EE7AE20E941A667AC085
:10D9B000FC0182A1882309F075C0CA0169EC7AE2F2
:10D9C0000E941A66CE016DE041E00E940F67F801E7
:10D9D0008185813029F4CE016FEE73E00E940166EB
:10D9E000CE0160E141E00E940F67F801878D4FC0D2
:10D9F000FC0182A1882369F0CA016DEA7AE20E94E3
:10DA00001A66CE0160E142E00E940F67F801878D3F
:10DA10000CC0CA016FEB7AE20E941A66CE0160E187
:10DA200042E00E940F67F80180A1882321F0CE0117
:10DA300067EF73E003C0CE016BEF73E00E940166F5
:10DA4000CE016DE042E00E940F67F80181858230CF
:10DA500049F5CE016FEE73E023C0CA0166EB7AE2AE
:10DA60000E941A66CE016DE043E00E940F67F80144
:10DA70008185833029F4CE016FEE73E00E94016648
:10DA8000CE0160E143E00E940F67F80181A1882385
:10DA900021F0CE0167EF73E003C0CE016BEF73E0BE
:10DAA0000E940166DF91CF911F910F910895CF934E
:10DAB000DF93EC0182E490E061E00E94E55C8C87FA
:10DAC0008AE491E061E00E94E55C8D8780E491E06A
:10DAD00060E00E94E55C8E8782E491E061E00E9454
:10DAE000E55C8F8780E691E061E00E94E55C888BD1
:10DAF000DF91CF910895623031F0633041F06130B1
:10DB000049F4089601C041960E948F610895C59618
:10DB10000E948F610895CF93DF93EC016115710529
:10DB200019F06230710591F40E94D12D8130910578
:10DB30005CF0833091051CF08530910529F4CE010D
:10DB400002960E948F6102C00E949761DF91CF917F
:10DB50000895CF93DF93EC016230710581F40E9448
:10DB6000D12D8530910531F08130910519F0823049
:10DB7000910529F4CE018C599F4F0E948F61DF914E
:10DB8000CF910895EF92FF920F931F93CF93DF935E
:10DB9000EC01653009F448C0663080F4623039F138
:10DBA000633030F46623F9F0613009F06FC01DC0B6
:10DBB0006330A9F1643009F069C034C0683009F4F9
:10DBC0004BC0693030F4663099F1673009F05EC0BF
:10DBD00032C06A3009F445C06A3008F43FC06B3087
:10DBE00009F054C048C008964FC04B964DC000E0A5
:10DBF00010E088EEE82EF12CEC0EFD1E802FF701D0
:10DC000060810E9412490F5F1F4F05301105B1F767
:10DC100091E09B83F70180818927808337C08756F5
:10DC20009F4F32C080E001C081E00E94172E2EC0BD
:10DC300082589F4F29C0FC01E751FF4F808191E03E
:10DC400089278083882311F086E901C080E00E9443
:10DC5000CB4081E08B831AC0839616C083599F4FB7
:10DC600013C0FC01E651FF4F8081882351F4CE019F
:10DC700083539F4F09C0FC01E651FF4F80818823E9
:10DC800029F4CE018F569F4F0E948F61DF91CF9173
:10DC90001F910F91FF90EF9008950F931F93CF93D3
:10DCA000DF93EC018A01653009F443C0663080F4EB
:10DCB000623051F1633030F46623F1F0613009F0E5
:10DCC0006AC01EC0633069F1643009F064C02DC0C1
:10DCD000683009F443C0693030F4663071F1673060
:10DCE00009F059C02EC06A3009F440C06A30D0F142
:10DCF0006B3009F050C045C0CA016EE87CE149C0F4
:10DD0000CA0165E87CE145C0C851DF4F888188239E
:10DD100021F0CA0164E37CE13CC0CA0166E47CE115
:10DD200038C0CA016AE67CE134C0CA016BE77CE115
:10DD300030C0CA0162E27CE12CC0CA0160EF7BE125
:10DD400028C0C751DF4F8881882321F0CA0161E0D4
:10DD50007CE11FC0CA0160E17CE11BC0CA0167E52C
:10DD60007CE117C0CA016FED7BE113C00E94C0289F
:10DD7000C651DF4F8883882349F4C8016CEB7BE1EF
:10DD800008C0C651DF4F8881882329F4C8016EEC92
:10DD90007BE10E941A66DF91CF911F910F91089548
:10DDA000CF93DF93EC010E94C028C651DF4F8883D8
:10DDB000DF91CF910895CF93DF93EC011B8685E629
:10DDC0008C870E94C0288D871E861F8681E0898BE4
:10DDD000888BDF91CF910895EF92FF920F931F935D
:10DDE000DF93CF930F92CDB7DEB78C017A016983B1
:10DDF0000E94C028F80183AB6981882311F092E06A
:10DE000002C094E0F80196836130A1F0613028F0FF
:10DE1000623011F16330E1F52AC0C70162EC7EE1A6
:10DE20000E941A66F80183A9882391F5C70167E06B
:10DE300040E00CC0C7016BEB7EE10E941A66F8015E
:10DE400083A9882329F5C70169E041E00E940F6793
:10DE5000C70166E474E01AC08823D1F4C70162ECFC
:10DE60007EE10E941A66C70167E042E00AC088238B
:10DE700079F4C7016BEB7EE10E941A66C70169E085
:10DE800043E00E940F67C7016CE474E00E940166E2
:10DE90000F90CF91DF911F910F91FF90EF90089518
:10DEA000CF93DF93EC010E94C0288BAB882311F045
:10DEB00082E08E831C821F82DF91CF910895EF92C2
:10DEC000FF920F931F93DF93CF93CDB7DEB72A97BF
:10DED0000FB6F894DEBF0FBECDBF8C01FC0112A6B9
:10DEE00081E0818F828F138A10924F147E010894F3
:10DEF000E11CF11CC7010E94DA8CD8015B96F70186
:10DF00008AE001900D928150E1F72A960FB6F894BD
:10DF1000DEBF0FBECDBFCF91DF911F910F91FF905C
:10DF2000EF900895CF93DF93EA016130F9F061300B
:10DF300028F06230F9F0633031F520C00E949F2D47
:10DF4000BC01FC0101900020E9F76E1B7F0B6B5EAA
:10DF50007F4F76956795CE0140E00E940F670E9443
:10DF60009F2DBC01CE010E9401660DC0CA016DEA61
:10DF70007CE107C0CA0165EA7CE103C0CA016BE924
:10DF80007CE10E941A66DF91CF91089580E00E94A3
:10DF9000AD1D0895EF92FF920F931F93DF93CF93E0
:10DFA0000F92CDB7DEB77C018A0169830E94D12D23
:10DFB00069816130B1F0613028F06230B9F06330CE
:10DFC00071F528C001978230910520F4C80163EEF5
:10DFD0007CE123C081E00E94AD1DC80160ED7CE1C1
:10DFE0001CC0019782309105D0F410C00197823097
:10DFF000910560F4F7018085882321F0C8016BEB5F
:10E000007CE10BC0C80163EC7CE107C0C8016DEC8A
:10E010007CE103C0C80169EC7CE10E941A660F90A4
:10E02000CF91DF911F910F91FF90EF9008950F9383
:10E030001F93DF93CF930F92CDB7DEB78C01698327
:10E040000E94D12D6981623049F0633011F1613055
:10E0500029F501978230910508F515C001978230A6
:10E06000910588F4F801808591E0892780870E94D6
:10E07000AD1DF8018085882311F40E94976181E02D
:10E08000F80183830BC080E00E94AD1D0E94976160
:10E0900005C080E00E94AD1D0E94262E0F90CF91FA
:10E0A000DF911F910F910895623019F0633051F4A0
:10E0B00003C00E94976108950E94CB280E943F40B0
:10E0C0000E9497610895FC01623029F0633091F05D
:10E0D0006130B1F403C08289882329F06485758595
:10E0E00088E591E004C0668577858AE591E00E9425
:10E0F0000E900895608971898CE591E00E940E90E0
:10E1000008950F931F93CF93DF938C01EA01613041
:10E1100071F0613030F0623059F1633009F079C04C
:10E1200059C0CA016BE57DE10E941A6672C0FC010C
:10E130008289882309F06DC0CA0166E47DE10E94EE
:10E140001A66F8018185813051F4CE016EE041E01C
:10E150000E940F67CE016FEE73E00E940166CE0150
:10E1600061E141E00E940F67F801648575854DC04B
:10E17000FC018289882371F0CA0166E47DE10E9476
:10E180001A66CE0161E142E00E940F67F8016485E2
:10E1900075850DC0CA0161E37DE10E941A66CE015A
:10E1A00061E142E00E940F67F80166857785CE0144
:10E1B00043E00E946A65F8018185823051F5CE0105
:10E1C0006EE042E00E940F67CE016FEE73E00E94A6
:10E1D00001661FC0CA0160E27DE10E941A66F80173
:10E1E0008185833051F4CE016EE043E00E940F67D9
:10E1F000CE016FEE73E00E940166CE0161E143E063
:10E200000E940F67F80160897189CE0143E00E9486
:10E210006A65DF91CF911F910F9108950F931F931E
:10E22000CF93DF938C01EA01613061F0613030F00F
:10E23000623039F1633009F04FC049C0CA016CE265
:10E2400076E248C0CA016AE176E20E941A66CE010F
:10E250006DE041E00E940F67F8018185813021F473
:10E26000CE016FEE73E003C0CE0163EF73E00E9456
:10E270000166CE0161E141E00E940F67F80164850B
:10E280001EC0CA016EE076E20E941A66CE016DE001
:10E2900042E00E940F67F8018185823021F4CE01AF
:10E2A0006FEE73E003C0CE0163EF73E00E9401667E
:10E2B000CE0161E142E00E940F67F8016585772792
:10E2C00067FD7095CE0142E00E946A6505C0CA01F3
:10E2D00066E276E20E941A66DF91CF911F910F915C
:10E2E0000895CF93DF93EB014423A1F1CB0160E0CC
:10E2F00040E00E940F67CE016BE17BE20E941A664C
:10E30000CE0160E041E00E940F67CE0166E07BE253
:10E310000E941A66CE0160E042E00E940F67CE01C3
:10E3200060E37BE20E941A66CE0160E043E00E9457
:10E330000F67CE0161EF7AE20E941A66CE0163E1B7
:10E3400043E00E940F67CE0166EF71E041E00E945A
:10E350006A6502C00E949761DF91CF910895CF93C3
:10E36000DF93EC0181E08C838F8388E591E06CED95
:10E3700070E00E94FE5C9D878C878AE591E06CEDE1
:10E3800070E00E94FE5C9F878E878CE591E064E6DA
:10E3900070E00E94FE5C998B888B0E94C0288A8B5B
:10E3A000DF91CF910895DF92EF92FF920F931F9329
:10E3B000CF93DF93EC018B018C819D8186958695AF
:10E3C000292F26952695821731F4442321F48A813A
:10E3D000882309F47FC0C8010E944A67EE24FF2405
:10E3E0008C818695869590E0880F991F880F991FDC
:10E3F0008E0D9F1D2E8130E082179307BCF5C8015A
:10E4000061E04E2D0E940F676C81E881F9816C7F7D
:10E410006E0D0488F589E02DCE01A80109950894B8
:10E42000E11CF11C84E0E816F104D1F61FC04C8118
:10E430004370C80161E00E940F676C81E881F98137
:10E440000488F589E02DCE01A80109950FC0492F58
:10E450004370C80160E00E940F67D801ED91FC9104
:10E460000190F081E02DC80160E209954C81437074
:10E47000C80160E00E940F678C818370833079F55A
:10E480002C8130E08E8190E00197281739073CF508
:10E49000D801ED91FC9111970190F081E02DC80118
:10E4A00069E00BC08C81882301F1D801ED91FC91CA
:10E4B0000190F081E02DC8016EE509958C818D8376
:10E4C0001B821A82DF91CF911F910F91FF90EF90E5
:10E4D000DF9008958B81882309F0A9CFB8CF8C8174
:10E4E00090E0837090700097E9F2D801ED91FC9173
:10E4F00011970190F081E02DC80168E0DECF0F9305
:10E500001F93CF93DF938C01EB01442341F4FC0173
:10E510008481882321F48581882309F474C0CE0185
:10E520000E944A67CE0160E040E00E940F67CE0182
:10E5300066EA7EE10E941A66F80186819781813041
:10E54000910519F182309105E9F1009709F058C061
:10E55000CE0160E041E00E940F67CE0161E97EE1FB
:10E560000E941A66CE0160E042E00E940F67CE0171
:10E570006CE77EE10E941A66CE0160E043E00E94F3
:10E580000F67CE0167E67EE139C0CE0160E041E071
:10E590000E940F67CE0162E57EE10E941A66CE01FD
:10E5A00060E042E00E940F67CE016DE37EE10E94D1
:10E5B0001A66CE0160E043E00E940F67CE0168E278
:10E5C0007EE11CC0CE0160E041E00E940F67CE01F9
:10E5D00063E17EE10E941A66CE0160E042E00E94A3
:10E5E0000F67CE016EEF7DE10E941A66CE0160E0FA
:10E5F00043E00E940F67CE0169EE7DE10E941A663A
:10E60000F80114821582DF91CF911F910F91089527
:10E61000CF93DF93EC018EE591E060E00E94E55C32
:10E6200090E021E082FF20E02F8F9C01217030706C
:10E6300029A321E081FF20E028A30E94C0288AA30B
:10E640008DEF9BE00E94AA5F181619061CF08F8DB3
:10E650008823D9F48DE79CE00E94AA5F181619065A
:10E660001CF088A1882389F489E79FE00E94AA5FB3
:10E67000181619061CF089A1882339F481E08BA3B0
:10E6800081E08A87DF91CF9108951BA2F9CF4F9245
:10E690005F926F927F928F929F92AF92BF92CF9232
:10E6A000DF92EF92FF920F931F93DF93CF93CDB73B
:10E6B000DEB7A6970FB6F894DEBF0FBECDBF6C01D4
:10E6C0007B01042FDC011F968C911F978823B1F5E5
:10E6D0008DEF9BE00E94C15F882361F48DE79CE091
:10E6E0000E94C15F882331F489E79FE00E94C15FE7
:10E6F000882321F181E0F6018787128AC70160E053
:10E7000040E00E940F6782E491E061E00E94E55CD6
:10E7100091E0882309F490E0D60151969C9351979B
:10E7200081E050968C9350971F968C911F97882369
:10E7300029F0C70161E574E00E940166002309F435
:10E7400081C0C7010E944A67C70160E040E00E94A3
:10E750000F67F6018785882351F0C70166E674E0EC
:10E760000E940166D60152961C92529736C00E94B2
:10E770003F4081E0F601808B0E94D12D83309105CE
:10E7800034F48130910574F4009739F026C0833059
:10E790009105F1F08530910501F50E949F2DBC0196
:10E7A000C70119C00E94CE2D082F192FD8016D91D5
:10E7B0008D016E3209F48DC2662309F48AC2D70135
:10E7C000ED91FC910190F081E02DC7010995EECF0C
:10E7D000C7016FE674E00E940166F6018585882313
:10E7E00099F0C70160E041E00E940F67C70160E750
:10E7F0007DE10E941A66C70160E042E00E940F6757
:10E80000C70165E87DE112C0C70160E041E00E94F8
:10E810000F67C70164EC7DE10E941A66C70160E0E2
:10E8200042E00E940F67C7016FEA7DE10E941A660D
:10E83000C70160E043E00E940F67C7016AE97DE11C
:10E840000E941A66CE0101960E946887D6011F9623
:10E850008C911F97882309F41BC18DEF9BE00E94C8
:10E86000C15F882359F08DEF9BE00E94DB5F5C0164
:10E870008DEF9BE00E94AA5F8C0104C000E010E0D5
:10E88000AA24BB248DE79CE00E94C15F882361F02D
:10E890008DE79CE00E94DB5FA80EB91E8DE79CE02F
:10E8A0000E94AA5F080F191F89E79FE00E94C15FBD
:10E8B000882381F089E79FE00E94DB5F880F991F22
:10E8C000A80EB91E89E79FE00E94AA5F880F991FD2
:10E8D000080F191FA114B10409F042C0F6011786F0
:10E8E000C70160E040E00E940F67C70160E77DE17B
:10E8F0000E941A66C70160E040E00E940F670E9414
:10E90000D12D8330910534F4813091056CF400975A
:10E9100021F020C085309105E9F40E949F2DBC01B3
:10E92000C7010E94016616C00E94CE2D082F192F24
:10E93000D8016D918D016E3209F4D6C1662309F4B8
:10E94000D3C1D701ED91FC910190F081E02DC70179
:10E950000995EECF0E943F4081E0F601808B98C080
:10E96000101611060CF04DC098012A193B09A90197
:10E9700037FF04C044275527421B530BCA01880F99
:10E98000991F840F951F880F991F880F991FB80131
:10E990000E94938E4B01D60151968C9151978823FA
:10E9A00091F12801662457FC6094762CB9018827E0
:10E9B00077FD8095982F2FEF30E040E050E00E94E7
:10E9C000608EA30192010E94C88E022FB501882794
:10E9D00077FD8095982F2FEF30E040E050E00E94C7
:10E9E000608EA30192010E94C88E802F60E0422FAA
:10E9F000F60120890E94513FD60150961C925097F3
:10EA000002C088249924F601828990E0881699062C
:10EA100068F4C70168E040E00E940F67C70166E73D
:10EA200074E00E940166D60152961C92F60162893A
:10EA3000685FC70140E00E940F67D60152960C91B3
:10EA4000529710E00BC0D701ED91FC910190F0813D
:10EA5000E02DC7016FEF09950F5F1F4F08151905CE
:10EA600090F3F601828A868591E08927868788233C
:10EA700031F0C70163E874E00E94016609C0D70164
:10EA8000ED91FC910190F081E02DC7016FEF0995A8
:10EA9000F6018385833009F46AC0843030F4813014
:10EAA00011F1823008F044C00AC0853009F4AFC0CB
:10EAB000853008F498C0863009F0FDC0D2C0D60178
:10EAC0001D968C911D97882309F0F5C0C7016CE055
:10EAD00041E00E940F678DEF9BE00E94B05F8C01C8
:10EAE0008DEF9BE08CC0F6018585882309F0E3C09B
:10EAF0008DEF9BE00E942561882309F0DCC08DEF3B
:10EB00009BE00E94AA5F8C01009771F0C7016FE043
:10EB100041E00E940F67C7016EE874E00E94016641
:10EB2000C70160E141E055C0C7016FE041E093C01B
:10EB3000C7016CE042E00E940F67D6011D968C91E0
:10EB40001D97813019F08DE69CE002C08DEE9BE0B0
:10EB500040960E94B05F8C01F6018585813019F0E6
:10EB60008DE69CE002C08DEE9BE0409648C0D60149
:10EB70001D968C911D97813019F08DE69CE002C0A6
:10EB80008DEE9BE040960E942561882309F093C09A
:10EB9000C70160E142E00E940F67F6018585813080
:10EBA00019F08DE69CE002C08DEE9BE040960E943D
:10EBB000AA5F8C01009799F0C7016FE042E00E94C4
:10EBC0000F67C7016EE874E00E940166C70160E14B
:10EBD00042E00E940F67C701B80143E05DC0C70172
:10EBE0006FE042E038C0C7016CE043E00E940F676D
:10EBF00089E79FE00E94B05F8C0189E79FE00E9457
:10EC00002561882341F3C70165E874E052C089E7B4
:10EC10009FE00E942561882309F04DC0C70160E193
:10EC200043E00E940F6789E79FE00E94AA5F8C0182
:10EC3000009771F0C7016FE043E00E940F67C701C2
:10EC40006EE874E00E940166C70160E143E0C1CF55
:10EC5000C7016FE043E00E940F67C70164E974E0F9
:10EC600028C00E94D12DD6011F962C911F972223D8
:10EC700011F5019782309105F0F41C968C911C9748
:10EC8000843668F4C70161E140E00E940F67F60135
:10EC90006485C70170E042E00E946A650CC084365A
:10ECA00051F4C70160E140E00E940F67C7016AE9C3
:10ECB00074E00E940166D6011B968C911B978F5FB2
:10ECC0001B968C931B978730D0F01B961C921B973A
:10ECD00016C0C70160E140E00E940F67C70169EDFF
:10ECE0007DE10E941A6679CDC70160E140E00E9493
:10ECF0000F67C70169ED7DE10E941A662BCEA696CB
:10ED00000FB6F894DEBF0FBECDBFCF91DF911F913C
:10ED10000F91FF90EF90DF90CF90BF90AF909F90BA
:10ED20008F907F906F905F904F900895CF93DF9377
:10ED3000EC0180EF99E4A2E0B0E08A839B83AC838E
:10ED4000BD8381E090E09AAB89AB83E090E09F8344
:10ED50008E831DAA81E088AB92E0988789878A8795
:10ED60008B871C868D870E946C8F64E170E00E9407
:10ED7000938E8BAB0E946C8F64E070E00E94938E48
:10ED80008CABDF91CF910895BF92CF92DF92EF923B
:10ED9000FF920F931F93CF93DF93EC018B0188A910
:10EDA000882341F4E881F9810480F581E02DCE01CA
:10EDB000099502C0442329F1C8010E944A67CC2466
:10EDC00019C0DF011496AA0FBB1FAC0FBD1FEE0FB9
:10EDD000FF1FEC0FFD1FC8016C9141850E940F675A
:10EDE000D801ED91FC910190F081E02DC8016FE414
:10EDF0000995C394EC2DF0E08E819F81E817F90707
:10EE000004F3C8016BA94CA90E940F67D801ED91CA
:10EE1000FC910190F081E02DC8016AE20995AE8174
:10EE2000BF81FD0131971396AA0FBB1FAC0FBD1F09
:10EE3000EE0FFF1FEC0FFD1FC8016C9141850E9472
:10EE40000F67D801ED91FC910190F081E02DC80190
:10EE500060E209954E81E42FE150FF27E7FDF09530
:10EE60003596EE0FFF1FEC0FFD1F80E090E004C011
:10EE700032912291338322830196242F281B27FF6E
:10EE8000F7CF89A99AA982309105E9F083309105DD
:10EE900049F08130910589F48885992787FD9095FF
:10EEA000019605C08885992787FD9095439664E172
:10EEB00070E00E94938E888710C08985992787FD0E
:10EEC0009095039605C08985992787FD90950196B1
:10EED00064E070E00E94938E8987C8016885498547
:10EEE0000E940F67D801ED91FC910190F081E02D17
:10EEF000C8016FE40995BB24B39480E4C82E8BE469
:10EF0000D82E8CE4E82EF12C22C0FC013496EE0FB2
:10EF1000FF1FEC0FFD1F20812417C1F4FC01EE0F31
:10EF2000FF1FEC0FFD1F91858985981779F418AAAA
:10EF3000C80161E041E00E940F67C8016EED7DE10C
:10EF40000E941A66CA82DB82EC82FD82B3948B2D0A
:10EF500090E02E813F81488582179307B4F28BA9F8
:10EF60004817C1F599858CA99817A1F58DA98F5FD0
:10EF70008DAB90E083709070009781F42F5F3F4FCE
:10EF80003F832E838A819B81AC81BD8188589341C8
:10EF9000A040B0408A839B83AC83BD830E946C8F6A
:10EFA00064E170E00E94938E8BAB0E946C8F64E0F2
:10EFB00070E00E94938E482F8CABC8016BA90E9411
:10EFC0000F67D801ED91FC910190F081E02DC8010F
:10EFD0006AE20995DF91CF911F910F91FF90EF9019
:10EFE000DF90CF90BF900895AF92BF92CF92DF9203
:10EFF000EF92FF920F931F93DF93CF930F92CDB7B2
:10F00000DEB75C017B01FC01C380865A9F4F4983B8
:10F010000E94FB8C49818823A9F1F501E75AFF4F33
:10F020008081882379F110820E9497612EC0F501BA
:10F03000EA5AFF4F8081882341F185010C5F1F4F01
:10F04000DD24F501EA5AFF4F1082C7010E944A678A
:10F0500014C0C701F50162814C2D0E940F67C701E2
:10F06000B8010E94C1658C01FC0180818A3029F4BD
:10F070000F5F1F4F0894C11CD11CF80180818823A9
:10F0800041F703C0442399F2D8CF0F90CF91DF917D
:10F090001F910F91FF90EF90DF90CF90BF90AF90B6
:10F0A0000895CF93DF93EC011A8E83E49BE069E12E
:10F0B00070E04FE050E00E946F37198EDF91CF91E2
:10F0C0000895EF92FF920F931F93DF93CF93CDB7E5
:10F0D000DEB764970FB6F894DEBF0FBECDBF8C01CC
:10F0E0007B01CE0101960E942C3EE114F10429F02F
:10F0F00082E0E816F10469F528C0F801818D8F5F80
:10F10000818F813019F08630E1F410C083E49BE0F8
:10F1100060E070E040E050E00E946F3782E00E94C3
:10F12000172EF801818D8F5F818F13C083E49BE0E0
:10F1300060E070E040E050E00E946F370E9497610D
:10F1400008C081E0F801828F04C0C80140960E9487
:10F150008F6164960FB6F894DEBF0FBECDBFCF911E
:10F16000DF911F910F91FF90EF900895CF93DF9360
:10F17000EC01FC01E75BFF4F108283E49BE069E157
:10F1800070E04FE050E00E946F371A8210924D14E9
:10F1900010924E141C821B82DF91CF9108950F9321
:10F1A0001F93CF93DF938C01EB01442339F4DC01EF
:10F1B0005A968C915A97882309F450C0CE0160E08A
:10F1C00040E00E940F67F801818D8330A1F0843008
:10F1D00028F4882341F08230E9F509C0843079F0C1
:10F1E0008530C1F521C0CE0162E377E220C0CE01B7
:10F1F00061EE76E21CC0CE0160E976E218C083E4DD
:10F200009BE060E070E040E050E00E946F37C80192
:10F2100002960E948F61D80159968C9159978F5F01
:10F2200059968C93599716C0CE016FE376E20E94EF
:10F230001A668FEF99E6A8E181509040A040E1F76F
:10F2400000C0000083E49BE069E170E04FE050E023
:10F250000E946F37D8015A961C925A97DF91CF912E
:10F260001F910F9108950F931F93CF93DF938C01FC
:10F27000EB01442339F4FC01E75BFF4F80818823D5
:10F2800009F4C5C0CE0160E040E00E940F67D801DC
:10F2900012968C911297843009F445C085306CF435
:10F2A000813011F182301CF48823D1F0ACC082305F
:10F2B00091F1833009F0A7C032C0893009F480C0D1
:10F2C0008A303CF4863009F44AC0873009F09BC08C
:10F2D00055C08A3009F481C08C3009F094C08FC0C9
:10F2E000CE016CE57AE203C0CE016BE07AE20E94C7
:10F2F0001A668FEF93EDA0E381509040A040E1F7B4
:10F3000000C0000083E49BE069E170E04FE050E062
:10F310000E946F3778C0CE016AEB79E2E8CFCE0168
:10F3200069E679E2E4CFCE0168E179E20E941A66EB
:10F3300083E49BE069E170E04FE050E00E946F37AA
:10F340008FEF93EDA0E381509040A040E1F700C023
:10F35000000086E591E061E00E94F88F54C0C8018A
:10F360008F5B9F4F0E948F618FEF93EDA0E38150E1
:10F370009040A040E1F700C0000026C080914E14EC
:10F38000882321F4CE0167EC78E210C0813049F483
:10F39000CE0166E778E20E941A6684E0F801828373
:10F3A00007C0823029F4CE0165E278E20E941A6635
:10F3B0008FEF99E6A8E181509040A040E1F7A0CFFF
:10F3C000C801C9960E948F61D80112968C9112973C
:10F3D0008F5F12968C93129716C080914D148823DC
:10F3E00051F0CE0163E877E20E941A66F80182814B
:10F3F0008F5F82837ECFCE0164ED77E278CF0E946B
:10F40000262E0E949761F801E75BFF4F1082DF9183
:10F41000CF911F910F9108958F929F92AF92BF92BB
:10F42000CF92DF92EF92FF920F931F93DF93CF93D0
:10F4300000D000D0CDB7DEB78C01C62E623009F403
:10F4400043C0633009F47EC0613009F07DC082E6BC
:10F4500091E040E050E0BA010E941F5D4B015C0169
:10F46000F8016485772767FD70956750704088279D
:10F4700077FD8095982F0E94341927E837E44CEBEC
:10F4800052E40E94DA172DEC3CEC4CEC5DE30E9458
:10F49000DA1720E030E040E251E40E94DA170E94DF
:10F4A0009419680D791D8A1D9B1D69837A838B834E
:10F4B0009C83CE01019662E671E044E050E00E9438
:10F4C000EE8FF801C38240C086E691E040E050E054
:10F4D000BA010E941F5D6B017C01F80165857727E9
:10F4E00067FD709567507040882777FD8095982F4D
:10F4F0000E94341927E837E44CEB52E40E94DA17F3
:10F500002DEC3CEC4CEC5DE30E94DA1720E030E09F
:10F5100040E251E40E94DA170E9494196C0D7D1D9F
:10F520008E1D9F1D69837A838B839C83CE010196F8
:10F5300066E671E044E050E00E94EE8F81E0F80161
:10F54000838302C00E9497610F900F900F900F90DD
:10F55000CF91DF911F910F91FF90EF90DF90CF90AF
:10F56000BF90AF909F908F9008951F93CF93DF939C
:10F57000EC0187E598E09983888385E297E09D8791
:10F580008C8789EC96E09F878E8714E01C8BCE01D8
:10F590000E960E940D691E8318868FEF89871A8642
:10F5A0008B87CE010E940D69DF91CF911F91089545
:10F5B000FC01678D660F80A1680F660F81A1680F3F
:10F5C0008EE591E00E94F88F08950F931F93DF93CB
:10F5D000CF930F92CDB7DEB78C01613009F473C0C1
:10F5E000613038F0623009F476C0633009F07AC0D7
:10F5F00072C0FC0183A191E0892783A3882309F4C9
:10F6000049C083E49BE00E94063788E591E060E012
:10F6100070E00E94FE5CF801278D332727FD3095AE
:10F62000829FB001839F700D929F700D11248DEF0A
:10F630009BE00E94F45EF80182A18823B1F48AE580
:10F6400091E060E070E00E94FE5CF80120A13327A9
:10F6500027FD3095829FB001839F700D929F700DA2
:10F6600011248DE79CE00E94F45E8CE591E060E05F
:10F6700070E00E94FE5CF80121A1332727FD309540
:10F68000829FB001839F700D929F700D112489E7B6
:10F690009FE010C08DEF9BE060E070E00E94F45EA0
:10F6A0008DE79CE060E070E00E94F45E89E79FE0F7
:10F6B00060E070E00E94F45E0E949761C8010C96C1
:10F6C0000E948F610FC069830E94D87AF80113A24B
:10F6D0006981628307C0C8010E94D87AF80113A229
:10F6E00081E082830F90CF91DF911F910F91089558
:10F6F0004F925F926F927F928F929F92AF92BF9242
:10F70000CF92DF92EF92FF920F931F93DF93CF93ED
:10F71000CDB7DEB768970FB6F894DEBF0FBECDBF8A
:10F720002C01DC0156968C915697882349F420E8E9
:10F730003BEB40E050E02D8B3E8B4F8B588F08C049
:10F7400080E894E4AFEFBFEF8D8B9E8BAF8BB88FCB
:10F7500000D000D0ADB7BEB711961D921D921D927C
:10F760001C9214973E010894611C711CC30140E077
:10F7700050E0BA0100E010E09801CC24DD247601CD
:10F780008824992454010E942D3E0F900F900F90D1
:10F790000F90F2016489C30170E00E948B3E2D89B5
:10F7A0003E894F89588DDC012D933D934D935C9399
:10F7B0001397C30140E053EA61EE71E12FE10E942B
:10F7C000A447EBE1F0E04E0E5F1EC2010E94218DC6
:10F7D000C20140E053EA61EE71E10E94DE8C68965E
:10F7E0000FB6F894DEBF0FBECDBFCF91DF911F9152
:10F7F0000F91FF90EF90DF90CF90BF90AF909F90D0
:10F800008F907F906F905F904F900895CF93DF938C
:10F810000E94DF45C0E0D0E08C2F60E00E941249DA
:10F820002196C530D105C1F7DF91CF910895EF92B0
:10F83000FF920F931F93DF93CF93CDB7DEB76497FB
:10F840000FB6F894DEBF0FBECDBF8C017B01CE0199
:10F8500001960E942C3EE114F10429F082E0E816A2
:10F86000F104C9F534C0F80183898530A1F18F5FB7
:10F87000838B83E49BE060E070E040E050E00E9416
:10F880006F37F8018389893019F08B30E1F409C0B2
:10F89000F801808D882329F08AE0838BC8010296C5
:10F8A00018C0C8010E94067C8DEF9BE060E070E00C
:10F8B0000E94F45E8DE79CE060E070E00E94F45EE0
:10F8C0000E94976108C081E0F80182A704C0C801C6
:10F8D0000A960E948F6164960FB6F894DEBF0FBE41
:10F8E000CDBFCF91DF911F910F91FF90EF900895C1
:10F8F0002F923F924F925F926F927F928F929F9240
:10F90000AF92BF92CF92DF92EF92FF920F931F932D
:10F91000DF93CF93CDB7DEB7AF970FB6F894DEBFC6
:10F920000FBECDBF3C012B014FA700D000D0ADB71B
:10F93000BEB711961D921D921D921C921497CE0176
:10F94000019640E050E0BA0100E010E09801CC24BC
:10F95000DD2476018824992454010E942D3E0F90C5
:10F960000F900F900F90F3018389853009F023C128
:10F970008589813019F0882331F009C07DE6272E72
:10F980007CE0372E04C06DEE262E6BE0362EC101D2
:10F9900040960E948E5F882321F1D30153968C916B
:10F9A00053978F5F53968C93539701E09A960C93DD
:10F9B0000E943F40F301028FC3010E94787BD30174
:10F9C00099968C919997882309F0F5C058968C9157
:10F9D0005897882309F0EFC088E053968C9353978B
:10F9E000EAC0C3014B960E94FB8C8823C9F0C20178
:10F9F0000E944A67C20160E040E00E940F67C201B6
:10FA00006DEB75E20E941A6683E49BE069E170E0A9
:10FA10004FE050E00E946F378AE0F301838BCBC048
:10FA2000D30155968C915597813019F0882331F088
:10FA300009C0EDE6FCE0FAA7E9A704C08DEE9BE063
:10FA40009AA789A789A59AA540960E94DB5F5C01C9
:10FA5000D30155968C915597813019F0882331F058
:10FA600009C0EDE6FCE0FCA7EBA704C08DEE9BE02F
:10FA70009CA78BA78BA59CA540960E94AA5FFC0122
:10FA80009C012A193B09A90137FF04C044275527C7
:10FA9000421B530B64E170E0469FC001479F900DED
:10FAA000569F900D1124BF010E94938E262ED301E4
:10FAB00059968C915997882379F17F010027F7FC9B
:10FAC0000095102FB901882777FD8095982F2FEF8B
:10FAD00030E040E050E00E94608EA80197010E9453
:10FAE000C88ED22EB501882777FD8095982F2FEFED
:10FAF00030E040E050E00E94608EA80197010E9433
:10FB0000C88E8D2D60E0422FF301228D0E94513F5F
:10FB1000D3015A961C925A97F30180A5281668F4CF
:10FB2000C20160E043E00E940F67C2016FE974E028
:10FB30000E940166D30198961C92C201F30160A550
:10FB400043E00E940F67D30198960C91989710E0BC
:10FB5000E22CFF240BC0D201ED91FC910190F081C9
:10FB6000E02DC2016FEF09950F5F1F4F0E151F05A6
:10FB700094F3F30120A686A197A1019697A386A3EB
:10FB800087309105C4F085A191E0892785A388235A
:10FB900031F0C20163E874E00E94016609C0D2013D
:10FBA000ED91FC910190F081E02DC2016FEF09957C
:10FBB000F30117A216A2D30153968C915397883064
:10FBC000C9F4C3014B960E94FB8C882399F0F30182
:10FBD000808D882339F089E0838BC30102960E94CF
:10FBE0008F6108C08AE0D30153968C93539781E0CC
:10FBF0009A968C93BFA5BB2329F4F30182A5882391
:10FC000009F4E7C1C20160E040E00E940F67D30140
:10FC100098961C92989753968C915397843009F438
:10FC2000EFC0853060F4813009F486C08130D0F0B7
:10FC3000823009F48FC0833009F0C7C18FC087308C
:10FC400009F432C1883038F4853009F4FAC08630BE
:10FC500009F0BBC106C1883009F43BC18A3009F004
:10FC6000B4C14DC1F3018589813019F0882331F089
:10FC700009C08DE69CE09EA78DA704C0ADEEBBE059
:10FC8000BEA7ADA78DA59EA540966CED70E00E9425
:10FC9000F45EF3018789882331F08DE79CE06CEDF9
:10FCA00070E00E94F45ED30158968C915897882397
:10FCB00001F157968C915797882321F0C2016CE689
:10FCC00075E203C0C2016AEC74E20E941A6683E422
:10FCD0009BE069E170E04FE050E00E946F378FEFEA
:10FCE00093EDA0E381509040A040E1F700C00000F8
:10FCF00015C0C20166E373E20E941A66D3019896AA
:10FD00001C9282E491E061E00E94E55C91E088232E
:10FD100009F490E0F301918F85E0838B8301055E08
:10FD20001F4FC8010E94218DC80140E053EA61EED7
:10FD300071E10E94DE8C49C1D30157968C9157978F
:10FD4000882321F0C2016BE175E22CC1C2016AE790
:10FD500074E228C1C20169E274E224C1C20168ED03
:10FD600073E20E941A668E010B5E1F4FC8010E944B
:10FD70001146DE011196F80184E101900D92815047
:10FD8000E1F72E010894411C511CC20162E070E0B1
:10FD90000E948B3EFC0180819181A281B381883ECB
:10FDA000F3E09F07F0E0AF07F0E0BF07BCF4C2014B
:10FDB00062E070E00E948B3E20E63AEE40E050E0C8
:10FDC000DC012D933D934D935C931397C20140E466
:10FDD0005BE46CE470E02FE10E94A4478FEF93EDA9
:10FDE000A0E381509040A040E1F700C0000083E410
:10FDF0009BE069E170E04FE050E00E946F37E5C0A2
:10FE0000C20167E873E20E941A668FEF9BE7A2E9DE
:10FE100081509040A040E1F700C00000D30153960C
:10FE20008C9153978F5F53968C9382E491E061E0BD
:10FE30000E94E55C91E0882309F490E0F301918F42
:10FE4000C4C0D30158968C915897882321F0C201E1
:10FE500067E873E203C0C20166E373E20E941A66B8
:10FE6000B4C0F3018789882359F08489833021F451
:10FE7000C20165EE72E21BC0C20162EF71E217C0FF
:10FE8000D30156968C915697882321F0C20164E9DC
:10FE900072E20DC0C20163E472E20E941A66F301CD
:10FEA00083898F5F838B05C0C20161EA71E20E9482
:10FEB0001A6683E49BE069E170E04FE050E00E9445
:10FEC0006F378FEF91EEA4E081509040A040E1F7B2
:10FED0007AC0D30158968C915897882321F0C2019B
:10FEE00060E571E25FC0F3018689882321F0C201D9
:10FEF0006FEF70E257C0C2016EEA70E253C0C301F7
:10FF00000E94067C80914F14882301F5D3015796F7
:10FF10008C9157978823B1F054968C9154978330E5
:10FF200089F484E054968C93549798961C929897F1
:10FF300086E053968C93C3010E94787BC20162EFE6
:10FF400071E230C0C2016BEB7FE12CC0813061F403
:10FF5000C2016DE570E20E941A66C3010E94787BBF
:10FF600087E0F301838B20C08230F1F4D3015796F0
:10FF70008C915797882399F054968C91549783309D
:10FF800071F484E054968C93549787E053968C9345
:10FF9000C3010E94787BC2016AE67FE103C0C2010F
:10FFA0006CE070E20E941A6683E49BE069E170E015
:10FFB0004FE050E00E946F378FEF93EDA0E3815048
:10FFC0009040A040E1F700C00000D3019A961C9237
:10FFD0009A97AF960FB6F894DEBF0FBECDBFCF9104
:10FFE000DF911F910F91FF90EF90DF90CF90BF9026
:10FFF000AF909F908F907F906F905F904F903F90C9
:020000021000EC
:100000002F9008950F931F93CF93DF93EC018B01F3
:100010001B8A1F8A188E80E691E061E00E94E55CF1
:1000200091E0882309F490E099A70230110511F1BD
:10003000033011053CF40115110589F0013011055B
:1000400009F512C00430110541F004301105ACF07F
:1000500005301105B9F481E08F8B81E0888F1D8A0E
:1000600083E08C8B81E004C081E08D8B94E09C8BDD
:100070008E8B08C01D8A83E003C081E08D8B84E0F5
:100080008C8B1E8ADF91CF911F910F910895CF9392
:10009000DF93EC01613061F0613028F0623069F08B
:1000A0006330C9F40FC02896CE0160E070E00EC046
:1000B0002896CE0162E070E009C02896CE0161E08A
:1000C00070E004C02896CE0163E070E00E940280D8
:1000D000CE010E948F61DF91CF910895EF92FF9240
:1000E0000F931F93DF93CF93CDB7DEB764970FB60F
:1000F000F894DEBF0FBECDBF8C017B01CE0101960F
:100100000E942C3EE114F10431F082E0E816F10483
:1001100009F063C009C0F80182818F5F82830CC03F
:1001200081E00E94172E59C0F8018281815082839C
:1001300087FD1282F80182818830B9F08B30B9F1E5
:10014000853009F045C083E49BE060E070E040E06A
:1001500050E00E946F37F80182818F5F8283809127
:100160004E148130E9F683E0DCCF83E49BE060E06D
:1001700070E040E050E00E946F37F80182818F5FAD
:10018000828382E490E061E00E94E55C9801225F56
:100190003F4F813021F4C90164E070E003C0C90120
:1001A00065E070E00E940280C8010E960EC083E4F4
:1001B0009BE060E070E040E050E00E946F37F801A3
:1001C00082818F5F8283C80105960E948F6105C07E
:1001D000F801E75BFF4F81E0808364960FB6F894E7
:1001E000DEBF0FBECDBFCF91DF911F910F91FF906A
:1001F000EF90089527ED37E0FC013183208324E060
:1002000026830E940D69089529EB37E0FC013183B4
:10021000208324E026830E940D6908952BE937E0AE
:10022000FC013183208324E026830E940D69089518
:10023000CF93DF93EC018DE797E099838883CE011C
:1002400008960E94363384E08E83CE010E940D69A9
:10025000DF91CF910895CF93DF93262F372FD901C8
:10026000FC01EB5AFF4F07C03081EC01C30FD11DD9
:100270002C833F5F30832D912223B1F720812135DC
:1002800029F4FC01EC5AFF4F108204C0FC01E20F7C
:10029000F11D1482FC01E95AFF4F442339F010820A
:1002A0008A5A9F4F21E0FC01208302C081E08083B5
:1002B000DF91CF910895EF92FF920F931F93DF93F9
:1002C000CF93CDB7DEB72A970FB6F894DEBF0FBE37
:1002D000CDBF8C01FC01138212821482EB5AFF4FB6
:1002E0001082FC01EA5AFF4F81E08083F801E85A4E
:1002F000FF4F80837E010894E11CF11CC7010E941E
:10030000DA8CD801A65ABF4FF7018AE001900D920E
:100310008150E1F7F801E95AFF4F1082F801E75ADE
:10032000FF4F10822A960FB6F894DEBF0FBECDBFE6
:10033000CF91DF911F910F91FF90EF9008951F9340
:10034000CF93DF93EC01142F70E080E090E020E485
:1003500032E44FE050E00E94608EAB01BC01CE0160
:10036000865A9F4F0E94DE8CC75ADF4F1883DF9159
:10037000CF911F910895AF92BF92CF92DF92EF92EB
:10038000FF920F931F93DF93CF93CDB7DEB76497A0
:100390000FB6F894DEBF0FBECDBF8C017B01CE013E
:1003A00001960E9411460E94DF45F80182819381E7
:1003B0008130910531F0F4E1AF2EB12CC12CD12C5C
:1003C00006C0E8EEAE2EE3E0BE2EC12CD12CF80123
:1003D000868197810097D9F4F3E0EF16F10469F074
:1003E00084E0E816F10471F0E1E0EE16F10409F0A2
:1003F00074C0F801F782E6824AC0CE01019660E03F
:1004000070E05CC0CE01019660E070E047C08130D2
:10041000910549F5F2E0EF16F104B9F083E0E81632
:10042000F10434F4E1E0EE16F10409F056C00AC01C
:10043000F3E0EF16F10469F084E0E816F10409F046
:100440004CC00CC082E090E01FC0F80117821682F9
:100450001EC0CE01019661E070E030C0CE01019671
:1004600061E070E01BC082309105B9F5F3E0EF1652
:10047000F10481F084E0E816F104E1F0E2E0EE1628
:10048000F10459F581E090E0F8019783868381E0DB
:10049000858323C0CE01019662E070E00E948B3E0E
:1004A000FC0120813181428153812A0D3B1D4C1D6D
:1004B0005D1D0FC0CE01019662E070E00E948B3E90
:1004C000FC0120813181428153812A193B094C0969
:1004D0005D092083318342835383CE01019648EE28
:1004E00053E060E070E00E94DC4664960FB6F8943A
:1004F000DEBF0FBECDBFCF91DF911F910F91FF9057
:10050000EF90DF90CF90BF90AF900895CF93DF939F
:100510006115710531F077FD13C06530710584F404
:100520000DC00E949761C0E0D0E08C2F60E00E9477
:1005300012492196C530D105C1F702C00E94BB8186
:10054000DF91CF91089529EC36E0FC0131832083BF
:1005500024E026830E940D6908951F93CF93DF93B3
:10056000EC018BE298E0998388838BE098E09B8391
:100570008A8314E018871A868FEF8B871C868D87F5
:10058000CE0102960E940D6989EC96E0998B888BCA
:100590001E8BCE0140960E940D69DF91CF911F9175
:1005A00008950F931F93CF93DF93EC018DE896E0AE
:1005B0009983888385E297E09987888789EC96E01C
:1005C0009B878A8714E0188BCE010A960E940D69DA
:1005D00081E597E09C8F8B8FCE0183960E944C33F0
:1005E000CE0183599F4F2DE636E0FC0131832083F5
:1005F000FE01ED58FF4F25E02083FE01EB58FF4F31
:100600001082FE01EA58FF4F0FEF0083FE01E95808
:10061000FF4F1082FE01E858FF4F00830E940D69D2
:10062000CE0182589F4F25E037E0FC0131832083C3
:10063000FE01EC57FF4F1083FE01EA57FF4F108277
:10064000FE01E957FF4F0083FE01E857FF4F10827C
:10065000FE01E757FF4F00830E940D69CE018F56C0
:100660009F4F27EE36E0FC0131832083FE01E956DF
:10067000FF4F10830E940D69CE0187569F4F0E9445
:100680001881CE0183539F4F0E94AD828CE08E83F0
:10069000FE01E851FF4F1082FE01E751FF4F10822B
:1006A000CE010E940D69DF91CF911F910F910895A6
:1006B000CF93DF93EC018BEA96E0998388838FE4F4
:1006C00096E099878887CE0108960E940D69CE0131
:1006D00041960E94B57ACE01C5960E94D18284E0EF
:1006E0008E83CE010E940D69DF91CF9108952FE492
:1006F00036E0FC01318320830E940D690895CF927A
:10070000DF92EF92FF920F931F93DF93CF9300D06E
:10071000CDB7DEB78C01CDB6DEB619820E94AE43EE
:10072000009729F081E0F801808770E037C04DB76D
:100730005EB7405450400FB6F8945EBF0FBE4DBF39
:100740000DB71EB70F5F1F4F70E07E010894E11CCC
:10075000F11CC80160E4A7017A830E944641F801B8
:1007600020817A812223D1F02E32B1F02981A80193
:10077000420F511D9A01FA0133974081433761F4CA
:10078000F90132974081433339F421503040F90167
:100790002081273609F47F5F0097D9F2872F0FB6A3
:1007A000F894DEBE0FBECDBE0F900F90CF91DF91BB
:1007B0001F910F91FF90EF90DF90CF900895CF930E
:1007C000DF93EC0118860E947F838F5F8E83DF9119
:1007D000CF9108956F927F928F929F92AF92BF9226
:1007E000CF92DF92EF92FF920F931F93DF93CF93FD
:1007F0000F92CDB7DEB7862E7A01A22E6DB67EB6E9
:100800000E94AE43009709F051C08DB79EB7805447
:1008100090400FB6F8949EBF0FBE8DBF0DB71EB7A8
:100820000F5F1F4FBB2499246E010894C11CD11C7B
:1008300024C0C80160E4A6010E944641F80120815D
:100840002223A1F1009711F42E3299F32981A801F6
:10085000420F511DFA0133972081233751F7FA01D6
:1008600032972081233329F741505040FA012081EB
:100870002736F9F60097D1F4B3948B2D90E08816C3
:100880009906BCF689818A1510F08A2D8150D8010D
:10089000F70190E003C02D9121939F5F9817D8F343
:1008A000F701E80FF11D108281E001C080E00FB672
:1008B000F8947EBE0FBE6DBE0F90CF91DF911F9159
:1008C0000F91FF90EF90DF90CF90BF90AF909F90EF
:1008D0008F907F906F9008950F931F93DF93CF9326
:1008E0000F92CDB7DEB78C01262F30E0FC01868158
:1008F00090E00197281739071CF00E94976122C0E9
:1009000069830E94D12D6981009729F083E49BE0DF
:1009100064EB74E015C069830E94CE2DAC01C80160
:1009200069812FE10E94EA83882321F00E94D62D5D
:10093000009741F00E94976183E49BE069EC74E0CA
:100940000E94A4370F90CF91DF911F910F910895CE
:100950009F92AF92BF92CF92DF92EF92FF920F934E
:100960001F93DF93CF93CDB7DEB78A01ADB6BEB686
:10097000CDB6DEB6DC0118962C911897222321F013
:10098000CA016AE67BE10DC0462F50E0FC012681DA
:1009900030E0215030404217530734F0C8016BE774
:1009A0007BE10E941A662EC02DB73EB7235130401E
:1009B0000FB6F8943EBF0FBE2DBFEDB6FEB608943D
:1009C000E11CF11CA70123E10E94EA83882349F47A
:1009D0000E94976183E49BE069EC74E00E94A43775
:1009E00011C0A3E19A2ED7016D917D01662351F0CC
:1009F000D801ED91FC910190F081E02DC80109959D
:100A00009A9489F78C2D9D2D0FB6F8949EBF0FBE3A
:100A10008DBF0FB6F894BEBE0FBEADBECF91DF91B5
:100A20001F910F91FF90EF90DF90CF90BF90AF900C
:100A30009F900895DF92EF92FF920F931F93CF93B1
:100A4000DF93EC018B01D42ECB010E94FF31B5E581
:100A5000EB2EF12CEC0EFD1E882361F1F701908145
:100A6000913540F5F801228133812115310511F1CD
:100A7000FE01E90FF11D84839F5FF7019083C80198
:100A80000E94FF31E9CFFE01EC5AFF4F108204C0F3
:100A9000FE01E80FF11D1482FE01E95AFF4FDD202F
:100AA00031F01082CA5ADF4F81E088830AC081E0AA
:100AB000808307C0FE01EB5AFF4F8081803541F7EC
:100AC000E2CFDF91CF911F910F91FF90EF90DF90D8
:100AD0000895FC01148E138E128E118E108E0CC090
:100AE000A82FB0E01696AA0FBB1FAE0FBF1F11961E
:100AF0001C921E928F5F808F808D843088F3108EC1
:100B000020E030E0A901248B358B468B578B10A257
:100B1000178E0895FC01168E158E20E030E0A90195
:100B200020873187428753872483358346835783C1
:100B300020833183428353830E9469850895FC0199
:100B4000168E158E20E030E0A9012087318742877C
:100B5000538724833583468357832083318342839D
:100B600053830E94698508952F923F924F925F921E
:100B70006F927F928F929F92AF92BF92CF92DF92AD
:100B8000EF92FF920F931F93DF93CF9300D000D08B
:100B900000D0CDB7DEB79E838D83FC01E58CF68C4B
:100BA000E61AF70A838D948D8E0D9F1D948F838F87
:100BB000F1E081309F0734F080E091E0ED81FE812B
:100BC000948F838FED81FE81838D948DFFEF803034
:100BD0009F0734F480E09FEFED81FE81948F838F37
:100BE000B701882777FD8095982F0E943419ED81F1
:100BF000FE8120813181428153810E94DA17562E75
:100C0000472E382E292EED81FE81638D748D882725
:100C100077FD8095982F0E943419ED81FE81248103
:100C20003581468157810E94DA1769837A838B83E5
:100C30009C83ED81FE81818D928D6701C81AD90A4E
:100C4000608C772483010A5F1F4F000F111F0E0F66
:100C50001F1FF80160817181882777FD8095982F8B
:100C60000E9434199B01AC01ED81FE816489758974
:100C7000868997890E94A917B62EA72E982E892EAD
:100C8000F801D182C082B601882777FD8095982F20
:100C90000E9434199B01AC01D501F4016B2F7A2F0E
:100CA0008F2F9E2F0E947C17262F372F482F592FCA
:100CB000ED81FE81248B358B468B578B0894611C0C
:100CC000711CF3E06F227724ED81FE81608E208518
:100CD0003185428553850E94DA17062FC72EB82E1C
:100CE000A92EED81FE81F28EE18EA2019101652F88
:100CF000742F832F922FB981AA81EB809C802B2F98
:100D00003A2F4E2D592D0E947C17F501202F3C2D96
:100D10004F2F5E2F0E947C170E949419660F771F39
:100D2000ED81FE8170A3678FCB0126960FB6F894F4
:100D3000DEBF0FBECDBFCF91DF911F910F91FF900E
:100D4000EF90DF90CF90BF90AF909F908F907F906B
:100D50006F905F904F903F902F9008950F931F9347
:100D6000CF93DF93EC018B018D8D9E8D86179707B6
:100D700029F0CE010E9469851E8F0D8FDF91CF91E2
:100D80001F910F910895FC01838D948D0895FC01AE
:100D900064897589868997890E949419CB01089581
:100DA000FC01878D90A10895FC0180818032A0F420
:100DB0008181862798E02CE8869508F482279A9509
:100DC000D9F781838081DF01A80FB11D12966C9342
:100DD000129780818F5F80830895FC0111821082B9
:100DE00012A214A213A20895FC011182108212A271
:100DF00014A213A20895FC011182108212A214A25F
:100E000013A20895CF93DF93EC018BA19CA10097CF
:100E100061F4653D19F481E090E035C019821882D3
:100E20001AA21CA21BA281E037C08BA19CA1813019
:100E3000910581F4603238F46DA38DA18823B1F05F
:100E400082E090E020C0198218821AA21CA21BA284
:100E500082E022C08BA19CA18230910551F4CE0189
:100E60000E94D48698818DA19817B8F083E090E015
:100E70000AC08BA19CA18330910579F489818617E2
:100E800029F484E090E09CA38BA307C01982188208
:100E90001AA21CA21BA283E08AA3DF91CF9108951E
:100EA000FC01E60FF11D82810895E62FF0E0DC01E0
:100EB000AE0FBF1F12962C9112973196E80FF91FB3
:100EC0003281932F80E030E0282B392BC90108951F
:100ED000FC011182108212A214A213A215A208957D
:100EE000FC011182108212A214A213A215A208956D
:100EF000FC0183A194A1009731F481E090E094A3D8
:100F000083A385ED089583A194A18130910539F4DF
:100F1000808190819923A1F022E030E01CC083A160
:100F200094A18230910579F495A1DF01A90FB11D3B
:100F300012968C9112979F5F95A32081921778F05B
:100F400023E030E008C083A194A18330910531F4FF
:100F5000818124E030E034A323A3089580E0089544
:100F60000E94D48608950F931F93DF93CF930F921F
:100F7000CDB7DEB78C0179830E94D486C801798110
:100F8000672F0E94D4860F90CF91DF911F910F9110
:100F90000895CF92DF92EF92FF920F931F936C010F
:100FA0007A018B01642F0E94D4865527412F302F60
:100FB0002F2DC601622F0E94D48698014427552701
:100FC000C601622F0E94D486E12EFF24002711273C
:100FD000C6016E2D0E94D4861F910F91FF90EF9055
:100FE000DF90CF900895FC01118210820895FC01DA
:100FF0007183608312821382148215821682178293
:101000001086118612861386148615861686178614
:10101000108A118A128A138A148A158A168A178AE4
:10102000108E118E0895CF93DF93EC014E875F876A
:10103000688B798B222329F08E859F85A889B989B1
:101040000CC08E859F85A889B9892A813B814C81F6
:101050005D81821B930BA40BB50B8E8B9F8BA88F8E
:10106000B98F81E08A8F8E899F89A88DB98D00976D
:10107000A105B10529F08881998161E00E94CB89A1
:101080008E899F89A88DB98DB7FF10C08E899F89E1
:10109000A88DB98DB095A095909581959F4FAF4F34
:1010A000BF4F8E8B9F8BA88FB98F1A8EDF91CF91F8
:1010B0000895CF93DF93EC016A8F8881998161E075
:1010C0000E94CB8981E090E0A0E0B0E08E8B9F8B06
:1010D000A88FB98FDF91CF910895FC01428353838C
:1010E000648375830895FC01808191810E94CB897E
:1010F0000895FC01808191810E94D18A0895EF9228
:10110000FF920F931F93CF93DF93EC017A018B0132
:101110002A893B894C895D898E899F89A88DB98DE3
:10112000820F931FA41FB51F8A8B9B8BAC8BBD8B2B
:101130008A899B89AC89BD89B7FD48C06A8D888141
:1011400099810E94BE898A899B89AC89BD898E1943
:101150009F09A00BB10B8A8B9B8BAC8BBD8B2A8D0F
:1011600088819981222319F00E94D18902C00E94AE
:10117000ED89182F8A8D882381F0112329F4888125
:10118000998161E00E94C7892A813B814C815D8100
:101190002F5F3F4F4F4F5F4F0FC0112329F48881BE
:1011A000998161E00E94C7892A813B814C815D81E0
:1011B00021503040404050402A833B834C835D8324
:1011C0008881998160E00E94C78901C010E081E0B8
:1011D0008127DF91CF911F910F91FF90EF9008959C
:1011E000EF92FF920F931F93CF93DF93EC017A015D
:1011F0008B018E899F89A88DB98D0097A105B105B6
:1012000009F45CC02A893B894C895D898E899F8954
:10121000A88DB98D820F931FA41FB51F8A8B9B8B3E
:10122000AC8BBD8B8A899B89AC89BD89B7FD44C0D5
:101230006A8D888199810E94BE898A899B89AC893F
:10124000BD898E199F09A00BB10B8A8B9B8BAC8B30
:10125000BD8B2A8D88819981222319F00E94D18922
:1012600002C00E94ED899A8D992379F0882331F587
:101270008881998161E00E94C7898A819B81AC81C4
:10128000BD810196A11DB11D0EC08823B9F48881CE
:10129000998161E00E94C7898A819B81AC81BD816F
:1012A0000197A109B1098A839B83AC83BD8388819F
:1012B000998160E00E94C78981E001C080E0DF91F0
:1012C000CF911F910F91FF90EF9008958F929F9271
:1012D000AF92BF92CF92DF92EF92FF920F931F9344
:1012E000CF93DF93FC01DC01EB0183E009900D92C9
:1012F0008150E1F7DF011396842F952FEC0183E0F5
:1013000009900D928150E1F7DF011696822F932FFD
:10131000EC0183E009900D928150E1F7DF0119960D
:10132000802F912FEC0183E009900D928150E1F71D
:10133000EF012C968E2D9F2DDC0183E00D900992FC
:101340008150E1F7EF012F968C2D9D2DDC0183E07C
:101350000D9009928150E1F781E0828B138AB28E61
:10136000A18EDF91CF911F910F91FF90EF90DF90B1
:10137000CF90BF90AF909F908F900895FC012389EC
:10138000222311F021E062270E94981D0895039600
:101390000E94981D089521E0622706960E94981DDC
:1013A00008950F931F93CF93DF93EC018C01075F98
:1013B0001F4FC8010E94B65B882349F4C8010E94F0
:1013C0004E259A89992321F091E0892701C080E078
:1013D000DF91CF911F910F9108950F931F93CF939A
:1013E000DF93EC018C01045F1F4FC8010E94B65BC4
:1013F000882349F4C8010E944E259A89992321F037
:1014000091E0892701C080E0DF91CF911F910F917A
:101410000895EF92FF920F931F93DF93CF93CDB771
:10142000DEB763970FB6F894DEBF0FBECDBF8C0159
:10143000DE011196E3E8F0E183E101900D92815025
:10144000E1F77E010894E11CF11CC7016EE5F8018B
:101450002785308941890E942245F801238D348DEA
:10146000818D928D820F931F60E00E94E55C682F52
:10147000C701F8012785308941890E94BF44C7010F
:101480000E94944463960FB6F894DEBF0FBECDBFA2
:10149000CF91DF911F910F91FF90EF900895DF9210
:1014A000EF92FF920F931F93CF93DF93EC01F62EF1
:1014B00061E00E944725CE01039661E00E94472526
:1014C0008E010A5F1F4FC80161E00E94981DC8018C
:1014D00061E00E9447250F2D10E0C80104969C8F03
:1014E0008B8FCE010E94098A898D9A8D60E00E94BF
:1014F000E55CD82E898D9A8D029660E00E94E55CAD
:10150000E82EC801880F991F880F991F0E964FEF7C
:101510005FEF6FEF7FEF0E941F5D6D8B7E8B8F8B78
:10152000988FE7FE0AC08E2D90E00F2C02C0959593
:1015300087950A94E2F7817001C081E08A8B8D2D36
:1015400090E002C095958795FA94E2F781709070CB
:101550008B8B8E01075F1F4FC8010E94B65B8823EB
:1015600041F4C80160E00E944725C8016A890E94D1
:10157000981D8E01045F1F4FC8010E94B65B88232F
:1015800041F4C80160E00E944725C8016A890E94B1
:10159000981DDF91CF911F910F91FF90EF90DF90F9
:1015A0000895EF92FF920F931F93DF93CF93CDB7E0
:1015B000DEB763970FB6F894DEBF0FBECDBF7C01D8
:1015C000062FDE011196E3E8F0E183E101900D9230
:1015D0008150E1F7CE0101966EE5F701278530894C
:1015E00041890E942245602F073708F066E78E0187
:1015F0000F5F1F4FC801F7012785308941890E947D
:10160000BF44C8010E94944463960FB6F894DEBFAD
:101610000FBECDBFCF91DF911F910F91FF90EF9043
:101620000895FF920F931F93CF93DF93EC018FB731
:10163000F894FF800D811E819F8191111F828FBFC1
:10164000BE016B5F7F4FAE01495F5F4F8C810E948F
:10165000585B882331F1FF2039F1888990E0FC0143
:101660003496EE0FFF1FEC0FFD1F118300830196D0
:1016700083709070888BC801029723E08D3F92079A
:1016800038F080E094E09B838A8323E030E00EC052
:10169000C80169890E94978B9B838A8320E030E090
:1016A00005C021E030E002C022E030E0C901DF9156
:1016B000CF911F910F91FF900895FC011382128228
:1016C00084810E94215B0895FC018DE898E091835C
:1016D000808364831782108A418B1186108613865B
:1016E000128615861486178616860895DF93CF9383
:1016F00000D000D0CDB7DEB7682F772767FD709593
:10170000660F771F660F771F6B5B744DCE010196D6
:1017100044E050E00E947C8F69817A818B819C81BA
:101720000F900F900F900F90CF91DF910895CF926F
:10173000DF92EF92FF920F931F93CF93DF93EC0111
:1017400029E0E22E93E1C92EDD2402E010E08E2D87
:101750000E94768B2E2D332727FD3095C617D7078D
:101760005CF48D2D992787FD9095820F931FB8010A
:101770000E94938ECE2C0AC08C2D992787FD9095C0
:10178000820F931FB8010E94938EDE2CE62ED61690
:10179000F4F28D2D0E94768B8B017C018C2D0E94A2
:1017A000768B9B01AC01DD2019F4C017D107E4F062
:1017B0008C2D833119F42C173D07B4F0C01BD10BCD
:1017C0004E195F09C49FC001C59F900DD49F900D15
:1017D0001124B901601B710B0E94938E6E0D7F1D49
:1017E0006F3F710519F014F06FEF70E0CB01DF91DE
:1017F000CF911F910F91FF90EF90DF90CF900895C0
:10180000DF93CF930F92CDB7DEB7BC01CE01019627
:1018100041E050E00E94D88F81E099819F3F09F418
:1018200080E00F90CF91DF91089584E890E00E94CE
:10183000008C809350140895CF93DF93EC010496AD
:1018400061E00E944725CE01079661E00E9447258E
:10185000CE010A9660E00E9447251B821A82DF9122
:10186000CF910895000000000000000000000895DE
:101870007F928F929F92AF92BF92CF92DF92EF9220
:10188000FF920F931F93CF93DF937C0134E0832E5D
:10189000912C880E991EC40160E00E94981D0E9440
:1018A000328C27E0C22ED12CCE0CDF1CC60160E0AA
:1018B0000E94981D0E94328C00E010E07724C0E066
:1018C000D0E09AE0A92EB12CAE0CBF1CC60161E09D
:1018D0000E94981D0E94328CC80101978A309105A0
:1018E00048F4CC0FDD1FC5010E944E25882361F00E
:1018F000C1600AC00D30110539F4C5010E944E25A2
:10190000882311F077247394C60160E00E94981D2B
:101910000E94328C0F5F1F4F00311105B9F6C401D0
:1019200061E00E94981D0E94328CC60160E00E9416
:10193000981D772041F080E094E0F7019383828343
:1019400023E030E005C0F701D383C28320E030E01C
:10195000C901DF91CF911F910F91FF90EF90DF9020
:10196000CF90BF90AF909F908F907F900895E5E9C2
:10197000F8E0DC011196FC93EE931496FB0163E012
:1019800001900D926150E1F7DC011796FA0143E0F6
:1019900001900D924150E1F7DC011A96F90183E0C4
:1019A00001900D928150E1F7089583E49BE00E943D
:1019B0008F360895FC01108211820895EF92FF92F4
:1019C0000F931F93CF93DF93EC017A018B0181E09A
:1019D000888319820E94D58C6A837B838C839D8344
:1019E000EE82FF8208871987DF91CF911F910F91B7
:1019F000FF90EF900895CF93DF93EC0188818823C7
:101A0000C9F089818823B1F40E94D58C2A813B8159
:101A10004C815D81621B730B840B950B2E813F8182
:101A200048855985621773078407950718F018824F
:101A300081E089838981DF91CF910895FC01108233
:101A40000895FC0111820895FC018281882371F4BC
:101A50001092C50080E18093C40082E08093C000B2
:101A600088E18093C10086E08093C2000895DF93EF
:101A7000CF9300D00F92CDB7DEB780912C14909108
:101A80002D149A8389838B81807F83608B83CE0121
:101A9000019660E00E94981D0F900F900F90CF91DB
:101AA000DF910895DF93CF9300D00F92CDB7DEB7CB
:101AB00080912C1490912D149A8389838B81807F3F
:101AC00083608B83CE01019661E00E94981D0F9088
:101AD0000F900F90CF91DF910895CF93DF93EC019A
:101AE000598348836A831B8204960E94F486CE0140
:101AF0008A960E946887CE010E94248DDF91CF9143
:101B00000895CF93DF93EC018B818823B9F088810E
:101B100099818130910549F40E94528D85E38A951F
:101B2000F1F7000081E080935214CE018A960E9462
:101B300078879A81992311F48093C600DF91CF9121
:101B40000895DF93CF93CDB7DEB729970FB6F894FA
:101B5000DEBF0FBECDBFFC0163838281882359F4B1
:101B6000662321F08091C100806C03C08091C10088
:101B70008F738093C100808191818130910589F5B7
:101B800080912C1490912D149A8389838B81807F6E
:101B900083608B83CE01019661E00E94472580918E
:101BA0002C1490912D149D838C838E81807F826074
:101BB0008E83CE01049661E00E94472580912C140B
:101BC00090912D1498878F838985807F8260898783
:101BD000CE01079660E00E94981D0E94378D1092FA
:101BE000521429960FB6F894DEBF0FBECDBFCF9129
:101BF000DF9108951F920F920FB60F920BB60F92BE
:101C000011242F933F934F935F936F937F938F9301
